
lab_exam.elf:     file format elf32-littlearm

Sections:
Idx Name          Size      VMA       LMA       File off  Algn
  0 .isr_vector   00000188  08000000  08000000  00010000  2**0
                  CONTENTS, ALLOC, LOAD, READONLY, DATA
  1 .text         00003a6c  08000190  08000190  00010190  2**4
                  CONTENTS, ALLOC, LOAD, READONLY, CODE
  2 .rodata       00000090  08003bfc  08003bfc  00013bfc  2**2
                  CONTENTS, ALLOC, LOAD, READONLY, DATA
  3 .ARM.extab    00000000  08003c8c  08003c8c  00020010  2**0
                  CONTENTS
  4 .ARM          00000008  08003c8c  08003c8c  00013c8c  2**2
                  CONTENTS, ALLOC, LOAD, READONLY, DATA
  5 .preinit_array 00000000  08003c94  08003c94  00020010  2**0
                  CONTENTS, ALLOC, LOAD, DATA
  6 .init_array   00000004  08003c94  08003c94  00013c94  2**2
                  CONTENTS, ALLOC, LOAD, DATA
  7 .fini_array   00000004  08003c98  08003c98  00013c98  2**2
                  CONTENTS, ALLOC, LOAD, DATA
  8 .data         00000010  20000000  08003c9c  00020000  2**2
                  CONTENTS, ALLOC, LOAD, DATA
  9 .bss          00004058  20000010  08003cac  00020010  2**2
                  ALLOC
 10 ._user_heap_stack 00000600  20004068  08003cac  00024068  2**0
                  ALLOC
 11 .ARM.attributes 00000030  00000000  00000000  00020010  2**0
                  CONTENTS, READONLY
 12 .debug_info   000146e9  00000000  00000000  00020040  2**0
                  CONTENTS, READONLY, DEBUGGING, OCTETS
 13 .debug_abbrev 000029e8  00000000  00000000  00034729  2**0
                  CONTENTS, READONLY, DEBUGGING, OCTETS
 14 .debug_aranges 00001040  00000000  00000000  00037118  2**3
                  CONTENTS, READONLY, DEBUGGING, OCTETS
 15 .debug_ranges 00000f48  00000000  00000000  00038158  2**3
                  CONTENTS, READONLY, DEBUGGING, OCTETS
 16 .debug_macro  00022362  00000000  00000000  000390a0  2**0
                  CONTENTS, READONLY, DEBUGGING, OCTETS
 17 .debug_line   00011dbf  00000000  00000000  0005b402  2**0
                  CONTENTS, READONLY, DEBUGGING, OCTETS
 18 .debug_str    000d2682  00000000  00000000  0006d1c1  2**0
                  CONTENTS, READONLY, DEBUGGING, OCTETS
 19 .comment      00000053  00000000  00000000  0013f843  2**0
                  CONTENTS, READONLY
 20 .debug_frame  000043ac  00000000  00000000  0013f898  2**2
                  CONTENTS, READONLY, DEBUGGING, OCTETS

Disassembly of section .text:

08000190 <__do_global_dtors_aux>:
 8000190:	b510      	push	{r4, lr}
 8000192:	4c05      	ldr	r4, [pc, #20]	; (80001a8 <__do_global_dtors_aux+0x18>)
 8000194:	7823      	ldrb	r3, [r4, #0]
 8000196:	b933      	cbnz	r3, 80001a6 <__do_global_dtors_aux+0x16>
 8000198:	4b04      	ldr	r3, [pc, #16]	; (80001ac <__do_global_dtors_aux+0x1c>)
 800019a:	b113      	cbz	r3, 80001a2 <__do_global_dtors_aux+0x12>
 800019c:	4804      	ldr	r0, [pc, #16]	; (80001b0 <__do_global_dtors_aux+0x20>)
 800019e:	f3af 8000 	nop.w
 80001a2:	2301      	movs	r3, #1
 80001a4:	7023      	strb	r3, [r4, #0]
 80001a6:	bd10      	pop	{r4, pc}
 80001a8:	20000010 	.word	0x20000010
 80001ac:	00000000 	.word	0x00000000
 80001b0:	08003be4 	.word	0x08003be4

080001b4 <frame_dummy>:
 80001b4:	b508      	push	{r3, lr}
 80001b6:	4b03      	ldr	r3, [pc, #12]	; (80001c4 <frame_dummy+0x10>)
 80001b8:	b11b      	cbz	r3, 80001c2 <frame_dummy+0xe>
 80001ba:	4903      	ldr	r1, [pc, #12]	; (80001c8 <frame_dummy+0x14>)
 80001bc:	4803      	ldr	r0, [pc, #12]	; (80001cc <frame_dummy+0x18>)
 80001be:	f3af 8000 	nop.w
 80001c2:	bd08      	pop	{r3, pc}
 80001c4:	00000000 	.word	0x00000000
 80001c8:	20000014 	.word	0x20000014
 80001cc:	08003be4 	.word	0x08003be4

080001d0 <strlen>:
 80001d0:	4603      	mov	r3, r0
 80001d2:	f813 2b01 	ldrb.w	r2, [r3], #1
 80001d6:	2a00      	cmp	r2, #0
 80001d8:	d1fb      	bne.n	80001d2 <strlen+0x2>
 80001da:	1a18      	subs	r0, r3, r0
 80001dc:	3801      	subs	r0, #1
 80001de:	4770      	bx	lr

080001e0 <__aeabi_uldivmod>:
 80001e0:	b953      	cbnz	r3, 80001f8 <__aeabi_uldivmod+0x18>
 80001e2:	b94a      	cbnz	r2, 80001f8 <__aeabi_uldivmod+0x18>
 80001e4:	2900      	cmp	r1, #0
 80001e6:	bf08      	it	eq
 80001e8:	2800      	cmpeq	r0, #0
 80001ea:	bf1c      	itt	ne
 80001ec:	f04f 31ff 	movne.w	r1, #4294967295
 80001f0:	f04f 30ff 	movne.w	r0, #4294967295
 80001f4:	f000 b96e 	b.w	80004d4 <__aeabi_idiv0>
 80001f8:	f1ad 0c08 	sub.w	ip, sp, #8
 80001fc:	e96d ce04 	strd	ip, lr, [sp, #-16]!
 8000200:	f000 f806 	bl	8000210 <__udivmoddi4>
 8000204:	f8dd e004 	ldr.w	lr, [sp, #4]
 8000208:	e9dd 2302 	ldrd	r2, r3, [sp, #8]
 800020c:	b004      	add	sp, #16
 800020e:	4770      	bx	lr

08000210 <__udivmoddi4>:
 8000210:	e92d 47f0 	stmdb	sp!, {r4, r5, r6, r7, r8, r9, sl, lr}
 8000214:	9d08      	ldr	r5, [sp, #32]
 8000216:	4604      	mov	r4, r0
 8000218:	468c      	mov	ip, r1
 800021a:	2b00      	cmp	r3, #0
 800021c:	f040 8083 	bne.w	8000326 <__udivmoddi4+0x116>
 8000220:	428a      	cmp	r2, r1
 8000222:	4617      	mov	r7, r2
 8000224:	d947      	bls.n	80002b6 <__udivmoddi4+0xa6>
 8000226:	fab2 f282 	clz	r2, r2
 800022a:	b142      	cbz	r2, 800023e <__udivmoddi4+0x2e>
 800022c:	f1c2 0020 	rsb	r0, r2, #32
 8000230:	fa24 f000 	lsr.w	r0, r4, r0
 8000234:	4091      	lsls	r1, r2
 8000236:	4097      	lsls	r7, r2
 8000238:	ea40 0c01 	orr.w	ip, r0, r1
 800023c:	4094      	lsls	r4, r2
 800023e:	ea4f 4817 	mov.w	r8, r7, lsr #16
 8000242:	0c23      	lsrs	r3, r4, #16
 8000244:	fbbc f6f8 	udiv	r6, ip, r8
 8000248:	fa1f fe87 	uxth.w	lr, r7
 800024c:	fb08 c116 	mls	r1, r8, r6, ip
 8000250:	ea43 4301 	orr.w	r3, r3, r1, lsl #16
 8000254:	fb06 f10e 	mul.w	r1, r6, lr
 8000258:	4299      	cmp	r1, r3
 800025a:	d909      	bls.n	8000270 <__udivmoddi4+0x60>
 800025c:	18fb      	adds	r3, r7, r3
 800025e:	f106 30ff 	add.w	r0, r6, #4294967295
 8000262:	f080 8119 	bcs.w	8000498 <__udivmoddi4+0x288>
 8000266:	4299      	cmp	r1, r3
 8000268:	f240 8116 	bls.w	8000498 <__udivmoddi4+0x288>
 800026c:	3e02      	subs	r6, #2
 800026e:	443b      	add	r3, r7
 8000270:	1a5b      	subs	r3, r3, r1
 8000272:	b2a4      	uxth	r4, r4
 8000274:	fbb3 f0f8 	udiv	r0, r3, r8
 8000278:	fb08 3310 	mls	r3, r8, r0, r3
 800027c:	ea44 4403 	orr.w	r4, r4, r3, lsl #16
 8000280:	fb00 fe0e 	mul.w	lr, r0, lr
 8000284:	45a6      	cmp	lr, r4
 8000286:	d909      	bls.n	800029c <__udivmoddi4+0x8c>
 8000288:	193c      	adds	r4, r7, r4
 800028a:	f100 33ff 	add.w	r3, r0, #4294967295
 800028e:	f080 8105 	bcs.w	800049c <__udivmoddi4+0x28c>
 8000292:	45a6      	cmp	lr, r4
 8000294:	f240 8102 	bls.w	800049c <__udivmoddi4+0x28c>
 8000298:	3802      	subs	r0, #2
 800029a:	443c      	add	r4, r7
 800029c:	ea40 4006 	orr.w	r0, r0, r6, lsl #16
 80002a0:	eba4 040e 	sub.w	r4, r4, lr
 80002a4:	2600      	movs	r6, #0
 80002a6:	b11d      	cbz	r5, 80002b0 <__udivmoddi4+0xa0>
 80002a8:	40d4      	lsrs	r4, r2
 80002aa:	2300      	movs	r3, #0
 80002ac:	e9c5 4300 	strd	r4, r3, [r5]
 80002b0:	4631      	mov	r1, r6
 80002b2:	e8bd 87f0 	ldmia.w	sp!, {r4, r5, r6, r7, r8, r9, sl, pc}
 80002b6:	b902      	cbnz	r2, 80002ba <__udivmoddi4+0xaa>
 80002b8:	deff      	udf	#255	; 0xff
 80002ba:	fab2 f282 	clz	r2, r2
 80002be:	2a00      	cmp	r2, #0
 80002c0:	d150      	bne.n	8000364 <__udivmoddi4+0x154>
 80002c2:	1bcb      	subs	r3, r1, r7
 80002c4:	ea4f 4e17 	mov.w	lr, r7, lsr #16
 80002c8:	fa1f f887 	uxth.w	r8, r7
 80002cc:	2601      	movs	r6, #1
 80002ce:	fbb3 fcfe 	udiv	ip, r3, lr
 80002d2:	0c21      	lsrs	r1, r4, #16
 80002d4:	fb0e 331c 	mls	r3, lr, ip, r3
 80002d8:	ea41 4103 	orr.w	r1, r1, r3, lsl #16
 80002dc:	fb08 f30c 	mul.w	r3, r8, ip
 80002e0:	428b      	cmp	r3, r1
 80002e2:	d907      	bls.n	80002f4 <__udivmoddi4+0xe4>
 80002e4:	1879      	adds	r1, r7, r1
 80002e6:	f10c 30ff 	add.w	r0, ip, #4294967295
 80002ea:	d202      	bcs.n	80002f2 <__udivmoddi4+0xe2>
 80002ec:	428b      	cmp	r3, r1
 80002ee:	f200 80e9 	bhi.w	80004c4 <__udivmoddi4+0x2b4>
 80002f2:	4684      	mov	ip, r0
 80002f4:	1ac9      	subs	r1, r1, r3
 80002f6:	b2a3      	uxth	r3, r4
 80002f8:	fbb1 f0fe 	udiv	r0, r1, lr
 80002fc:	fb0e 1110 	mls	r1, lr, r0, r1
 8000300:	ea43 4401 	orr.w	r4, r3, r1, lsl #16
 8000304:	fb08 f800 	mul.w	r8, r8, r0
 8000308:	45a0      	cmp	r8, r4
 800030a:	d907      	bls.n	800031c <__udivmoddi4+0x10c>
 800030c:	193c      	adds	r4, r7, r4
 800030e:	f100 33ff 	add.w	r3, r0, #4294967295
 8000312:	d202      	bcs.n	800031a <__udivmoddi4+0x10a>
 8000314:	45a0      	cmp	r8, r4
 8000316:	f200 80d9 	bhi.w	80004cc <__udivmoddi4+0x2bc>
 800031a:	4618      	mov	r0, r3
 800031c:	eba4 0408 	sub.w	r4, r4, r8
 8000320:	ea40 400c 	orr.w	r0, r0, ip, lsl #16
 8000324:	e7bf      	b.n	80002a6 <__udivmoddi4+0x96>
 8000326:	428b      	cmp	r3, r1
 8000328:	d909      	bls.n	800033e <__udivmoddi4+0x12e>
 800032a:	2d00      	cmp	r5, #0
 800032c:	f000 80b1 	beq.w	8000492 <__udivmoddi4+0x282>
 8000330:	2600      	movs	r6, #0
 8000332:	e9c5 0100 	strd	r0, r1, [r5]
 8000336:	4630      	mov	r0, r6
 8000338:	4631      	mov	r1, r6
 800033a:	e8bd 87f0 	ldmia.w	sp!, {r4, r5, r6, r7, r8, r9, sl, pc}
 800033e:	fab3 f683 	clz	r6, r3
 8000342:	2e00      	cmp	r6, #0
 8000344:	d14a      	bne.n	80003dc <__udivmoddi4+0x1cc>
 8000346:	428b      	cmp	r3, r1
 8000348:	d302      	bcc.n	8000350 <__udivmoddi4+0x140>
 800034a:	4282      	cmp	r2, r0
 800034c:	f200 80b8 	bhi.w	80004c0 <__udivmoddi4+0x2b0>
 8000350:	1a84      	subs	r4, r0, r2
 8000352:	eb61 0103 	sbc.w	r1, r1, r3
 8000356:	2001      	movs	r0, #1
 8000358:	468c      	mov	ip, r1
 800035a:	2d00      	cmp	r5, #0
 800035c:	d0a8      	beq.n	80002b0 <__udivmoddi4+0xa0>
 800035e:	e9c5 4c00 	strd	r4, ip, [r5]
 8000362:	e7a5      	b.n	80002b0 <__udivmoddi4+0xa0>
 8000364:	f1c2 0320 	rsb	r3, r2, #32
 8000368:	fa20 f603 	lsr.w	r6, r0, r3
 800036c:	4097      	lsls	r7, r2
 800036e:	fa01 f002 	lsl.w	r0, r1, r2
 8000372:	ea4f 4e17 	mov.w	lr, r7, lsr #16
 8000376:	40d9      	lsrs	r1, r3
 8000378:	4330      	orrs	r0, r6
 800037a:	0c03      	lsrs	r3, r0, #16
 800037c:	fbb1 f6fe 	udiv	r6, r1, lr
 8000380:	fa1f f887 	uxth.w	r8, r7
 8000384:	fb0e 1116 	mls	r1, lr, r6, r1
 8000388:	ea43 4301 	orr.w	r3, r3, r1, lsl #16
 800038c:	fb06 f108 	mul.w	r1, r6, r8
 8000390:	4299      	cmp	r1, r3
 8000392:	fa04 f402 	lsl.w	r4, r4, r2
 8000396:	d909      	bls.n	80003ac <__udivmoddi4+0x19c>
 8000398:	18fb      	adds	r3, r7, r3
 800039a:	f106 3cff 	add.w	ip, r6, #4294967295
 800039e:	f080 808d 	bcs.w	80004bc <__udivmoddi4+0x2ac>
 80003a2:	4299      	cmp	r1, r3
 80003a4:	f240 808a 	bls.w	80004bc <__udivmoddi4+0x2ac>
 80003a8:	3e02      	subs	r6, #2
 80003aa:	443b      	add	r3, r7
 80003ac:	1a5b      	subs	r3, r3, r1
 80003ae:	b281      	uxth	r1, r0
 80003b0:	fbb3 f0fe 	udiv	r0, r3, lr
 80003b4:	fb0e 3310 	mls	r3, lr, r0, r3
 80003b8:	ea41 4103 	orr.w	r1, r1, r3, lsl #16
 80003bc:	fb00 f308 	mul.w	r3, r0, r8
 80003c0:	428b      	cmp	r3, r1
 80003c2:	d907      	bls.n	80003d4 <__udivmoddi4+0x1c4>
 80003c4:	1879      	adds	r1, r7, r1
 80003c6:	f100 3cff 	add.w	ip, r0, #4294967295
 80003ca:	d273      	bcs.n	80004b4 <__udivmoddi4+0x2a4>
 80003cc:	428b      	cmp	r3, r1
 80003ce:	d971      	bls.n	80004b4 <__udivmoddi4+0x2a4>
 80003d0:	3802      	subs	r0, #2
 80003d2:	4439      	add	r1, r7
 80003d4:	1acb      	subs	r3, r1, r3
 80003d6:	ea40 4606 	orr.w	r6, r0, r6, lsl #16
 80003da:	e778      	b.n	80002ce <__udivmoddi4+0xbe>
 80003dc:	f1c6 0c20 	rsb	ip, r6, #32
 80003e0:	fa03 f406 	lsl.w	r4, r3, r6
 80003e4:	fa22 f30c 	lsr.w	r3, r2, ip
 80003e8:	431c      	orrs	r4, r3
 80003ea:	fa20 f70c 	lsr.w	r7, r0, ip
 80003ee:	fa01 f306 	lsl.w	r3, r1, r6
 80003f2:	ea4f 4e14 	mov.w	lr, r4, lsr #16
 80003f6:	fa21 f10c 	lsr.w	r1, r1, ip
 80003fa:	431f      	orrs	r7, r3
 80003fc:	0c3b      	lsrs	r3, r7, #16
 80003fe:	fbb1 f9fe 	udiv	r9, r1, lr
 8000402:	fa1f f884 	uxth.w	r8, r4
 8000406:	fb0e 1119 	mls	r1, lr, r9, r1
 800040a:	ea43 4101 	orr.w	r1, r3, r1, lsl #16
 800040e:	fb09 fa08 	mul.w	sl, r9, r8
 8000412:	458a      	cmp	sl, r1
 8000414:	fa02 f206 	lsl.w	r2, r2, r6
 8000418:	fa00 f306 	lsl.w	r3, r0, r6
 800041c:	d908      	bls.n	8000430 <__udivmoddi4+0x220>
 800041e:	1861      	adds	r1, r4, r1
 8000420:	f109 30ff 	add.w	r0, r9, #4294967295
 8000424:	d248      	bcs.n	80004b8 <__udivmoddi4+0x2a8>
 8000426:	458a      	cmp	sl, r1
 8000428:	d946      	bls.n	80004b8 <__udivmoddi4+0x2a8>
 800042a:	f1a9 0902 	sub.w	r9, r9, #2
 800042e:	4421      	add	r1, r4
 8000430:	eba1 010a 	sub.w	r1, r1, sl
 8000434:	b2bf      	uxth	r7, r7
 8000436:	fbb1 f0fe 	udiv	r0, r1, lr
 800043a:	fb0e 1110 	mls	r1, lr, r0, r1
 800043e:	ea47 4701 	orr.w	r7, r7, r1, lsl #16
 8000442:	fb00 f808 	mul.w	r8, r0, r8
 8000446:	45b8      	cmp	r8, r7
 8000448:	d907      	bls.n	800045a <__udivmoddi4+0x24a>
 800044a:	19e7      	adds	r7, r4, r7
 800044c:	f100 31ff 	add.w	r1, r0, #4294967295
 8000450:	d22e      	bcs.n	80004b0 <__udivmoddi4+0x2a0>
 8000452:	45b8      	cmp	r8, r7
 8000454:	d92c      	bls.n	80004b0 <__udivmoddi4+0x2a0>
 8000456:	3802      	subs	r0, #2
 8000458:	4427      	add	r7, r4
 800045a:	ea40 4009 	orr.w	r0, r0, r9, lsl #16
 800045e:	eba7 0708 	sub.w	r7, r7, r8
 8000462:	fba0 8902 	umull	r8, r9, r0, r2
 8000466:	454f      	cmp	r7, r9
 8000468:	46c6      	mov	lr, r8
 800046a:	4649      	mov	r1, r9
 800046c:	d31a      	bcc.n	80004a4 <__udivmoddi4+0x294>
 800046e:	d017      	beq.n	80004a0 <__udivmoddi4+0x290>
 8000470:	b15d      	cbz	r5, 800048a <__udivmoddi4+0x27a>
 8000472:	ebb3 020e 	subs.w	r2, r3, lr
 8000476:	eb67 0701 	sbc.w	r7, r7, r1
 800047a:	fa07 fc0c 	lsl.w	ip, r7, ip
 800047e:	40f2      	lsrs	r2, r6
 8000480:	ea4c 0202 	orr.w	r2, ip, r2
 8000484:	40f7      	lsrs	r7, r6
 8000486:	e9c5 2700 	strd	r2, r7, [r5]
 800048a:	2600      	movs	r6, #0
 800048c:	4631      	mov	r1, r6
 800048e:	e8bd 87f0 	ldmia.w	sp!, {r4, r5, r6, r7, r8, r9, sl, pc}
 8000492:	462e      	mov	r6, r5
 8000494:	4628      	mov	r0, r5
 8000496:	e70b      	b.n	80002b0 <__udivmoddi4+0xa0>
 8000498:	4606      	mov	r6, r0
 800049a:	e6e9      	b.n	8000270 <__udivmoddi4+0x60>
 800049c:	4618      	mov	r0, r3
 800049e:	e6fd      	b.n	800029c <__udivmoddi4+0x8c>
 80004a0:	4543      	cmp	r3, r8
 80004a2:	d2e5      	bcs.n	8000470 <__udivmoddi4+0x260>
 80004a4:	ebb8 0e02 	subs.w	lr, r8, r2
 80004a8:	eb69 0104 	sbc.w	r1, r9, r4
 80004ac:	3801      	subs	r0, #1
 80004ae:	e7df      	b.n	8000470 <__udivmoddi4+0x260>
 80004b0:	4608      	mov	r0, r1
 80004b2:	e7d2      	b.n	800045a <__udivmoddi4+0x24a>
 80004b4:	4660      	mov	r0, ip
 80004b6:	e78d      	b.n	80003d4 <__udivmoddi4+0x1c4>
 80004b8:	4681      	mov	r9, r0
 80004ba:	e7b9      	b.n	8000430 <__udivmoddi4+0x220>
 80004bc:	4666      	mov	r6, ip
 80004be:	e775      	b.n	80003ac <__udivmoddi4+0x19c>
 80004c0:	4630      	mov	r0, r6
 80004c2:	e74a      	b.n	800035a <__udivmoddi4+0x14a>
 80004c4:	f1ac 0c02 	sub.w	ip, ip, #2
 80004c8:	4439      	add	r1, r7
 80004ca:	e713      	b.n	80002f4 <__udivmoddi4+0xe4>
 80004cc:	3802      	subs	r0, #2
 80004ce:	443c      	add	r4, r7
 80004d0:	e724      	b.n	800031c <__udivmoddi4+0x10c>
 80004d2:	bf00      	nop

080004d4 <__aeabi_idiv0>:
 80004d4:	4770      	bx	lr
 80004d6:	bf00      	nop

080004d8 <vApplicationGetIdleTaskMemory>:
/* USER CODE BEGIN GET_IDLE_TASK_MEMORY */
static StaticTask_t xIdleTaskTCBBuffer;
static StackType_t xIdleStack[configMINIMAL_STACK_SIZE];

void vApplicationGetIdleTaskMemory( StaticTask_t **ppxIdleTaskTCBBuffer, StackType_t **ppxIdleTaskStackBuffer, uint32_t *pulIdleTaskStackSize )
{
 80004d8:	b480      	push	{r7}
 80004da:	b085      	sub	sp, #20
 80004dc:	af00      	add	r7, sp, #0
 80004de:	60f8      	str	r0, [r7, #12]
 80004e0:	60b9      	str	r1, [r7, #8]
 80004e2:	607a      	str	r2, [r7, #4]
  *ppxIdleTaskTCBBuffer = &xIdleTaskTCBBuffer;
 80004e4:	68fb      	ldr	r3, [r7, #12]
 80004e6:	4a07      	ldr	r2, [pc, #28]	; (8000504 <vApplicationGetIdleTaskMemory+0x2c>)
 80004e8:	601a      	str	r2, [r3, #0]
  *ppxIdleTaskStackBuffer = &xIdleStack[0];
 80004ea:	68bb      	ldr	r3, [r7, #8]
 80004ec:	4a06      	ldr	r2, [pc, #24]	; (8000508 <vApplicationGetIdleTaskMemory+0x30>)
 80004ee:	601a      	str	r2, [r3, #0]
  *pulIdleTaskStackSize = configMINIMAL_STACK_SIZE;
 80004f0:	687b      	ldr	r3, [r7, #4]
 80004f2:	2280      	movs	r2, #128	; 0x80
 80004f4:	601a      	str	r2, [r3, #0]
  /* place for user code */
}
 80004f6:	bf00      	nop
 80004f8:	3714      	adds	r7, #20
 80004fa:	46bd      	mov	sp, r7
 80004fc:	f85d 7b04 	ldr.w	r7, [sp], #4
 8000500:	4770      	bx	lr
 8000502:	bf00      	nop
 8000504:	2000002c 	.word	0x2000002c
 8000508:	20000080 	.word	0x20000080

0800050c <ledperiodtask>:

/* USER CODE END PFP */

/* Private user code ---------------------------------------------------------*/
/* USER CODE BEGIN 0 */
    void ledperiodtask(void *pvParam){
 800050c:	b580      	push	{r7, lr}
 800050e:	b084      	sub	sp, #16
 8000510:	af00      	add	r7, sp, #0
 8000512:	6078      	str	r0, [r7, #4]

    	ledinfo_t *led=(ledinfo_t*)pvParam;
 8000514:	687b      	ldr	r3, [r7, #4]
 8000516:	60fb      	str	r3, [r7, #12]
    	uint16_t pin=led->pin;
 8000518:	68fb      	ldr	r3, [r7, #12]
 800051a:	681b      	ldr	r3, [r3, #0]
 800051c:	817b      	strh	r3, [r7, #10]
    		HAL_GPIO_TogglePin(GPIOD, pin);
 800051e:	897b      	ldrh	r3, [r7, #10]
 8000520:	4619      	mov	r1, r3
 8000522:	480e      	ldr	r0, [pc, #56]	; (800055c <ledperiodtask+0x50>)
 8000524:	f000 fdad 	bl	8001082 <HAL_GPIO_TogglePin>
    		HAL_UART_Transmit(&huart2, (uint8_t*)pvParam, strlen((char*)pvParam), HAL_MAX_DELAY);
 8000528:	6878      	ldr	r0, [r7, #4]
 800052a:	f7ff fe51 	bl	80001d0 <strlen>
 800052e:	4603      	mov	r3, r0
 8000530:	b29a      	uxth	r2, r3
 8000532:	f04f 33ff 	mov.w	r3, #4294967295
 8000536:	6879      	ldr	r1, [r7, #4]
 8000538:	4809      	ldr	r0, [pc, #36]	; (8000560 <ledperiodtask+0x54>)
 800053a:	f001 fd81 	bl	8002040 <HAL_UART_Transmit>
    		portYIELD();
 800053e:	4b09      	ldr	r3, [pc, #36]	; (8000564 <ledperiodtask+0x58>)
 8000540:	f04f 5280 	mov.w	r2, #268435456	; 0x10000000
 8000544:	601a      	str	r2, [r3, #0]
 8000546:	f3bf 8f4f 	dsb	sy
 800054a:	f3bf 8f6f 	isb	sy

    	vTaskDelete(NULL);
 800054e:	2000      	movs	r0, #0
 8000550:	f002 fb04 	bl	8002b5c <vTaskDelete>

    }
 8000554:	bf00      	nop
 8000556:	3710      	adds	r7, #16
 8000558:	46bd      	mov	sp, r7
 800055a:	bd80      	pop	{r7, pc}
 800055c:	40020c00 	.word	0x40020c00
 8000560:	20003fd8 	.word	0x20003fd8
 8000564:	e000ed04 	.word	0xe000ed04

08000568 <main>:
/**
  * @brief  The application entry point.
  * @retval int
  */
int main(void)
{
 8000568:	b5b0      	push	{r4, r5, r7, lr}
 800056a:	b08c      	sub	sp, #48	; 0x30
 800056c:	af02      	add	r7, sp, #8
  /* USER CODE END 1 */

  /* MCU Configuration--------------------------------------------------------*/

  /* Reset of all peripherals, Initializes the Flash interface and the Systick. */
  HAL_Init();
 800056e:	f000 faaf 	bl	8000ad0 <HAL_Init>
  /* USER CODE BEGIN Init */

  /* USER CODE END Init */

  /* Configure the system clock */
  SystemClock_Config();
 8000572:	f000 f87f 	bl	8000674 <SystemClock_Config>
  /* USER CODE BEGIN SysInit */

  /* USER CODE END SysInit */

  /* Initialize all configured peripherals */
  MX_GPIO_Init();
 8000576:	f000 f911 	bl	800079c <MX_GPIO_Init>
  MX_USART2_UART_Init();
 800057a:	f000 f8e3 	bl	8000744 <MX_USART2_UART_Init>
  /* USER CODE BEGIN 2 */
  Message = "xRet";
 800057e:	4b30      	ldr	r3, [pc, #192]	; (8000640 <main+0xd8>)
 8000580:	627b      	str	r3, [r7, #36]	; 0x24
  	HAL_UART_Transmit(&huart2, (uint8_t*)Message, strlen((char*)Message), HAL_MAX_DELAY);
 8000582:	6a78      	ldr	r0, [r7, #36]	; 0x24
 8000584:	f7ff fe24 	bl	80001d0 <strlen>
 8000588:	4603      	mov	r3, r0
 800058a:	b29a      	uxth	r2, r3
 800058c:	f04f 33ff 	mov.w	r3, #4294967295
 8000590:	6a79      	ldr	r1, [r7, #36]	; 0x24
 8000592:	482c      	ldr	r0, [pc, #176]	; (8000644 <main+0xdc>)
 8000594:	f001 fd54 	bl	8002040 <HAL_UART_Transmit>
  /* add queues, ... */
  /* USER CODE END RTOS_QUEUES */

  /* Create the thread(s) */
  /* definition and creation of defaultTask */
  osThreadDef(defaultTask, StartDefaultTask, osPriorityIdle, 0, 128);
 8000598:	4b2b      	ldr	r3, [pc, #172]	; (8000648 <main+0xe0>)
 800059a:	1d3c      	adds	r4, r7, #4
 800059c:	461d      	mov	r5, r3
 800059e:	cd0f      	ldmia	r5!, {r0, r1, r2, r3}
 80005a0:	c40f      	stmia	r4!, {r0, r1, r2, r3}
 80005a2:	e895 0007 	ldmia.w	r5, {r0, r1, r2}
 80005a6:	e884 0007 	stmia.w	r4, {r0, r1, r2}
  defaultTaskHandle = osThreadCreate(osThread(defaultTask), NULL);
 80005aa:	1d3b      	adds	r3, r7, #4
 80005ac:	2100      	movs	r1, #0
 80005ae:	4618      	mov	r0, r3
 80005b0:	f002 f82d 	bl	800260e <osThreadCreate>
 80005b4:	4603      	mov	r3, r0
 80005b6:	4a25      	ldr	r2, [pc, #148]	; (800064c <main+0xe4>)
 80005b8:	6013      	str	r3, [r2, #0]

  /* USER CODE BEGIN RTOS_THREADS */
  xRet = xTaskCreate(ledperiodtask, "Task1", configMINIMAL_STACK_SIZE, "led1\r\n", 1,NULL);
 80005ba:	2300      	movs	r3, #0
 80005bc:	9301      	str	r3, [sp, #4]
 80005be:	2301      	movs	r3, #1
 80005c0:	9300      	str	r3, [sp, #0]
 80005c2:	4b23      	ldr	r3, [pc, #140]	; (8000650 <main+0xe8>)
 80005c4:	2280      	movs	r2, #128	; 0x80
 80005c6:	4923      	ldr	r1, [pc, #140]	; (8000654 <main+0xec>)
 80005c8:	4823      	ldr	r0, [pc, #140]	; (8000658 <main+0xf0>)
 80005ca:	f002 f991 	bl	80028f0 <xTaskCreate>
 80005ce:	6238      	str	r0, [r7, #32]
  if(xRet!=pdTRUE)
 80005d0:	6a3b      	ldr	r3, [r7, #32]
 80005d2:	2b01      	cmp	r3, #1
 80005d4:	d001      	beq.n	80005da <main+0x72>
	  Error_Handler();
 80005d6:	f000 f94d 	bl	8000874 <Error_Handler>
  xRet = xTaskCreate(ledperiodtask, "Task2", configMINIMAL_STACK_SIZE, "led2\r\n", 2,NULL);
 80005da:	2300      	movs	r3, #0
 80005dc:	9301      	str	r3, [sp, #4]
 80005de:	2302      	movs	r3, #2
 80005e0:	9300      	str	r3, [sp, #0]
 80005e2:	4b1e      	ldr	r3, [pc, #120]	; (800065c <main+0xf4>)
 80005e4:	2280      	movs	r2, #128	; 0x80
 80005e6:	491e      	ldr	r1, [pc, #120]	; (8000660 <main+0xf8>)
 80005e8:	481b      	ldr	r0, [pc, #108]	; (8000658 <main+0xf0>)
 80005ea:	f002 f981 	bl	80028f0 <xTaskCreate>
 80005ee:	6238      	str	r0, [r7, #32]
   if(xRet!=pdTRUE)
 80005f0:	6a3b      	ldr	r3, [r7, #32]
 80005f2:	2b01      	cmp	r3, #1
 80005f4:	d001      	beq.n	80005fa <main+0x92>
 	  Error_Handler();
 80005f6:	f000 f93d 	bl	8000874 <Error_Handler>
   xRet = xTaskCreate(ledperiodtask, "Task3", configMINIMAL_STACK_SIZE, "led3\r\n", 3,NULL);
 80005fa:	2300      	movs	r3, #0
 80005fc:	9301      	str	r3, [sp, #4]
 80005fe:	2303      	movs	r3, #3
 8000600:	9300      	str	r3, [sp, #0]
 8000602:	4b18      	ldr	r3, [pc, #96]	; (8000664 <main+0xfc>)
 8000604:	2280      	movs	r2, #128	; 0x80
 8000606:	4918      	ldr	r1, [pc, #96]	; (8000668 <main+0x100>)
 8000608:	4813      	ldr	r0, [pc, #76]	; (8000658 <main+0xf0>)
 800060a:	f002 f971 	bl	80028f0 <xTaskCreate>
 800060e:	6238      	str	r0, [r7, #32]
    if(xRet!=pdTRUE)
 8000610:	6a3b      	ldr	r3, [r7, #32]
 8000612:	2b01      	cmp	r3, #1
 8000614:	d001      	beq.n	800061a <main+0xb2>
  	  Error_Handler();
 8000616:	f000 f92d 	bl	8000874 <Error_Handler>
    xRet = xTaskCreate(ledperiodtask, "Task4", configMINIMAL_STACK_SIZE, "led4\r\n", 4,NULL);
 800061a:	2300      	movs	r3, #0
 800061c:	9301      	str	r3, [sp, #4]
 800061e:	2304      	movs	r3, #4
 8000620:	9300      	str	r3, [sp, #0]
 8000622:	4b12      	ldr	r3, [pc, #72]	; (800066c <main+0x104>)
 8000624:	2280      	movs	r2, #128	; 0x80
 8000626:	4912      	ldr	r1, [pc, #72]	; (8000670 <main+0x108>)
 8000628:	480b      	ldr	r0, [pc, #44]	; (8000658 <main+0xf0>)
 800062a:	f002 f961 	bl	80028f0 <xTaskCreate>
 800062e:	6238      	str	r0, [r7, #32]
     if(xRet!=pdTRUE)
 8000630:	6a3b      	ldr	r3, [r7, #32]
 8000632:	2b01      	cmp	r3, #1
 8000634:	d001      	beq.n	800063a <main+0xd2>
   	  Error_Handler();
 8000636:	f000 f91d 	bl	8000874 <Error_Handler>
  /* USER CODE END RTOS_THREADS */

  /* Start scheduler */
  osKernelStart();
 800063a:	f001 ffe1 	bl	8002600 <osKernelStart>

  /* We should never get here as control is now taken by the scheduler */
  /* Infinite loop */
  /* USER CODE BEGIN WHILE */
  while (1)
 800063e:	e7fe      	b.n	800063e <main+0xd6>
 8000640:	08003c08 	.word	0x08003c08
 8000644:	20003fd8 	.word	0x20003fd8
 8000648:	08003c50 	.word	0x08003c50
 800064c:	20003fd4 	.word	0x20003fd4
 8000650:	08003c10 	.word	0x08003c10
 8000654:	08003c18 	.word	0x08003c18
 8000658:	0800050d 	.word	0x0800050d
 800065c:	08003c20 	.word	0x08003c20
 8000660:	08003c28 	.word	0x08003c28
 8000664:	08003c30 	.word	0x08003c30
 8000668:	08003c38 	.word	0x08003c38
 800066c:	08003c40 	.word	0x08003c40
 8000670:	08003c48 	.word	0x08003c48

08000674 <SystemClock_Config>:
/**
  * @brief System Clock Configuration
  * @retval None
  */
void SystemClock_Config(void)
{
 8000674:	b580      	push	{r7, lr}
 8000676:	b094      	sub	sp, #80	; 0x50
 8000678:	af00      	add	r7, sp, #0
  RCC_OscInitTypeDef RCC_OscInitStruct = {0};
 800067a:	f107 0320 	add.w	r3, r7, #32
 800067e:	2230      	movs	r2, #48	; 0x30
 8000680:	2100      	movs	r1, #0
 8000682:	4618      	mov	r0, r3
 8000684:	f003 faa6 	bl	8003bd4 <memset>
  RCC_ClkInitTypeDef RCC_ClkInitStruct = {0};
 8000688:	f107 030c 	add.w	r3, r7, #12
 800068c:	2200      	movs	r2, #0
 800068e:	601a      	str	r2, [r3, #0]
 8000690:	605a      	str	r2, [r3, #4]
 8000692:	609a      	str	r2, [r3, #8]
 8000694:	60da      	str	r2, [r3, #12]
 8000696:	611a      	str	r2, [r3, #16]

  /** Configure the main internal regulator output voltage
  */
  __HAL_RCC_PWR_CLK_ENABLE();
 8000698:	2300      	movs	r3, #0
 800069a:	60bb      	str	r3, [r7, #8]
 800069c:	4b27      	ldr	r3, [pc, #156]	; (800073c <SystemClock_Config+0xc8>)
 800069e:	6c1b      	ldr	r3, [r3, #64]	; 0x40
 80006a0:	4a26      	ldr	r2, [pc, #152]	; (800073c <SystemClock_Config+0xc8>)
 80006a2:	f043 5380 	orr.w	r3, r3, #268435456	; 0x10000000
 80006a6:	6413      	str	r3, [r2, #64]	; 0x40
 80006a8:	4b24      	ldr	r3, [pc, #144]	; (800073c <SystemClock_Config+0xc8>)
 80006aa:	6c1b      	ldr	r3, [r3, #64]	; 0x40
 80006ac:	f003 5380 	and.w	r3, r3, #268435456	; 0x10000000
 80006b0:	60bb      	str	r3, [r7, #8]
 80006b2:	68bb      	ldr	r3, [r7, #8]
  __HAL_PWR_VOLTAGESCALING_CONFIG(PWR_REGULATOR_VOLTAGE_SCALE1);
 80006b4:	2300      	movs	r3, #0
 80006b6:	607b      	str	r3, [r7, #4]
 80006b8:	4b21      	ldr	r3, [pc, #132]	; (8000740 <SystemClock_Config+0xcc>)
 80006ba:	681b      	ldr	r3, [r3, #0]
 80006bc:	4a20      	ldr	r2, [pc, #128]	; (8000740 <SystemClock_Config+0xcc>)
 80006be:	f443 4380 	orr.w	r3, r3, #16384	; 0x4000
 80006c2:	6013      	str	r3, [r2, #0]
 80006c4:	4b1e      	ldr	r3, [pc, #120]	; (8000740 <SystemClock_Config+0xcc>)
 80006c6:	681b      	ldr	r3, [r3, #0]
 80006c8:	f403 4380 	and.w	r3, r3, #16384	; 0x4000
 80006cc:	607b      	str	r3, [r7, #4]
 80006ce:	687b      	ldr	r3, [r7, #4]
  /** Initializes the RCC Oscillators according to the specified parameters
  * in the RCC_OscInitTypeDef structure.
  */
  RCC_OscInitStruct.OscillatorType = RCC_OSCILLATORTYPE_HSI;
 80006d0:	2302      	movs	r3, #2
 80006d2:	623b      	str	r3, [r7, #32]
  RCC_OscInitStruct.HSIState = RCC_HSI_ON;
 80006d4:	2301      	movs	r3, #1
 80006d6:	62fb      	str	r3, [r7, #44]	; 0x2c
  RCC_OscInitStruct.HSICalibrationValue = RCC_HSICALIBRATION_DEFAULT;
 80006d8:	2310      	movs	r3, #16
 80006da:	633b      	str	r3, [r7, #48]	; 0x30
  RCC_OscInitStruct.PLL.PLLState = RCC_PLL_ON;
 80006dc:	2302      	movs	r3, #2
 80006de:	63bb      	str	r3, [r7, #56]	; 0x38
  RCC_OscInitStruct.PLL.PLLSource = RCC_PLLSOURCE_HSI;
 80006e0:	2300      	movs	r3, #0
 80006e2:	63fb      	str	r3, [r7, #60]	; 0x3c
  RCC_OscInitStruct.PLL.PLLM = 8;
 80006e4:	2308      	movs	r3, #8
 80006e6:	643b      	str	r3, [r7, #64]	; 0x40
  RCC_OscInitStruct.PLL.PLLN = 50;
 80006e8:	2332      	movs	r3, #50	; 0x32
 80006ea:	647b      	str	r3, [r7, #68]	; 0x44
  RCC_OscInitStruct.PLL.PLLP = RCC_PLLP_DIV4;
 80006ec:	2304      	movs	r3, #4
 80006ee:	64bb      	str	r3, [r7, #72]	; 0x48
  RCC_OscInitStruct.PLL.PLLQ = 7;
 80006f0:	2307      	movs	r3, #7
 80006f2:	64fb      	str	r3, [r7, #76]	; 0x4c
  if (HAL_RCC_OscConfig(&RCC_OscInitStruct) != HAL_OK)
 80006f4:	f107 0320 	add.w	r3, r7, #32
 80006f8:	4618      	mov	r0, r3
 80006fa:	f000 fcdd 	bl	80010b8 <HAL_RCC_OscConfig>
 80006fe:	4603      	mov	r3, r0
 8000700:	2b00      	cmp	r3, #0
 8000702:	d001      	beq.n	8000708 <SystemClock_Config+0x94>
  {
    Error_Handler();
 8000704:	f000 f8b6 	bl	8000874 <Error_Handler>
  }
  /** Initializes the CPU, AHB and APB buses clocks
  */
  RCC_ClkInitStruct.ClockType = RCC_CLOCKTYPE_HCLK|RCC_CLOCKTYPE_SYSCLK
 8000708:	230f      	movs	r3, #15
 800070a:	60fb      	str	r3, [r7, #12]
                              |RCC_CLOCKTYPE_PCLK1|RCC_CLOCKTYPE_PCLK2;
  RCC_ClkInitStruct.SYSCLKSource = RCC_SYSCLKSOURCE_PLLCLK;
 800070c:	2302      	movs	r3, #2
 800070e:	613b      	str	r3, [r7, #16]
  RCC_ClkInitStruct.AHBCLKDivider = RCC_SYSCLK_DIV1;
 8000710:	2300      	movs	r3, #0
 8000712:	617b      	str	r3, [r7, #20]
  RCC_ClkInitStruct.APB1CLKDivider = RCC_HCLK_DIV1;
 8000714:	2300      	movs	r3, #0
 8000716:	61bb      	str	r3, [r7, #24]
  RCC_ClkInitStruct.APB2CLKDivider = RCC_HCLK_DIV1;
 8000718:	2300      	movs	r3, #0
 800071a:	61fb      	str	r3, [r7, #28]

  if (HAL_RCC_ClockConfig(&RCC_ClkInitStruct, FLASH_LATENCY_0) != HAL_OK)
 800071c:	f107 030c 	add.w	r3, r7, #12
 8000720:	2100      	movs	r1, #0
 8000722:	4618      	mov	r0, r3
 8000724:	f000 ff40 	bl	80015a8 <HAL_RCC_ClockConfig>
 8000728:	4603      	mov	r3, r0
 800072a:	2b00      	cmp	r3, #0
 800072c:	d001      	beq.n	8000732 <SystemClock_Config+0xbe>
  {
    Error_Handler();
 800072e:	f000 f8a1 	bl	8000874 <Error_Handler>
  }
}
 8000732:	bf00      	nop
 8000734:	3750      	adds	r7, #80	; 0x50
 8000736:	46bd      	mov	sp, r7
 8000738:	bd80      	pop	{r7, pc}
 800073a:	bf00      	nop
 800073c:	40023800 	.word	0x40023800
 8000740:	40007000 	.word	0x40007000

08000744 <MX_USART2_UART_Init>:
  * @brief USART2 Initialization Function
  * @param None
  * @retval None
  */
static void MX_USART2_UART_Init(void)
{
 8000744:	b580      	push	{r7, lr}
 8000746:	af00      	add	r7, sp, #0
  /* USER CODE END USART2_Init 0 */

  /* USER CODE BEGIN USART2_Init 1 */

  /* USER CODE END USART2_Init 1 */
  huart2.Instance = USART2;
 8000748:	4b12      	ldr	r3, [pc, #72]	; (8000794 <MX_USART2_UART_Init+0x50>)
 800074a:	4a13      	ldr	r2, [pc, #76]	; (8000798 <MX_USART2_UART_Init+0x54>)
 800074c:	601a      	str	r2, [r3, #0]
  huart2.Init.BaudRate = 115200;
 800074e:	4b11      	ldr	r3, [pc, #68]	; (8000794 <MX_USART2_UART_Init+0x50>)
 8000750:	f44f 32e1 	mov.w	r2, #115200	; 0x1c200
 8000754:	605a      	str	r2, [r3, #4]
  huart2.Init.WordLength = UART_WORDLENGTH_8B;
 8000756:	4b0f      	ldr	r3, [pc, #60]	; (8000794 <MX_USART2_UART_Init+0x50>)
 8000758:	2200      	movs	r2, #0
 800075a:	609a      	str	r2, [r3, #8]
  huart2.Init.StopBits = UART_STOPBITS_1;
 800075c:	4b0d      	ldr	r3, [pc, #52]	; (8000794 <MX_USART2_UART_Init+0x50>)
 800075e:	2200      	movs	r2, #0
 8000760:	60da      	str	r2, [r3, #12]
  huart2.Init.Parity = UART_PARITY_NONE;
 8000762:	4b0c      	ldr	r3, [pc, #48]	; (8000794 <MX_USART2_UART_Init+0x50>)
 8000764:	2200      	movs	r2, #0
 8000766:	611a      	str	r2, [r3, #16]
  huart2.Init.Mode = UART_MODE_TX_RX;
 8000768:	4b0a      	ldr	r3, [pc, #40]	; (8000794 <MX_USART2_UART_Init+0x50>)
 800076a:	220c      	movs	r2, #12
 800076c:	615a      	str	r2, [r3, #20]
  huart2.Init.HwFlowCtl = UART_HWCONTROL_NONE;
 800076e:	4b09      	ldr	r3, [pc, #36]	; (8000794 <MX_USART2_UART_Init+0x50>)
 8000770:	2200      	movs	r2, #0
 8000772:	619a      	str	r2, [r3, #24]
  huart2.Init.OverSampling = UART_OVERSAMPLING_16;
 8000774:	4b07      	ldr	r3, [pc, #28]	; (8000794 <MX_USART2_UART_Init+0x50>)
 8000776:	2200      	movs	r2, #0
 8000778:	61da      	str	r2, [r3, #28]
  if (HAL_MultiProcessor_Init(&huart2, 0, UART_WAKEUPMETHOD_IDLELINE) != HAL_OK)
 800077a:	2200      	movs	r2, #0
 800077c:	2100      	movs	r1, #0
 800077e:	4805      	ldr	r0, [pc, #20]	; (8000794 <MX_USART2_UART_Init+0x50>)
 8000780:	f001 fbee 	bl	8001f60 <HAL_MultiProcessor_Init>
 8000784:	4603      	mov	r3, r0
 8000786:	2b00      	cmp	r3, #0
 8000788:	d001      	beq.n	800078e <MX_USART2_UART_Init+0x4a>
  {
    Error_Handler();
 800078a:	f000 f873 	bl	8000874 <Error_Handler>
  }
  /* USER CODE BEGIN USART2_Init 2 */

  /* USER CODE END USART2_Init 2 */

}
 800078e:	bf00      	nop
 8000790:	bd80      	pop	{r7, pc}
 8000792:	bf00      	nop
 8000794:	20003fd8 	.word	0x20003fd8
 8000798:	40004400 	.word	0x40004400

0800079c <MX_GPIO_Init>:
  * @brief GPIO Initialization Function
  * @param None
  * @retval None
  */
static void MX_GPIO_Init(void)
{
 800079c:	b580      	push	{r7, lr}
 800079e:	b088      	sub	sp, #32
 80007a0:	af00      	add	r7, sp, #0
  GPIO_InitTypeDef GPIO_InitStruct = {0};
 80007a2:	f107 030c 	add.w	r3, r7, #12
 80007a6:	2200      	movs	r2, #0
 80007a8:	601a      	str	r2, [r3, #0]
 80007aa:	605a      	str	r2, [r3, #4]
 80007ac:	609a      	str	r2, [r3, #8]
 80007ae:	60da      	str	r2, [r3, #12]
 80007b0:	611a      	str	r2, [r3, #16]

  /* GPIO Ports Clock Enable */
  __HAL_RCC_GPIOH_CLK_ENABLE();
 80007b2:	2300      	movs	r3, #0
 80007b4:	60bb      	str	r3, [r7, #8]
 80007b6:	4b20      	ldr	r3, [pc, #128]	; (8000838 <MX_GPIO_Init+0x9c>)
 80007b8:	6b1b      	ldr	r3, [r3, #48]	; 0x30
 80007ba:	4a1f      	ldr	r2, [pc, #124]	; (8000838 <MX_GPIO_Init+0x9c>)
 80007bc:	f043 0380 	orr.w	r3, r3, #128	; 0x80
 80007c0:	6313      	str	r3, [r2, #48]	; 0x30
 80007c2:	4b1d      	ldr	r3, [pc, #116]	; (8000838 <MX_GPIO_Init+0x9c>)
 80007c4:	6b1b      	ldr	r3, [r3, #48]	; 0x30
 80007c6:	f003 0380 	and.w	r3, r3, #128	; 0x80
 80007ca:	60bb      	str	r3, [r7, #8]
 80007cc:	68bb      	ldr	r3, [r7, #8]
  __HAL_RCC_GPIOA_CLK_ENABLE();
 80007ce:	2300      	movs	r3, #0
 80007d0:	607b      	str	r3, [r7, #4]
 80007d2:	4b19      	ldr	r3, [pc, #100]	; (8000838 <MX_GPIO_Init+0x9c>)
 80007d4:	6b1b      	ldr	r3, [r3, #48]	; 0x30
 80007d6:	4a18      	ldr	r2, [pc, #96]	; (8000838 <MX_GPIO_Init+0x9c>)
 80007d8:	f043 0301 	orr.w	r3, r3, #1
 80007dc:	6313      	str	r3, [r2, #48]	; 0x30
 80007de:	4b16      	ldr	r3, [pc, #88]	; (8000838 <MX_GPIO_Init+0x9c>)
 80007e0:	6b1b      	ldr	r3, [r3, #48]	; 0x30
 80007e2:	f003 0301 	and.w	r3, r3, #1
 80007e6:	607b      	str	r3, [r7, #4]
 80007e8:	687b      	ldr	r3, [r7, #4]
  __HAL_RCC_GPIOD_CLK_ENABLE();
 80007ea:	2300      	movs	r3, #0
 80007ec:	603b      	str	r3, [r7, #0]
 80007ee:	4b12      	ldr	r3, [pc, #72]	; (8000838 <MX_GPIO_Init+0x9c>)
 80007f0:	6b1b      	ldr	r3, [r3, #48]	; 0x30
 80007f2:	4a11      	ldr	r2, [pc, #68]	; (8000838 <MX_GPIO_Init+0x9c>)
 80007f4:	f043 0308 	orr.w	r3, r3, #8
 80007f8:	6313      	str	r3, [r2, #48]	; 0x30
 80007fa:	4b0f      	ldr	r3, [pc, #60]	; (8000838 <MX_GPIO_Init+0x9c>)
 80007fc:	6b1b      	ldr	r3, [r3, #48]	; 0x30
 80007fe:	f003 0308 	and.w	r3, r3, #8
 8000802:	603b      	str	r3, [r7, #0]
 8000804:	683b      	ldr	r3, [r7, #0]

  /*Configure GPIO pin Output Level */
  HAL_GPIO_WritePin(GPIOD, GPIO_PIN_12|GPIO_PIN_13|GPIO_PIN_14|GPIO_PIN_15, GPIO_PIN_RESET);
 8000806:	2200      	movs	r2, #0
 8000808:	f44f 4170 	mov.w	r1, #61440	; 0xf000
 800080c:	480b      	ldr	r0, [pc, #44]	; (800083c <MX_GPIO_Init+0xa0>)
 800080e:	f000 fc1f 	bl	8001050 <HAL_GPIO_WritePin>

  /*Configure GPIO pins : PD12 PD13 PD14 PD15 */
  GPIO_InitStruct.Pin = GPIO_PIN_12|GPIO_PIN_13|GPIO_PIN_14|GPIO_PIN_15;
 8000812:	f44f 4370 	mov.w	r3, #61440	; 0xf000
 8000816:	60fb      	str	r3, [r7, #12]
  GPIO_InitStruct.Mode = GPIO_MODE_OUTPUT_PP;
 8000818:	2301      	movs	r3, #1
 800081a:	613b      	str	r3, [r7, #16]
  GPIO_InitStruct.Pull = GPIO_NOPULL;
 800081c:	2300      	movs	r3, #0
 800081e:	617b      	str	r3, [r7, #20]
  GPIO_InitStruct.Speed = GPIO_SPEED_FREQ_LOW;
 8000820:	2300      	movs	r3, #0
 8000822:	61bb      	str	r3, [r7, #24]
  HAL_GPIO_Init(GPIOD, &GPIO_InitStruct);
 8000824:	f107 030c 	add.w	r3, r7, #12
 8000828:	4619      	mov	r1, r3
 800082a:	4804      	ldr	r0, [pc, #16]	; (800083c <MX_GPIO_Init+0xa0>)
 800082c:	f000 fa74 	bl	8000d18 <HAL_GPIO_Init>

}
 8000830:	bf00      	nop
 8000832:	3720      	adds	r7, #32
 8000834:	46bd      	mov	sp, r7
 8000836:	bd80      	pop	{r7, pc}
 8000838:	40023800 	.word	0x40023800
 800083c:	40020c00 	.word	0x40020c00

08000840 <StartDefaultTask>:
  * @param  argument: Not used
  * @retval None
  */
/* USER CODE END Header_StartDefaultTask */
void StartDefaultTask(void const * argument)
{
 8000840:	b580      	push	{r7, lr}
 8000842:	b082      	sub	sp, #8
 8000844:	af00      	add	r7, sp, #0
 8000846:	6078      	str	r0, [r7, #4]
  /* USER CODE BEGIN 5 */
  /* Infinite loop */
  for(;;)
  {
    osDelay(1);
 8000848:	2001      	movs	r0, #1
 800084a:	f001 ff2c 	bl	80026a6 <osDelay>
 800084e:	e7fb      	b.n	8000848 <StartDefaultTask+0x8>

08000850 <HAL_TIM_PeriodElapsedCallback>:
  * a global variable "uwTick" used as application time base.
  * @param  htim : TIM handle
  * @retval None
  */
void HAL_TIM_PeriodElapsedCallback(TIM_HandleTypeDef *htim)
{
 8000850:	b580      	push	{r7, lr}
 8000852:	b082      	sub	sp, #8
 8000854:	af00      	add	r7, sp, #0
 8000856:	6078      	str	r0, [r7, #4]
  /* USER CODE BEGIN Callback 0 */

  /* USER CODE END Callback 0 */
  if (htim->Instance == TIM6) {
 8000858:	687b      	ldr	r3, [r7, #4]
 800085a:	681b      	ldr	r3, [r3, #0]
 800085c:	4a04      	ldr	r2, [pc, #16]	; (8000870 <HAL_TIM_PeriodElapsedCallback+0x20>)
 800085e:	4293      	cmp	r3, r2
 8000860:	d101      	bne.n	8000866 <HAL_TIM_PeriodElapsedCallback+0x16>
    HAL_IncTick();
 8000862:	f000 f957 	bl	8000b14 <HAL_IncTick>
  }
  /* USER CODE BEGIN Callback 1 */

  /* USER CODE END Callback 1 */
}
 8000866:	bf00      	nop
 8000868:	3708      	adds	r7, #8
 800086a:	46bd      	mov	sp, r7
 800086c:	bd80      	pop	{r7, pc}
 800086e:	bf00      	nop
 8000870:	40001000 	.word	0x40001000

08000874 <Error_Handler>:
/**
  * @brief  This function is executed in case of error occurrence.
  * @retval None
  */
void Error_Handler(void)
{
 8000874:	b480      	push	{r7}
 8000876:	af00      	add	r7, sp, #0
  \details Disables IRQ interrupts by setting the I-bit in the CPSR.
           Can only be executed in Privileged modes.
 */
__STATIC_FORCEINLINE void __disable_irq(void)
{
  __ASM volatile ("cpsid i" : : : "memory");
 8000878:	b672      	cpsid	i
}
 800087a:	bf00      	nop
  /* USER CODE BEGIN Error_Handler_Debug */
  /* User can add his own implementation to report the HAL error return state */
  __disable_irq();
  while (1)
 800087c:	e7fe      	b.n	800087c <Error_Handler+0x8>
	...

08000880 <HAL_MspInit>:
/* USER CODE END 0 */
/**
  * Initializes the Global MSP.
  */
void HAL_MspInit(void)
{
 8000880:	b580      	push	{r7, lr}
 8000882:	b082      	sub	sp, #8
 8000884:	af00      	add	r7, sp, #0
  /* USER CODE BEGIN MspInit 0 */

  /* USER CODE END MspInit 0 */

  __HAL_RCC_SYSCFG_CLK_ENABLE();
 8000886:	2300      	movs	r3, #0
 8000888:	607b      	str	r3, [r7, #4]
 800088a:	4b12      	ldr	r3, [pc, #72]	; (80008d4 <HAL_MspInit+0x54>)
 800088c:	6c5b      	ldr	r3, [r3, #68]	; 0x44
 800088e:	4a11      	ldr	r2, [pc, #68]	; (80008d4 <HAL_MspInit+0x54>)
 8000890:	f443 4380 	orr.w	r3, r3, #16384	; 0x4000
 8000894:	6453      	str	r3, [r2, #68]	; 0x44
 8000896:	4b0f      	ldr	r3, [pc, #60]	; (80008d4 <HAL_MspInit+0x54>)
 8000898:	6c5b      	ldr	r3, [r3, #68]	; 0x44
 800089a:	f403 4380 	and.w	r3, r3, #16384	; 0x4000
 800089e:	607b      	str	r3, [r7, #4]
 80008a0:	687b      	ldr	r3, [r7, #4]
  __HAL_RCC_PWR_CLK_ENABLE();
 80008a2:	2300      	movs	r3, #0
 80008a4:	603b      	str	r3, [r7, #0]
 80008a6:	4b0b      	ldr	r3, [pc, #44]	; (80008d4 <HAL_MspInit+0x54>)
 80008a8:	6c1b      	ldr	r3, [r3, #64]	; 0x40
 80008aa:	4a0a      	ldr	r2, [pc, #40]	; (80008d4 <HAL_MspInit+0x54>)
 80008ac:	f043 5380 	orr.w	r3, r3, #268435456	; 0x10000000
 80008b0:	6413      	str	r3, [r2, #64]	; 0x40
 80008b2:	4b08      	ldr	r3, [pc, #32]	; (80008d4 <HAL_MspInit+0x54>)
 80008b4:	6c1b      	ldr	r3, [r3, #64]	; 0x40
 80008b6:	f003 5380 	and.w	r3, r3, #268435456	; 0x10000000
 80008ba:	603b      	str	r3, [r7, #0]
 80008bc:	683b      	ldr	r3, [r7, #0]

  /* System interrupt init*/
  /* PendSV_IRQn interrupt configuration */
  HAL_NVIC_SetPriority(PendSV_IRQn, 15, 0);
 80008be:	2200      	movs	r2, #0
 80008c0:	210f      	movs	r1, #15
 80008c2:	f06f 0001 	mvn.w	r0, #1
 80008c6:	f000 f9fd 	bl	8000cc4 <HAL_NVIC_SetPriority>

  /* USER CODE BEGIN MspInit 1 */

  /* USER CODE END MspInit 1 */
}
 80008ca:	bf00      	nop
 80008cc:	3708      	adds	r7, #8
 80008ce:	46bd      	mov	sp, r7
 80008d0:	bd80      	pop	{r7, pc}
 80008d2:	bf00      	nop
 80008d4:	40023800 	.word	0x40023800

080008d8 <HAL_UART_MspInit>:
* This function configures the hardware resources used in this example
* @param huart: UART handle pointer
* @retval None
*/
void HAL_UART_MspInit(UART_HandleTypeDef* huart)
{
 80008d8:	b580      	push	{r7, lr}
 80008da:	b08a      	sub	sp, #40	; 0x28
 80008dc:	af00      	add	r7, sp, #0
 80008de:	6078      	str	r0, [r7, #4]
  GPIO_InitTypeDef GPIO_InitStruct = {0};
 80008e0:	f107 0314 	add.w	r3, r7, #20
 80008e4:	2200      	movs	r2, #0
 80008e6:	601a      	str	r2, [r3, #0]
 80008e8:	605a      	str	r2, [r3, #4]
 80008ea:	609a      	str	r2, [r3, #8]
 80008ec:	60da      	str	r2, [r3, #12]
 80008ee:	611a      	str	r2, [r3, #16]
  if(huart->Instance==USART2)
 80008f0:	687b      	ldr	r3, [r7, #4]
 80008f2:	681b      	ldr	r3, [r3, #0]
 80008f4:	4a19      	ldr	r2, [pc, #100]	; (800095c <HAL_UART_MspInit+0x84>)
 80008f6:	4293      	cmp	r3, r2
 80008f8:	d12b      	bne.n	8000952 <HAL_UART_MspInit+0x7a>
  {
  /* USER CODE BEGIN USART2_MspInit 0 */

  /* USER CODE END USART2_MspInit 0 */
    /* Peripheral clock enable */
    __HAL_RCC_USART2_CLK_ENABLE();
 80008fa:	2300      	movs	r3, #0
 80008fc:	613b      	str	r3, [r7, #16]
 80008fe:	4b18      	ldr	r3, [pc, #96]	; (8000960 <HAL_UART_MspInit+0x88>)
 8000900:	6c1b      	ldr	r3, [r3, #64]	; 0x40
 8000902:	4a17      	ldr	r2, [pc, #92]	; (8000960 <HAL_UART_MspInit+0x88>)
 8000904:	f443 3300 	orr.w	r3, r3, #131072	; 0x20000
 8000908:	6413      	str	r3, [r2, #64]	; 0x40
 800090a:	4b15      	ldr	r3, [pc, #84]	; (8000960 <HAL_UART_MspInit+0x88>)
 800090c:	6c1b      	ldr	r3, [r3, #64]	; 0x40
 800090e:	f403 3300 	and.w	r3, r3, #131072	; 0x20000
 8000912:	613b      	str	r3, [r7, #16]
 8000914:	693b      	ldr	r3, [r7, #16]

    __HAL_RCC_GPIOA_CLK_ENABLE();
 8000916:	2300      	movs	r3, #0
 8000918:	60fb      	str	r3, [r7, #12]
 800091a:	4b11      	ldr	r3, [pc, #68]	; (8000960 <HAL_UART_MspInit+0x88>)
 800091c:	6b1b      	ldr	r3, [r3, #48]	; 0x30
 800091e:	4a10      	ldr	r2, [pc, #64]	; (8000960 <HAL_UART_MspInit+0x88>)
 8000920:	f043 0301 	orr.w	r3, r3, #1
 8000924:	6313      	str	r3, [r2, #48]	; 0x30
 8000926:	4b0e      	ldr	r3, [pc, #56]	; (8000960 <HAL_UART_MspInit+0x88>)
 8000928:	6b1b      	ldr	r3, [r3, #48]	; 0x30
 800092a:	f003 0301 	and.w	r3, r3, #1
 800092e:	60fb      	str	r3, [r7, #12]
 8000930:	68fb      	ldr	r3, [r7, #12]
    /**USART2 GPIO Configuration
    PA2     ------> USART2_TX
    PA3     ------> USART2_RX
    */
    GPIO_InitStruct.Pin = GPIO_PIN_2|GPIO_PIN_3;
 8000932:	230c      	movs	r3, #12
 8000934:	617b      	str	r3, [r7, #20]
    GPIO_InitStruct.Mode = GPIO_MODE_AF_PP;
 8000936:	2302      	movs	r3, #2
 8000938:	61bb      	str	r3, [r7, #24]
    GPIO_InitStruct.Pull = GPIO_NOPULL;
 800093a:	2300      	movs	r3, #0
 800093c:	61fb      	str	r3, [r7, #28]
    GPIO_InitStruct.Speed = GPIO_SPEED_FREQ_VERY_HIGH;
 800093e:	2303      	movs	r3, #3
 8000940:	623b      	str	r3, [r7, #32]
    GPIO_InitStruct.Alternate = GPIO_AF7_USART2;
 8000942:	2307      	movs	r3, #7
 8000944:	627b      	str	r3, [r7, #36]	; 0x24
    HAL_GPIO_Init(GPIOA, &GPIO_InitStruct);
 8000946:	f107 0314 	add.w	r3, r7, #20
 800094a:	4619      	mov	r1, r3
 800094c:	4805      	ldr	r0, [pc, #20]	; (8000964 <HAL_UART_MspInit+0x8c>)
 800094e:	f000 f9e3 	bl	8000d18 <HAL_GPIO_Init>
  /* USER CODE BEGIN USART2_MspInit 1 */

  /* USER CODE END USART2_MspInit 1 */
  }

}
 8000952:	bf00      	nop
 8000954:	3728      	adds	r7, #40	; 0x28
 8000956:	46bd      	mov	sp, r7
 8000958:	bd80      	pop	{r7, pc}
 800095a:	bf00      	nop
 800095c:	40004400 	.word	0x40004400
 8000960:	40023800 	.word	0x40023800
 8000964:	40020000 	.word	0x40020000

08000968 <HAL_InitTick>:
  *         reset by HAL_Init() or at any time when clock is configured, by HAL_RCC_ClockConfig().
  * @param  TickPriority: Tick interrupt priority.
  * @retval HAL status
  */
HAL_StatusTypeDef HAL_InitTick(uint32_t TickPriority)
{
 8000968:	b580      	push	{r7, lr}
 800096a:	b08c      	sub	sp, #48	; 0x30
 800096c:	af00      	add	r7, sp, #0
 800096e:	6078      	str	r0, [r7, #4]
  RCC_ClkInitTypeDef    clkconfig;
  uint32_t              uwTimclock = 0;
 8000970:	2300      	movs	r3, #0
 8000972:	62fb      	str	r3, [r7, #44]	; 0x2c
  uint32_t              uwPrescalerValue = 0;
 8000974:	2300      	movs	r3, #0
 8000976:	62bb      	str	r3, [r7, #40]	; 0x28
  uint32_t              pFLatency;
  /*Configure the TIM6 IRQ priority */
  HAL_NVIC_SetPriority(TIM6_DAC_IRQn, TickPriority ,0);
 8000978:	2200      	movs	r2, #0
 800097a:	6879      	ldr	r1, [r7, #4]
 800097c:	2036      	movs	r0, #54	; 0x36
 800097e:	f000 f9a1 	bl	8000cc4 <HAL_NVIC_SetPriority>

  /* Enable the TIM6 global Interrupt */
  HAL_NVIC_EnableIRQ(TIM6_DAC_IRQn);
 8000982:	2036      	movs	r0, #54	; 0x36
 8000984:	f000 f9ba 	bl	8000cfc <HAL_NVIC_EnableIRQ>
  /* Enable TIM6 clock */
  __HAL_RCC_TIM6_CLK_ENABLE();
 8000988:	2300      	movs	r3, #0
 800098a:	60fb      	str	r3, [r7, #12]
 800098c:	4b1e      	ldr	r3, [pc, #120]	; (8000a08 <HAL_InitTick+0xa0>)
 800098e:	6c1b      	ldr	r3, [r3, #64]	; 0x40
 8000990:	4a1d      	ldr	r2, [pc, #116]	; (8000a08 <HAL_InitTick+0xa0>)
 8000992:	f043 0310 	orr.w	r3, r3, #16
 8000996:	6413      	str	r3, [r2, #64]	; 0x40
 8000998:	4b1b      	ldr	r3, [pc, #108]	; (8000a08 <HAL_InitTick+0xa0>)
 800099a:	6c1b      	ldr	r3, [r3, #64]	; 0x40
 800099c:	f003 0310 	and.w	r3, r3, #16
 80009a0:	60fb      	str	r3, [r7, #12]
 80009a2:	68fb      	ldr	r3, [r7, #12]

  /* Get clock configuration */
  HAL_RCC_GetClockConfig(&clkconfig, &pFLatency);
 80009a4:	f107 0210 	add.w	r2, r7, #16
 80009a8:	f107 0314 	add.w	r3, r7, #20
 80009ac:	4611      	mov	r1, r2
 80009ae:	4618      	mov	r0, r3
 80009b0:	f000 fff6 	bl	80019a0 <HAL_RCC_GetClockConfig>

  /* Compute TIM6 clock */
  uwTimclock = HAL_RCC_GetPCLK1Freq();
 80009b4:	f000 ffcc 	bl	8001950 <HAL_RCC_GetPCLK1Freq>
 80009b8:	62f8      	str	r0, [r7, #44]	; 0x2c
  /* Compute the prescaler value to have TIM6 counter clock equal to 1MHz */
  uwPrescalerValue = (uint32_t) ((uwTimclock / 1000000U) - 1U);
 80009ba:	6afb      	ldr	r3, [r7, #44]	; 0x2c
 80009bc:	4a13      	ldr	r2, [pc, #76]	; (8000a0c <HAL_InitTick+0xa4>)
 80009be:	fba2 2303 	umull	r2, r3, r2, r3
 80009c2:	0c9b      	lsrs	r3, r3, #18
 80009c4:	3b01      	subs	r3, #1
 80009c6:	62bb      	str	r3, [r7, #40]	; 0x28

  /* Initialize TIM6 */
  htim6.Instance = TIM6;
 80009c8:	4b11      	ldr	r3, [pc, #68]	; (8000a10 <HAL_InitTick+0xa8>)
 80009ca:	4a12      	ldr	r2, [pc, #72]	; (8000a14 <HAL_InitTick+0xac>)
 80009cc:	601a      	str	r2, [r3, #0]
  + Period = [(TIM6CLK/1000) - 1]. to have a (1/1000) s time base.
  + Prescaler = (uwTimclock/1000000 - 1) to have a 1MHz counter clock.
  + ClockDivision = 0
  + Counter direction = Up
  */
  htim6.Init.Period = (1000000U / 1000U) - 1U;
 80009ce:	4b10      	ldr	r3, [pc, #64]	; (8000a10 <HAL_InitTick+0xa8>)
 80009d0:	f240 32e7 	movw	r2, #999	; 0x3e7
 80009d4:	60da      	str	r2, [r3, #12]
  htim6.Init.Prescaler = uwPrescalerValue;
 80009d6:	4a0e      	ldr	r2, [pc, #56]	; (8000a10 <HAL_InitTick+0xa8>)
 80009d8:	6abb      	ldr	r3, [r7, #40]	; 0x28
 80009da:	6053      	str	r3, [r2, #4]
  htim6.Init.ClockDivision = 0;
 80009dc:	4b0c      	ldr	r3, [pc, #48]	; (8000a10 <HAL_InitTick+0xa8>)
 80009de:	2200      	movs	r2, #0
 80009e0:	611a      	str	r2, [r3, #16]
  htim6.Init.CounterMode = TIM_COUNTERMODE_UP;
 80009e2:	4b0b      	ldr	r3, [pc, #44]	; (8000a10 <HAL_InitTick+0xa8>)
 80009e4:	2200      	movs	r2, #0
 80009e6:	609a      	str	r2, [r3, #8]
  if(HAL_TIM_Base_Init(&htim6) == HAL_OK)
 80009e8:	4809      	ldr	r0, [pc, #36]	; (8000a10 <HAL_InitTick+0xa8>)
 80009ea:	f001 f80b 	bl	8001a04 <HAL_TIM_Base_Init>
 80009ee:	4603      	mov	r3, r0
 80009f0:	2b00      	cmp	r3, #0
 80009f2:	d104      	bne.n	80009fe <HAL_InitTick+0x96>
  {
    /* Start the TIM time Base generation in interrupt mode */
    return HAL_TIM_Base_Start_IT(&htim6);
 80009f4:	4806      	ldr	r0, [pc, #24]	; (8000a10 <HAL_InitTick+0xa8>)
 80009f6:	f001 f85f 	bl	8001ab8 <HAL_TIM_Base_Start_IT>
 80009fa:	4603      	mov	r3, r0
 80009fc:	e000      	b.n	8000a00 <HAL_InitTick+0x98>
  }

  /* Return function status */
  return HAL_ERROR;
 80009fe:	2301      	movs	r3, #1
}
 8000a00:	4618      	mov	r0, r3
 8000a02:	3730      	adds	r7, #48	; 0x30
 8000a04:	46bd      	mov	sp, r7
 8000a06:	bd80      	pop	{r7, pc}
 8000a08:	40023800 	.word	0x40023800
 8000a0c:	431bde83 	.word	0x431bde83
 8000a10:	2000401c 	.word	0x2000401c
 8000a14:	40001000 	.word	0x40001000

08000a18 <NMI_Handler>:
/******************************************************************************/
/**
  * @brief This function handles Non maskable interrupt.
  */
void NMI_Handler(void)
{
 8000a18:	b480      	push	{r7}
 8000a1a:	af00      	add	r7, sp, #0
  /* USER CODE BEGIN NonMaskableInt_IRQn 0 */

  /* USER CODE END NonMaskableInt_IRQn 0 */
  /* USER CODE BEGIN NonMaskableInt_IRQn 1 */
  while (1)
 8000a1c:	e7fe      	b.n	8000a1c <NMI_Handler+0x4>

08000a1e <HardFault_Handler>:

/**
  * @brief This function handles Hard fault interrupt.
  */
void HardFault_Handler(void)
{
 8000a1e:	b480      	push	{r7}
 8000a20:	af00      	add	r7, sp, #0
  /* USER CODE BEGIN HardFault_IRQn 0 */

  /* USER CODE END HardFault_IRQn 0 */
  while (1)
 8000a22:	e7fe      	b.n	8000a22 <HardFault_Handler+0x4>

08000a24 <MemManage_Handler>:

/**
  * @brief This function handles Memory management fault.
  */
void MemManage_Handler(void)
{
 8000a24:	b480      	push	{r7}
 8000a26:	af00      	add	r7, sp, #0
  /* USER CODE BEGIN MemoryManagement_IRQn 0 */

  /* USER CODE END MemoryManagement_IRQn 0 */
  while (1)
 8000a28:	e7fe      	b.n	8000a28 <MemManage_Handler+0x4>

08000a2a <BusFault_Handler>:

/**
  * @brief This function handles Pre-fetch fault, memory access fault.
  */
void BusFault_Handler(void)
{
 8000a2a:	b480      	push	{r7}
 8000a2c:	af00      	add	r7, sp, #0
  /* USER CODE BEGIN BusFault_IRQn 0 */

  /* USER CODE END BusFault_IRQn 0 */
  while (1)
 8000a2e:	e7fe      	b.n	8000a2e <BusFault_Handler+0x4>

08000a30 <UsageFault_Handler>:

/**
  * @brief This function handles Undefined instruction or illegal state.
  */
void UsageFault_Handler(void)
{
 8000a30:	b480      	push	{r7}
 8000a32:	af00      	add	r7, sp, #0
  /* USER CODE BEGIN UsageFault_IRQn 0 */

  /* USER CODE END UsageFault_IRQn 0 */
  while (1)
 8000a34:	e7fe      	b.n	8000a34 <UsageFault_Handler+0x4>

08000a36 <DebugMon_Handler>:

/**
  * @brief This function handles Debug monitor.
  */
void DebugMon_Handler(void)
{
 8000a36:	b480      	push	{r7}
 8000a38:	af00      	add	r7, sp, #0

  /* USER CODE END DebugMonitor_IRQn 0 */
  /* USER CODE BEGIN DebugMonitor_IRQn 1 */

  /* USER CODE END DebugMonitor_IRQn 1 */
}
 8000a3a:	bf00      	nop
 8000a3c:	46bd      	mov	sp, r7
 8000a3e:	f85d 7b04 	ldr.w	r7, [sp], #4
 8000a42:	4770      	bx	lr

08000a44 <TIM6_DAC_IRQHandler>:

/**
  * @brief This function handles TIM6 global interrupt, DAC1 and DAC2 underrun error interrupts.
  */
void TIM6_DAC_IRQHandler(void)
{
 8000a44:	b580      	push	{r7, lr}
 8000a46:	af00      	add	r7, sp, #0
  /* USER CODE BEGIN TIM6_DAC_IRQn 0 */

  /* USER CODE END TIM6_DAC_IRQn 0 */
  HAL_TIM_IRQHandler(&htim6);
 8000a48:	4802      	ldr	r0, [pc, #8]	; (8000a54 <TIM6_DAC_IRQHandler+0x10>)
 8000a4a:	f001 f8a5 	bl	8001b98 <HAL_TIM_IRQHandler>
  /* USER CODE BEGIN TIM6_DAC_IRQn 1 */

  /* USER CODE END TIM6_DAC_IRQn 1 */
}
 8000a4e:	bf00      	nop
 8000a50:	bd80      	pop	{r7, pc}
 8000a52:	bf00      	nop
 8000a54:	2000401c 	.word	0x2000401c

08000a58 <SystemInit>:
  *         configuration.
  * @param  None
  * @retval None
  */
void SystemInit(void)
{
 8000a58:	b480      	push	{r7}
 8000a5a:	af00      	add	r7, sp, #0
  /* FPU settings ------------------------------------------------------------*/
  #if (__FPU_PRESENT == 1) && (__FPU_USED == 1)
    SCB->CPACR |= ((3UL << 10*2)|(3UL << 11*2));  /* set CP10 and CP11 Full Access */
 8000a5c:	4b06      	ldr	r3, [pc, #24]	; (8000a78 <SystemInit+0x20>)
 8000a5e:	f8d3 3088 	ldr.w	r3, [r3, #136]	; 0x88
 8000a62:	4a05      	ldr	r2, [pc, #20]	; (8000a78 <SystemInit+0x20>)
 8000a64:	f443 0370 	orr.w	r3, r3, #15728640	; 0xf00000
 8000a68:	f8c2 3088 	str.w	r3, [r2, #136]	; 0x88

  /* Configure the Vector Table location -------------------------------------*/
#if defined(USER_VECT_TAB_ADDRESS)
  SCB->VTOR = VECT_TAB_BASE_ADDRESS | VECT_TAB_OFFSET; /* Vector Table Relocation in Internal SRAM */
#endif /* USER_VECT_TAB_ADDRESS */
}
 8000a6c:	bf00      	nop
 8000a6e:	46bd      	mov	sp, r7
 8000a70:	f85d 7b04 	ldr.w	r7, [sp], #4
 8000a74:	4770      	bx	lr
 8000a76:	bf00      	nop
 8000a78:	e000ed00 	.word	0xe000ed00

08000a7c <Reset_Handler>:

    .section  .text.Reset_Handler
  .weak  Reset_Handler
  .type  Reset_Handler, %function
Reset_Handler:  
  ldr   sp, =_estack     /* set stack pointer */
 8000a7c:	f8df d034 	ldr.w	sp, [pc, #52]	; 8000ab4 <LoopFillZerobss+0x12>

/* Copy the data segment initializers from flash to SRAM */  
  ldr r0, =_sdata
 8000a80:	480d      	ldr	r0, [pc, #52]	; (8000ab8 <LoopFillZerobss+0x16>)
  ldr r1, =_edata
 8000a82:	490e      	ldr	r1, [pc, #56]	; (8000abc <LoopFillZerobss+0x1a>)
  ldr r2, =_sidata
 8000a84:	4a0e      	ldr	r2, [pc, #56]	; (8000ac0 <LoopFillZerobss+0x1e>)
  movs r3, #0
 8000a86:	2300      	movs	r3, #0
  b LoopCopyDataInit
 8000a88:	e002      	b.n	8000a90 <LoopCopyDataInit>

08000a8a <CopyDataInit>:

CopyDataInit:
  ldr r4, [r2, r3]
 8000a8a:	58d4      	ldr	r4, [r2, r3]
  str r4, [r0, r3]
 8000a8c:	50c4      	str	r4, [r0, r3]
  adds r3, r3, #4
 8000a8e:	3304      	adds	r3, #4

08000a90 <LoopCopyDataInit>:

LoopCopyDataInit:
  adds r4, r0, r3
 8000a90:	18c4      	adds	r4, r0, r3
  cmp r4, r1
 8000a92:	428c      	cmp	r4, r1
  bcc CopyDataInit
 8000a94:	d3f9      	bcc.n	8000a8a <CopyDataInit>
  
/* Zero fill the bss segment. */
  ldr r2, =_sbss
 8000a96:	4a0b      	ldr	r2, [pc, #44]	; (8000ac4 <LoopFillZerobss+0x22>)
  ldr r4, =_ebss
 8000a98:	4c0b      	ldr	r4, [pc, #44]	; (8000ac8 <LoopFillZerobss+0x26>)
  movs r3, #0
 8000a9a:	2300      	movs	r3, #0
  b LoopFillZerobss
 8000a9c:	e001      	b.n	8000aa2 <LoopFillZerobss>

08000a9e <FillZerobss>:

FillZerobss:
  str  r3, [r2]
 8000a9e:	6013      	str	r3, [r2, #0]
  adds r2, r2, #4
 8000aa0:	3204      	adds	r2, #4

08000aa2 <LoopFillZerobss>:

LoopFillZerobss:
  cmp r2, r4
 8000aa2:	42a2      	cmp	r2, r4
  bcc FillZerobss
 8000aa4:	d3fb      	bcc.n	8000a9e <FillZerobss>

/* Call the clock system intitialization function.*/
  bl  SystemInit   
 8000aa6:	f7ff ffd7 	bl	8000a58 <SystemInit>
/* Call static constructors */
    bl __libc_init_array
 8000aaa:	f003 f86f 	bl	8003b8c <__libc_init_array>
/* Call the application's entry point.*/
  bl  main
 8000aae:	f7ff fd5b 	bl	8000568 <main>
  bx  lr    
 8000ab2:	4770      	bx	lr
  ldr   sp, =_estack     /* set stack pointer */
 8000ab4:	20020000 	.word	0x20020000
  ldr r0, =_sdata
 8000ab8:	20000000 	.word	0x20000000
  ldr r1, =_edata
 8000abc:	20000010 	.word	0x20000010
  ldr r2, =_sidata
 8000ac0:	08003c9c 	.word	0x08003c9c
  ldr r2, =_sbss
 8000ac4:	20000010 	.word	0x20000010
  ldr r4, =_ebss
 8000ac8:	20004068 	.word	0x20004068

08000acc <ADC_IRQHandler>:
 * @retval None       
*/
    .section  .text.Default_Handler,"ax",%progbits
Default_Handler:
Infinite_Loop:
  b  Infinite_Loop
 8000acc:	e7fe      	b.n	8000acc <ADC_IRQHandler>
	...

08000ad0 <HAL_Init>:
  *         need to ensure that the SysTick time base is always set to 1 millisecond
  *         to have correct HAL operation.
  * @retval HAL status
  */
HAL_StatusTypeDef HAL_Init(void)
{
 8000ad0:	b580      	push	{r7, lr}
 8000ad2:	af00      	add	r7, sp, #0
  /* Configure Flash prefetch, Instruction cache, Data cache */ 
#if (INSTRUCTION_CACHE_ENABLE != 0U)
  __HAL_FLASH_INSTRUCTION_CACHE_ENABLE();
 8000ad4:	4b0e      	ldr	r3, [pc, #56]	; (8000b10 <HAL_Init+0x40>)
 8000ad6:	681b      	ldr	r3, [r3, #0]
 8000ad8:	4a0d      	ldr	r2, [pc, #52]	; (8000b10 <HAL_Init+0x40>)
 8000ada:	f443 7300 	orr.w	r3, r3, #512	; 0x200
 8000ade:	6013      	str	r3, [r2, #0]
#endif /* INSTRUCTION_CACHE_ENABLE */

#if (DATA_CACHE_ENABLE != 0U)
  __HAL_FLASH_DATA_CACHE_ENABLE();
 8000ae0:	4b0b      	ldr	r3, [pc, #44]	; (8000b10 <HAL_Init+0x40>)
 8000ae2:	681b      	ldr	r3, [r3, #0]
 8000ae4:	4a0a      	ldr	r2, [pc, #40]	; (8000b10 <HAL_Init+0x40>)
 8000ae6:	f443 6380 	orr.w	r3, r3, #1024	; 0x400
 8000aea:	6013      	str	r3, [r2, #0]
#endif /* DATA_CACHE_ENABLE */

#if (PREFETCH_ENABLE != 0U)
  __HAL_FLASH_PREFETCH_BUFFER_ENABLE();
 8000aec:	4b08      	ldr	r3, [pc, #32]	; (8000b10 <HAL_Init+0x40>)
 8000aee:	681b      	ldr	r3, [r3, #0]
 8000af0:	4a07      	ldr	r2, [pc, #28]	; (8000b10 <HAL_Init+0x40>)
 8000af2:	f443 7380 	orr.w	r3, r3, #256	; 0x100
 8000af6:	6013      	str	r3, [r2, #0]
#endif /* PREFETCH_ENABLE */

  /* Set Interrupt Group Priority */
  HAL_NVIC_SetPriorityGrouping(NVIC_PRIORITYGROUP_4);
 8000af8:	2003      	movs	r0, #3
 8000afa:	f000 f8d8 	bl	8000cae <HAL_NVIC_SetPriorityGrouping>

  /* Use systick as time base source and configure 1ms tick (default clock after Reset is HSI) */
  HAL_InitTick(TICK_INT_PRIORITY);
 8000afe:	2000      	movs	r0, #0
 8000b00:	f7ff ff32 	bl	8000968 <HAL_InitTick>

  /* Init the low level hardware */
  HAL_MspInit();
 8000b04:	f7ff febc 	bl	8000880 <HAL_MspInit>

  /* Return function status */
  return HAL_OK;
 8000b08:	2300      	movs	r3, #0
}
 8000b0a:	4618      	mov	r0, r3
 8000b0c:	bd80      	pop	{r7, pc}
 8000b0e:	bf00      	nop
 8000b10:	40023c00 	.word	0x40023c00

08000b14 <HAL_IncTick>:
 * @note This function is declared as __weak to be overwritten in case of other 
  *      implementations in user file.
  * @retval None
  */
__weak void HAL_IncTick(void)
{
 8000b14:	b480      	push	{r7}
 8000b16:	af00      	add	r7, sp, #0
  uwTick += uwTickFreq;
 8000b18:	4b06      	ldr	r3, [pc, #24]	; (8000b34 <HAL_IncTick+0x20>)
 8000b1a:	781b      	ldrb	r3, [r3, #0]
 8000b1c:	461a      	mov	r2, r3
 8000b1e:	4b06      	ldr	r3, [pc, #24]	; (8000b38 <HAL_IncTick+0x24>)
 8000b20:	681b      	ldr	r3, [r3, #0]
 8000b22:	4413      	add	r3, r2
 8000b24:	4a04      	ldr	r2, [pc, #16]	; (8000b38 <HAL_IncTick+0x24>)
 8000b26:	6013      	str	r3, [r2, #0]
}
 8000b28:	bf00      	nop
 8000b2a:	46bd      	mov	sp, r7
 8000b2c:	f85d 7b04 	ldr.w	r7, [sp], #4
 8000b30:	4770      	bx	lr
 8000b32:	bf00      	nop
 8000b34:	20000008 	.word	0x20000008
 8000b38:	20004064 	.word	0x20004064

08000b3c <HAL_GetTick>:
  * @note This function is declared as __weak to be overwritten in case of other 
  *       implementations in user file.
  * @retval tick value
  */
__weak uint32_t HAL_GetTick(void)
{
 8000b3c:	b480      	push	{r7}
 8000b3e:	af00      	add	r7, sp, #0
  return uwTick;
 8000b40:	4b03      	ldr	r3, [pc, #12]	; (8000b50 <HAL_GetTick+0x14>)
 8000b42:	681b      	ldr	r3, [r3, #0]
}
 8000b44:	4618      	mov	r0, r3
 8000b46:	46bd      	mov	sp, r7
 8000b48:	f85d 7b04 	ldr.w	r7, [sp], #4
 8000b4c:	4770      	bx	lr
 8000b4e:	bf00      	nop
 8000b50:	20004064 	.word	0x20004064

08000b54 <__NVIC_SetPriorityGrouping>:
           In case of a conflict between priority grouping and available
           priority bits (__NVIC_PRIO_BITS), the smallest possible priority group is set.
  \param [in]      PriorityGroup  Priority grouping field.
 */
__STATIC_INLINE void __NVIC_SetPriorityGrouping(uint32_t PriorityGroup)
{
 8000b54:	b480      	push	{r7}
 8000b56:	b085      	sub	sp, #20
 8000b58:	af00      	add	r7, sp, #0
 8000b5a:	6078      	str	r0, [r7, #4]
  uint32_t reg_value;
  uint32_t PriorityGroupTmp = (PriorityGroup & (uint32_t)0x07UL);             /* only values 0..7 are used          */
 8000b5c:	687b      	ldr	r3, [r7, #4]
 8000b5e:	f003 0307 	and.w	r3, r3, #7
 8000b62:	60fb      	str	r3, [r7, #12]

  reg_value  =  SCB->AIRCR;                                                   /* read old register configuration    */
 8000b64:	4b0c      	ldr	r3, [pc, #48]	; (8000b98 <__NVIC_SetPriorityGrouping+0x44>)
 8000b66:	68db      	ldr	r3, [r3, #12]
 8000b68:	60bb      	str	r3, [r7, #8]
  reg_value &= ~((uint32_t)(SCB_AIRCR_VECTKEY_Msk | SCB_AIRCR_PRIGROUP_Msk)); /* clear bits to change               */
 8000b6a:	68ba      	ldr	r2, [r7, #8]
 8000b6c:	f64f 03ff 	movw	r3, #63743	; 0xf8ff
 8000b70:	4013      	ands	r3, r2
 8000b72:	60bb      	str	r3, [r7, #8]
  reg_value  =  (reg_value                                   |
                ((uint32_t)0x5FAUL << SCB_AIRCR_VECTKEY_Pos) |
                (PriorityGroupTmp << SCB_AIRCR_PRIGROUP_Pos)  );              /* Insert write key and priority group */
 8000b74:	68fb      	ldr	r3, [r7, #12]
 8000b76:	021a      	lsls	r2, r3, #8
                ((uint32_t)0x5FAUL << SCB_AIRCR_VECTKEY_Pos) |
 8000b78:	68bb      	ldr	r3, [r7, #8]
 8000b7a:	4313      	orrs	r3, r2
  reg_value  =  (reg_value                                   |
 8000b7c:	f043 63bf 	orr.w	r3, r3, #100139008	; 0x5f80000
 8000b80:	f443 3300 	orr.w	r3, r3, #131072	; 0x20000
 8000b84:	60bb      	str	r3, [r7, #8]
  SCB->AIRCR =  reg_value;
 8000b86:	4a04      	ldr	r2, [pc, #16]	; (8000b98 <__NVIC_SetPriorityGrouping+0x44>)
 8000b88:	68bb      	ldr	r3, [r7, #8]
 8000b8a:	60d3      	str	r3, [r2, #12]
}
 8000b8c:	bf00      	nop
 8000b8e:	3714      	adds	r7, #20
 8000b90:	46bd      	mov	sp, r7
 8000b92:	f85d 7b04 	ldr.w	r7, [sp], #4
 8000b96:	4770      	bx	lr
 8000b98:	e000ed00 	.word	0xe000ed00

08000b9c <__NVIC_GetPriorityGrouping>:
  \brief   Get Priority Grouping
  \details Reads the priority grouping field from the NVIC Interrupt Controller.
  \return                Priority grouping field (SCB->AIRCR [10:8] PRIGROUP field).
 */
__STATIC_INLINE uint32_t __NVIC_GetPriorityGrouping(void)
{
 8000b9c:	b480      	push	{r7}
 8000b9e:	af00      	add	r7, sp, #0
  return ((uint32_t)((SCB->AIRCR & SCB_AIRCR_PRIGROUP_Msk) >> SCB_AIRCR_PRIGROUP_Pos));
 8000ba0:	4b04      	ldr	r3, [pc, #16]	; (8000bb4 <__NVIC_GetPriorityGrouping+0x18>)
 8000ba2:	68db      	ldr	r3, [r3, #12]
 8000ba4:	0a1b      	lsrs	r3, r3, #8
 8000ba6:	f003 0307 	and.w	r3, r3, #7
}
 8000baa:	4618      	mov	r0, r3
 8000bac:	46bd      	mov	sp, r7
 8000bae:	f85d 7b04 	ldr.w	r7, [sp], #4
 8000bb2:	4770      	bx	lr
 8000bb4:	e000ed00 	.word	0xe000ed00

08000bb8 <__NVIC_EnableIRQ>:
  \details Enables a device specific interrupt in the NVIC interrupt controller.
  \param [in]      IRQn  Device specific interrupt number.
  \note    IRQn must not be negative.
 */
__STATIC_INLINE void __NVIC_EnableIRQ(IRQn_Type IRQn)
{
 8000bb8:	b480      	push	{r7}
 8000bba:	b083      	sub	sp, #12
 8000bbc:	af00      	add	r7, sp, #0
 8000bbe:	4603      	mov	r3, r0
 8000bc0:	71fb      	strb	r3, [r7, #7]
  if ((int32_t)(IRQn) >= 0)
 8000bc2:	f997 3007 	ldrsb.w	r3, [r7, #7]
 8000bc6:	2b00      	cmp	r3, #0
 8000bc8:	db0b      	blt.n	8000be2 <__NVIC_EnableIRQ+0x2a>
  {
    NVIC->ISER[(((uint32_t)IRQn) >> 5UL)] = (uint32_t)(1UL << (((uint32_t)IRQn) & 0x1FUL));
 8000bca:	79fb      	ldrb	r3, [r7, #7]
 8000bcc:	f003 021f 	and.w	r2, r3, #31
 8000bd0:	4907      	ldr	r1, [pc, #28]	; (8000bf0 <__NVIC_EnableIRQ+0x38>)
 8000bd2:	f997 3007 	ldrsb.w	r3, [r7, #7]
 8000bd6:	095b      	lsrs	r3, r3, #5
 8000bd8:	2001      	movs	r0, #1
 8000bda:	fa00 f202 	lsl.w	r2, r0, r2
 8000bde:	f841 2023 	str.w	r2, [r1, r3, lsl #2]
  }
}
 8000be2:	bf00      	nop
 8000be4:	370c      	adds	r7, #12
 8000be6:	46bd      	mov	sp, r7
 8000be8:	f85d 7b04 	ldr.w	r7, [sp], #4
 8000bec:	4770      	bx	lr
 8000bee:	bf00      	nop
 8000bf0:	e000e100 	.word	0xe000e100

08000bf4 <__NVIC_SetPriority>:
  \param [in]      IRQn  Interrupt number.
  \param [in]  priority  Priority to set.
  \note    The priority cannot be set for every processor exception.
 */
__STATIC_INLINE void __NVIC_SetPriority(IRQn_Type IRQn, uint32_t priority)
{
 8000bf4:	b480      	push	{r7}
 8000bf6:	b083      	sub	sp, #12
 8000bf8:	af00      	add	r7, sp, #0
 8000bfa:	4603      	mov	r3, r0
 8000bfc:	6039      	str	r1, [r7, #0]
 8000bfe:	71fb      	strb	r3, [r7, #7]
  if ((int32_t)(IRQn) >= 0)
 8000c00:	f997 3007 	ldrsb.w	r3, [r7, #7]
 8000c04:	2b00      	cmp	r3, #0
 8000c06:	db0a      	blt.n	8000c1e <__NVIC_SetPriority+0x2a>
  {
    NVIC->IP[((uint32_t)IRQn)]               = (uint8_t)((priority << (8U - __NVIC_PRIO_BITS)) & (uint32_t)0xFFUL);
 8000c08:	683b      	ldr	r3, [r7, #0]
 8000c0a:	b2da      	uxtb	r2, r3
 8000c0c:	490c      	ldr	r1, [pc, #48]	; (8000c40 <__NVIC_SetPriority+0x4c>)
 8000c0e:	f997 3007 	ldrsb.w	r3, [r7, #7]
 8000c12:	0112      	lsls	r2, r2, #4
 8000c14:	b2d2      	uxtb	r2, r2
 8000c16:	440b      	add	r3, r1
 8000c18:	f883 2300 	strb.w	r2, [r3, #768]	; 0x300
  }
  else
  {
    SCB->SHP[(((uint32_t)IRQn) & 0xFUL)-4UL] = (uint8_t)((priority << (8U - __NVIC_PRIO_BITS)) & (uint32_t)0xFFUL);
  }
}
 8000c1c:	e00a      	b.n	8000c34 <__NVIC_SetPriority+0x40>
    SCB->SHP[(((uint32_t)IRQn) & 0xFUL)-4UL] = (uint8_t)((priority << (8U - __NVIC_PRIO_BITS)) & (uint32_t)0xFFUL);
 8000c1e:	683b      	ldr	r3, [r7, #0]
 8000c20:	b2da      	uxtb	r2, r3
 8000c22:	4908      	ldr	r1, [pc, #32]	; (8000c44 <__NVIC_SetPriority+0x50>)
 8000c24:	79fb      	ldrb	r3, [r7, #7]
 8000c26:	f003 030f 	and.w	r3, r3, #15
 8000c2a:	3b04      	subs	r3, #4
 8000c2c:	0112      	lsls	r2, r2, #4
 8000c2e:	b2d2      	uxtb	r2, r2
 8000c30:	440b      	add	r3, r1
 8000c32:	761a      	strb	r2, [r3, #24]
}
 8000c34:	bf00      	nop
 8000c36:	370c      	adds	r7, #12
 8000c38:	46bd      	mov	sp, r7
 8000c3a:	f85d 7b04 	ldr.w	r7, [sp], #4
 8000c3e:	4770      	bx	lr
 8000c40:	e000e100 	.word	0xe000e100
 8000c44:	e000ed00 	.word	0xe000ed00

08000c48 <NVIC_EncodePriority>:
  \param [in]   PreemptPriority  Preemptive priority value (starting from 0).
  \param [in]       SubPriority  Subpriority value (starting from 0).
  \return                        Encoded priority. Value can be used in the function \ref NVIC_SetPriority().
 */
__STATIC_INLINE uint32_t NVIC_EncodePriority (uint32_t PriorityGroup, uint32_t PreemptPriority, uint32_t SubPriority)
{
 8000c48:	b480      	push	{r7}
 8000c4a:	b089      	sub	sp, #36	; 0x24
 8000c4c:	af00      	add	r7, sp, #0
 8000c4e:	60f8      	str	r0, [r7, #12]
 8000c50:	60b9      	str	r1, [r7, #8]
 8000c52:	607a      	str	r2, [r7, #4]
  uint32_t PriorityGroupTmp = (PriorityGroup & (uint32_t)0x07UL);   /* only values 0..7 are used          */
 8000c54:	68fb      	ldr	r3, [r7, #12]
 8000c56:	f003 0307 	and.w	r3, r3, #7
 8000c5a:	61fb      	str	r3, [r7, #28]
  uint32_t PreemptPriorityBits;
  uint32_t SubPriorityBits;

  PreemptPriorityBits = ((7UL - PriorityGroupTmp) > (uint32_t)(__NVIC_PRIO_BITS)) ? (uint32_t)(__NVIC_PRIO_BITS) : (uint32_t)(7UL - PriorityGroupTmp);
 8000c5c:	69fb      	ldr	r3, [r7, #28]
 8000c5e:	f1c3 0307 	rsb	r3, r3, #7
 8000c62:	2b04      	cmp	r3, #4
 8000c64:	bf28      	it	cs
 8000c66:	2304      	movcs	r3, #4
 8000c68:	61bb      	str	r3, [r7, #24]
  SubPriorityBits     = ((PriorityGroupTmp + (uint32_t)(__NVIC_PRIO_BITS)) < (uint32_t)7UL) ? (uint32_t)0UL : (uint32_t)((PriorityGroupTmp - 7UL) + (uint32_t)(__NVIC_PRIO_BITS));
 8000c6a:	69fb      	ldr	r3, [r7, #28]
 8000c6c:	3304      	adds	r3, #4
 8000c6e:	2b06      	cmp	r3, #6
 8000c70:	d902      	bls.n	8000c78 <NVIC_EncodePriority+0x30>
 8000c72:	69fb      	ldr	r3, [r7, #28]
 8000c74:	3b03      	subs	r3, #3
 8000c76:	e000      	b.n	8000c7a <NVIC_EncodePriority+0x32>
 8000c78:	2300      	movs	r3, #0
 8000c7a:	617b      	str	r3, [r7, #20]

  return (
           ((PreemptPriority & (uint32_t)((1UL << (PreemptPriorityBits)) - 1UL)) << SubPriorityBits) |
 8000c7c:	f04f 32ff 	mov.w	r2, #4294967295
 8000c80:	69bb      	ldr	r3, [r7, #24]
 8000c82:	fa02 f303 	lsl.w	r3, r2, r3
 8000c86:	43da      	mvns	r2, r3
 8000c88:	68bb      	ldr	r3, [r7, #8]
 8000c8a:	401a      	ands	r2, r3
 8000c8c:	697b      	ldr	r3, [r7, #20]
 8000c8e:	409a      	lsls	r2, r3
           ((SubPriority     & (uint32_t)((1UL << (SubPriorityBits    )) - 1UL)))
 8000c90:	f04f 31ff 	mov.w	r1, #4294967295
 8000c94:	697b      	ldr	r3, [r7, #20]
 8000c96:	fa01 f303 	lsl.w	r3, r1, r3
 8000c9a:	43d9      	mvns	r1, r3
 8000c9c:	687b      	ldr	r3, [r7, #4]
 8000c9e:	400b      	ands	r3, r1
           ((PreemptPriority & (uint32_t)((1UL << (PreemptPriorityBits)) - 1UL)) << SubPriorityBits) |
 8000ca0:	4313      	orrs	r3, r2
         );
}
 8000ca2:	4618      	mov	r0, r3
 8000ca4:	3724      	adds	r7, #36	; 0x24
 8000ca6:	46bd      	mov	sp, r7
 8000ca8:	f85d 7b04 	ldr.w	r7, [sp], #4
 8000cac:	4770      	bx	lr

08000cae <HAL_NVIC_SetPriorityGrouping>:
  * @note   When the NVIC_PriorityGroup_0 is selected, IRQ preemption is no more possible. 
  *         The pending IRQ priority will be managed only by the subpriority. 
  * @retval None
  */
void HAL_NVIC_SetPriorityGrouping(uint32_t PriorityGroup)
{
 8000cae:	b580      	push	{r7, lr}
 8000cb0:	b082      	sub	sp, #8
 8000cb2:	af00      	add	r7, sp, #0
 8000cb4:	6078      	str	r0, [r7, #4]
  /* Check the parameters */
  assert_param(IS_NVIC_PRIORITY_GROUP(PriorityGroup));
  
  /* Set the PRIGROUP[10:8] bits according to the PriorityGroup parameter value */
  NVIC_SetPriorityGrouping(PriorityGroup);
 8000cb6:	6878      	ldr	r0, [r7, #4]
 8000cb8:	f7ff ff4c 	bl	8000b54 <__NVIC_SetPriorityGrouping>
}
 8000cbc:	bf00      	nop
 8000cbe:	3708      	adds	r7, #8
 8000cc0:	46bd      	mov	sp, r7
 8000cc2:	bd80      	pop	{r7, pc}

08000cc4 <HAL_NVIC_SetPriority>:
  *         This parameter can be a value between 0 and 15
  *         A lower priority value indicates a higher priority.          
  * @retval None
  */
void HAL_NVIC_SetPriority(IRQn_Type IRQn, uint32_t PreemptPriority, uint32_t SubPriority)
{ 
 8000cc4:	b580      	push	{r7, lr}
 8000cc6:	b086      	sub	sp, #24
 8000cc8:	af00      	add	r7, sp, #0
 8000cca:	4603      	mov	r3, r0
 8000ccc:	60b9      	str	r1, [r7, #8]
 8000cce:	607a      	str	r2, [r7, #4]
 8000cd0:	73fb      	strb	r3, [r7, #15]
  uint32_t prioritygroup = 0x00U;
 8000cd2:	2300      	movs	r3, #0
 8000cd4:	617b      	str	r3, [r7, #20]
  
  /* Check the parameters */
  assert_param(IS_NVIC_SUB_PRIORITY(SubPriority));
  assert_param(IS_NVIC_PREEMPTION_PRIORITY(PreemptPriority));
  
  prioritygroup = NVIC_GetPriorityGrouping();
 8000cd6:	f7ff ff61 	bl	8000b9c <__NVIC_GetPriorityGrouping>
 8000cda:	6178      	str	r0, [r7, #20]
  
  NVIC_SetPriority(IRQn, NVIC_EncodePriority(prioritygroup, PreemptPriority, SubPriority));
 8000cdc:	687a      	ldr	r2, [r7, #4]
 8000cde:	68b9      	ldr	r1, [r7, #8]
 8000ce0:	6978      	ldr	r0, [r7, #20]
 8000ce2:	f7ff ffb1 	bl	8000c48 <NVIC_EncodePriority>
 8000ce6:	4602      	mov	r2, r0
 8000ce8:	f997 300f 	ldrsb.w	r3, [r7, #15]
 8000cec:	4611      	mov	r1, r2
 8000cee:	4618      	mov	r0, r3
 8000cf0:	f7ff ff80 	bl	8000bf4 <__NVIC_SetPriority>
}
 8000cf4:	bf00      	nop
 8000cf6:	3718      	adds	r7, #24
 8000cf8:	46bd      	mov	sp, r7
 8000cfa:	bd80      	pop	{r7, pc}

08000cfc <HAL_NVIC_EnableIRQ>:
  *         This parameter can be an enumerator of IRQn_Type enumeration
  *         (For the complete STM32 Devices IRQ Channels list, please refer to the appropriate CMSIS device file (stm32f4xxxx.h))
  * @retval None
  */
void HAL_NVIC_EnableIRQ(IRQn_Type IRQn)
{
 8000cfc:	b580      	push	{r7, lr}
 8000cfe:	b082      	sub	sp, #8
 8000d00:	af00      	add	r7, sp, #0
 8000d02:	4603      	mov	r3, r0
 8000d04:	71fb      	strb	r3, [r7, #7]
  /* Check the parameters */
  assert_param(IS_NVIC_DEVICE_IRQ(IRQn));
  
  /* Enable interrupt */
  NVIC_EnableIRQ(IRQn);
 8000d06:	f997 3007 	ldrsb.w	r3, [r7, #7]
 8000d0a:	4618      	mov	r0, r3
 8000d0c:	f7ff ff54 	bl	8000bb8 <__NVIC_EnableIRQ>
}
 8000d10:	bf00      	nop
 8000d12:	3708      	adds	r7, #8
 8000d14:	46bd      	mov	sp, r7
 8000d16:	bd80      	pop	{r7, pc}

08000d18 <HAL_GPIO_Init>:
  * @param  GPIO_Init pointer to a GPIO_InitTypeDef structure that contains
  *         the configuration information for the specified GPIO peripheral.
  * @retval None
  */
void HAL_GPIO_Init(GPIO_TypeDef  *GPIOx, GPIO_InitTypeDef *GPIO_Init)
{
 8000d18:	b480      	push	{r7}
 8000d1a:	b089      	sub	sp, #36	; 0x24
 8000d1c:	af00      	add	r7, sp, #0
 8000d1e:	6078      	str	r0, [r7, #4]
 8000d20:	6039      	str	r1, [r7, #0]
  uint32_t position;
  uint32_t ioposition = 0x00U;
 8000d22:	2300      	movs	r3, #0
 8000d24:	617b      	str	r3, [r7, #20]
  uint32_t iocurrent = 0x00U;
 8000d26:	2300      	movs	r3, #0
 8000d28:	613b      	str	r3, [r7, #16]
  uint32_t temp = 0x00U;
 8000d2a:	2300      	movs	r3, #0
 8000d2c:	61bb      	str	r3, [r7, #24]
  assert_param(IS_GPIO_ALL_INSTANCE(GPIOx));
  assert_param(IS_GPIO_PIN(GPIO_Init->Pin));
  assert_param(IS_GPIO_MODE(GPIO_Init->Mode));

  /* Configure the port pins */
  for(position = 0U; position < GPIO_NUMBER; position++)
 8000d2e:	2300      	movs	r3, #0
 8000d30:	61fb      	str	r3, [r7, #28]
 8000d32:	e16b      	b.n	800100c <HAL_GPIO_Init+0x2f4>
  {
    /* Get the IO position */
    ioposition = 0x01U << position;
 8000d34:	2201      	movs	r2, #1
 8000d36:	69fb      	ldr	r3, [r7, #28]
 8000d38:	fa02 f303 	lsl.w	r3, r2, r3
 8000d3c:	617b      	str	r3, [r7, #20]
    /* Get the current IO position */
    iocurrent = (uint32_t)(GPIO_Init->Pin) & ioposition;
 8000d3e:	683b      	ldr	r3, [r7, #0]
 8000d40:	681b      	ldr	r3, [r3, #0]
 8000d42:	697a      	ldr	r2, [r7, #20]
 8000d44:	4013      	ands	r3, r2
 8000d46:	613b      	str	r3, [r7, #16]

    if(iocurrent == ioposition)
 8000d48:	693a      	ldr	r2, [r7, #16]
 8000d4a:	697b      	ldr	r3, [r7, #20]
 8000d4c:	429a      	cmp	r2, r3
 8000d4e:	f040 815a 	bne.w	8001006 <HAL_GPIO_Init+0x2ee>
    {
      /*--------------------- GPIO Mode Configuration ------------------------*/
      /* In case of Output or Alternate function mode selection */
      if(((GPIO_Init->Mode & GPIO_MODE) == MODE_OUTPUT) || \
 8000d52:	683b      	ldr	r3, [r7, #0]
 8000d54:	685b      	ldr	r3, [r3, #4]
 8000d56:	f003 0303 	and.w	r3, r3, #3
 8000d5a:	2b01      	cmp	r3, #1
 8000d5c:	d005      	beq.n	8000d6a <HAL_GPIO_Init+0x52>
          (GPIO_Init->Mode & GPIO_MODE) == MODE_AF)
 8000d5e:	683b      	ldr	r3, [r7, #0]
 8000d60:	685b      	ldr	r3, [r3, #4]
 8000d62:	f003 0303 	and.w	r3, r3, #3
      if(((GPIO_Init->Mode & GPIO_MODE) == MODE_OUTPUT) || \
 8000d66:	2b02      	cmp	r3, #2
 8000d68:	d130      	bne.n	8000dcc <HAL_GPIO_Init+0xb4>
      {
        /* Check the Speed parameter */
        assert_param(IS_GPIO_SPEED(GPIO_Init->Speed));
        /* Configure the IO Speed */
        temp = GPIOx->OSPEEDR; 
 8000d6a:	687b      	ldr	r3, [r7, #4]
 8000d6c:	689b      	ldr	r3, [r3, #8]
 8000d6e:	61bb      	str	r3, [r7, #24]
        temp &= ~(GPIO_OSPEEDER_OSPEEDR0 << (position * 2U));
 8000d70:	69fb      	ldr	r3, [r7, #28]
 8000d72:	005b      	lsls	r3, r3, #1
 8000d74:	2203      	movs	r2, #3
 8000d76:	fa02 f303 	lsl.w	r3, r2, r3
 8000d7a:	43db      	mvns	r3, r3
 8000d7c:	69ba      	ldr	r2, [r7, #24]
 8000d7e:	4013      	ands	r3, r2
 8000d80:	61bb      	str	r3, [r7, #24]
        temp |= (GPIO_Init->Speed << (position * 2U));
 8000d82:	683b      	ldr	r3, [r7, #0]
 8000d84:	68da      	ldr	r2, [r3, #12]
 8000d86:	69fb      	ldr	r3, [r7, #28]
 8000d88:	005b      	lsls	r3, r3, #1
 8000d8a:	fa02 f303 	lsl.w	r3, r2, r3
 8000d8e:	69ba      	ldr	r2, [r7, #24]
 8000d90:	4313      	orrs	r3, r2
 8000d92:	61bb      	str	r3, [r7, #24]
        GPIOx->OSPEEDR = temp;
 8000d94:	687b      	ldr	r3, [r7, #4]
 8000d96:	69ba      	ldr	r2, [r7, #24]
 8000d98:	609a      	str	r2, [r3, #8]

        /* Configure the IO Output Type */
        temp = GPIOx->OTYPER;
 8000d9a:	687b      	ldr	r3, [r7, #4]
 8000d9c:	685b      	ldr	r3, [r3, #4]
 8000d9e:	61bb      	str	r3, [r7, #24]
        temp &= ~(GPIO_OTYPER_OT_0 << position) ;
 8000da0:	2201      	movs	r2, #1
 8000da2:	69fb      	ldr	r3, [r7, #28]
 8000da4:	fa02 f303 	lsl.w	r3, r2, r3
 8000da8:	43db      	mvns	r3, r3
 8000daa:	69ba      	ldr	r2, [r7, #24]
 8000dac:	4013      	ands	r3, r2
 8000dae:	61bb      	str	r3, [r7, #24]
        temp |= (((GPIO_Init->Mode & OUTPUT_TYPE) >> OUTPUT_TYPE_Pos) << position);
 8000db0:	683b      	ldr	r3, [r7, #0]
 8000db2:	685b      	ldr	r3, [r3, #4]
 8000db4:	091b      	lsrs	r3, r3, #4
 8000db6:	f003 0201 	and.w	r2, r3, #1
 8000dba:	69fb      	ldr	r3, [r7, #28]
 8000dbc:	fa02 f303 	lsl.w	r3, r2, r3
 8000dc0:	69ba      	ldr	r2, [r7, #24]
 8000dc2:	4313      	orrs	r3, r2
 8000dc4:	61bb      	str	r3, [r7, #24]
        GPIOx->OTYPER = temp;
 8000dc6:	687b      	ldr	r3, [r7, #4]
 8000dc8:	69ba      	ldr	r2, [r7, #24]
 8000dca:	605a      	str	r2, [r3, #4]
       }

      if((GPIO_Init->Mode & GPIO_MODE) != MODE_ANALOG)
 8000dcc:	683b      	ldr	r3, [r7, #0]
 8000dce:	685b      	ldr	r3, [r3, #4]
 8000dd0:	f003 0303 	and.w	r3, r3, #3
 8000dd4:	2b03      	cmp	r3, #3
 8000dd6:	d017      	beq.n	8000e08 <HAL_GPIO_Init+0xf0>
      {
        /* Check the parameters */
        assert_param(IS_GPIO_PULL(GPIO_Init->Pull));
        
        /* Activate the Pull-up or Pull down resistor for the current IO */
        temp = GPIOx->PUPDR;
 8000dd8:	687b      	ldr	r3, [r7, #4]
 8000dda:	68db      	ldr	r3, [r3, #12]
 8000ddc:	61bb      	str	r3, [r7, #24]
        temp &= ~(GPIO_PUPDR_PUPDR0 << (position * 2U));
 8000dde:	69fb      	ldr	r3, [r7, #28]
 8000de0:	005b      	lsls	r3, r3, #1
 8000de2:	2203      	movs	r2, #3
 8000de4:	fa02 f303 	lsl.w	r3, r2, r3
 8000de8:	43db      	mvns	r3, r3
 8000dea:	69ba      	ldr	r2, [r7, #24]
 8000dec:	4013      	ands	r3, r2
 8000dee:	61bb      	str	r3, [r7, #24]
        temp |= ((GPIO_Init->Pull) << (position * 2U));
 8000df0:	683b      	ldr	r3, [r7, #0]
 8000df2:	689a      	ldr	r2, [r3, #8]
 8000df4:	69fb      	ldr	r3, [r7, #28]
 8000df6:	005b      	lsls	r3, r3, #1
 8000df8:	fa02 f303 	lsl.w	r3, r2, r3
 8000dfc:	69ba      	ldr	r2, [r7, #24]
 8000dfe:	4313      	orrs	r3, r2
 8000e00:	61bb      	str	r3, [r7, #24]
        GPIOx->PUPDR = temp;
 8000e02:	687b      	ldr	r3, [r7, #4]
 8000e04:	69ba      	ldr	r2, [r7, #24]
 8000e06:	60da      	str	r2, [r3, #12]
      }

      /* In case of Alternate function mode selection */
      if((GPIO_Init->Mode & GPIO_MODE) == MODE_AF)
 8000e08:	683b      	ldr	r3, [r7, #0]
 8000e0a:	685b      	ldr	r3, [r3, #4]
 8000e0c:	f003 0303 	and.w	r3, r3, #3
 8000e10:	2b02      	cmp	r3, #2
 8000e12:	d123      	bne.n	8000e5c <HAL_GPIO_Init+0x144>
      {
        /* Check the Alternate function parameter */
        assert_param(IS_GPIO_AF(GPIO_Init->Alternate));
        /* Configure Alternate function mapped with the current IO */
        temp = GPIOx->AFR[position >> 3U];
 8000e14:	69fb      	ldr	r3, [r7, #28]
 8000e16:	08da      	lsrs	r2, r3, #3
 8000e18:	687b      	ldr	r3, [r7, #4]
 8000e1a:	3208      	adds	r2, #8
 8000e1c:	f853 3022 	ldr.w	r3, [r3, r2, lsl #2]
 8000e20:	61bb      	str	r3, [r7, #24]
        temp &= ~(0xFU << ((uint32_t)(position & 0x07U) * 4U)) ;
 8000e22:	69fb      	ldr	r3, [r7, #28]
 8000e24:	f003 0307 	and.w	r3, r3, #7
 8000e28:	009b      	lsls	r3, r3, #2
 8000e2a:	220f      	movs	r2, #15
 8000e2c:	fa02 f303 	lsl.w	r3, r2, r3
 8000e30:	43db      	mvns	r3, r3
 8000e32:	69ba      	ldr	r2, [r7, #24]
 8000e34:	4013      	ands	r3, r2
 8000e36:	61bb      	str	r3, [r7, #24]
        temp |= ((uint32_t)(GPIO_Init->Alternate) << (((uint32_t)position & 0x07U) * 4U));
 8000e38:	683b      	ldr	r3, [r7, #0]
 8000e3a:	691a      	ldr	r2, [r3, #16]
 8000e3c:	69fb      	ldr	r3, [r7, #28]
 8000e3e:	f003 0307 	and.w	r3, r3, #7
 8000e42:	009b      	lsls	r3, r3, #2
 8000e44:	fa02 f303 	lsl.w	r3, r2, r3
 8000e48:	69ba      	ldr	r2, [r7, #24]
 8000e4a:	4313      	orrs	r3, r2
 8000e4c:	61bb      	str	r3, [r7, #24]
        GPIOx->AFR[position >> 3U] = temp;
 8000e4e:	69fb      	ldr	r3, [r7, #28]
 8000e50:	08da      	lsrs	r2, r3, #3
 8000e52:	687b      	ldr	r3, [r7, #4]
 8000e54:	3208      	adds	r2, #8
 8000e56:	69b9      	ldr	r1, [r7, #24]
 8000e58:	f843 1022 	str.w	r1, [r3, r2, lsl #2]
      }

      /* Configure IO Direction mode (Input, Output, Alternate or Analog) */
      temp = GPIOx->MODER;
 8000e5c:	687b      	ldr	r3, [r7, #4]
 8000e5e:	681b      	ldr	r3, [r3, #0]
 8000e60:	61bb      	str	r3, [r7, #24]
      temp &= ~(GPIO_MODER_MODER0 << (position * 2U));
 8000e62:	69fb      	ldr	r3, [r7, #28]
 8000e64:	005b      	lsls	r3, r3, #1
 8000e66:	2203      	movs	r2, #3
 8000e68:	fa02 f303 	lsl.w	r3, r2, r3
 8000e6c:	43db      	mvns	r3, r3
 8000e6e:	69ba      	ldr	r2, [r7, #24]
 8000e70:	4013      	ands	r3, r2
 8000e72:	61bb      	str	r3, [r7, #24]
      temp |= ((GPIO_Init->Mode & GPIO_MODE) << (position * 2U));
 8000e74:	683b      	ldr	r3, [r7, #0]
 8000e76:	685b      	ldr	r3, [r3, #4]
 8000e78:	f003 0203 	and.w	r2, r3, #3
 8000e7c:	69fb      	ldr	r3, [r7, #28]
 8000e7e:	005b      	lsls	r3, r3, #1
 8000e80:	fa02 f303 	lsl.w	r3, r2, r3
 8000e84:	69ba      	ldr	r2, [r7, #24]
 8000e86:	4313      	orrs	r3, r2
 8000e88:	61bb      	str	r3, [r7, #24]
      GPIOx->MODER = temp;
 8000e8a:	687b      	ldr	r3, [r7, #4]
 8000e8c:	69ba      	ldr	r2, [r7, #24]
 8000e8e:	601a      	str	r2, [r3, #0]

      /*--------------------- EXTI Mode Configuration ------------------------*/
      /* Configure the External Interrupt or event for the current IO */
      if((GPIO_Init->Mode & EXTI_MODE) != 0x00U)
 8000e90:	683b      	ldr	r3, [r7, #0]
 8000e92:	685b      	ldr	r3, [r3, #4]
 8000e94:	f403 3340 	and.w	r3, r3, #196608	; 0x30000
 8000e98:	2b00      	cmp	r3, #0
 8000e9a:	f000 80b4 	beq.w	8001006 <HAL_GPIO_Init+0x2ee>
      {
        /* Enable SYSCFG Clock */
        __HAL_RCC_SYSCFG_CLK_ENABLE();
 8000e9e:	2300      	movs	r3, #0
 8000ea0:	60fb      	str	r3, [r7, #12]
 8000ea2:	4b60      	ldr	r3, [pc, #384]	; (8001024 <HAL_GPIO_Init+0x30c>)
 8000ea4:	6c5b      	ldr	r3, [r3, #68]	; 0x44
 8000ea6:	4a5f      	ldr	r2, [pc, #380]	; (8001024 <HAL_GPIO_Init+0x30c>)
 8000ea8:	f443 4380 	orr.w	r3, r3, #16384	; 0x4000
 8000eac:	6453      	str	r3, [r2, #68]	; 0x44
 8000eae:	4b5d      	ldr	r3, [pc, #372]	; (8001024 <HAL_GPIO_Init+0x30c>)
 8000eb0:	6c5b      	ldr	r3, [r3, #68]	; 0x44
 8000eb2:	f403 4380 	and.w	r3, r3, #16384	; 0x4000
 8000eb6:	60fb      	str	r3, [r7, #12]
 8000eb8:	68fb      	ldr	r3, [r7, #12]

        temp = SYSCFG->EXTICR[position >> 2U];
 8000eba:	4a5b      	ldr	r2, [pc, #364]	; (8001028 <HAL_GPIO_Init+0x310>)
 8000ebc:	69fb      	ldr	r3, [r7, #28]
 8000ebe:	089b      	lsrs	r3, r3, #2
 8000ec0:	3302      	adds	r3, #2
 8000ec2:	f852 3023 	ldr.w	r3, [r2, r3, lsl #2]
 8000ec6:	61bb      	str	r3, [r7, #24]
        temp &= ~(0x0FU << (4U * (position & 0x03U)));
 8000ec8:	69fb      	ldr	r3, [r7, #28]
 8000eca:	f003 0303 	and.w	r3, r3, #3
 8000ece:	009b      	lsls	r3, r3, #2
 8000ed0:	220f      	movs	r2, #15
 8000ed2:	fa02 f303 	lsl.w	r3, r2, r3
 8000ed6:	43db      	mvns	r3, r3
 8000ed8:	69ba      	ldr	r2, [r7, #24]
 8000eda:	4013      	ands	r3, r2
 8000edc:	61bb      	str	r3, [r7, #24]
        temp |= ((uint32_t)(GPIO_GET_INDEX(GPIOx)) << (4U * (position & 0x03U)));
 8000ede:	687b      	ldr	r3, [r7, #4]
 8000ee0:	4a52      	ldr	r2, [pc, #328]	; (800102c <HAL_GPIO_Init+0x314>)
 8000ee2:	4293      	cmp	r3, r2
 8000ee4:	d02b      	beq.n	8000f3e <HAL_GPIO_Init+0x226>
 8000ee6:	687b      	ldr	r3, [r7, #4]
 8000ee8:	4a51      	ldr	r2, [pc, #324]	; (8001030 <HAL_GPIO_Init+0x318>)
 8000eea:	4293      	cmp	r3, r2
 8000eec:	d025      	beq.n	8000f3a <HAL_GPIO_Init+0x222>
 8000eee:	687b      	ldr	r3, [r7, #4]
 8000ef0:	4a50      	ldr	r2, [pc, #320]	; (8001034 <HAL_GPIO_Init+0x31c>)
 8000ef2:	4293      	cmp	r3, r2
 8000ef4:	d01f      	beq.n	8000f36 <HAL_GPIO_Init+0x21e>
 8000ef6:	687b      	ldr	r3, [r7, #4]
 8000ef8:	4a4f      	ldr	r2, [pc, #316]	; (8001038 <HAL_GPIO_Init+0x320>)
 8000efa:	4293      	cmp	r3, r2
 8000efc:	d019      	beq.n	8000f32 <HAL_GPIO_Init+0x21a>
 8000efe:	687b      	ldr	r3, [r7, #4]
 8000f00:	4a4e      	ldr	r2, [pc, #312]	; (800103c <HAL_GPIO_Init+0x324>)
 8000f02:	4293      	cmp	r3, r2
 8000f04:	d013      	beq.n	8000f2e <HAL_GPIO_Init+0x216>
 8000f06:	687b      	ldr	r3, [r7, #4]
 8000f08:	4a4d      	ldr	r2, [pc, #308]	; (8001040 <HAL_GPIO_Init+0x328>)
 8000f0a:	4293      	cmp	r3, r2
 8000f0c:	d00d      	beq.n	8000f2a <HAL_GPIO_Init+0x212>
 8000f0e:	687b      	ldr	r3, [r7, #4]
 8000f10:	4a4c      	ldr	r2, [pc, #304]	; (8001044 <HAL_GPIO_Init+0x32c>)
 8000f12:	4293      	cmp	r3, r2
 8000f14:	d007      	beq.n	8000f26 <HAL_GPIO_Init+0x20e>
 8000f16:	687b      	ldr	r3, [r7, #4]
 8000f18:	4a4b      	ldr	r2, [pc, #300]	; (8001048 <HAL_GPIO_Init+0x330>)
 8000f1a:	4293      	cmp	r3, r2
 8000f1c:	d101      	bne.n	8000f22 <HAL_GPIO_Init+0x20a>
 8000f1e:	2307      	movs	r3, #7
 8000f20:	e00e      	b.n	8000f40 <HAL_GPIO_Init+0x228>
 8000f22:	2308      	movs	r3, #8
 8000f24:	e00c      	b.n	8000f40 <HAL_GPIO_Init+0x228>
 8000f26:	2306      	movs	r3, #6
 8000f28:	e00a      	b.n	8000f40 <HAL_GPIO_Init+0x228>
 8000f2a:	2305      	movs	r3, #5
 8000f2c:	e008      	b.n	8000f40 <HAL_GPIO_Init+0x228>
 8000f2e:	2304      	movs	r3, #4
 8000f30:	e006      	b.n	8000f40 <HAL_GPIO_Init+0x228>
 8000f32:	2303      	movs	r3, #3
 8000f34:	e004      	b.n	8000f40 <HAL_GPIO_Init+0x228>
 8000f36:	2302      	movs	r3, #2
 8000f38:	e002      	b.n	8000f40 <HAL_GPIO_Init+0x228>
 8000f3a:	2301      	movs	r3, #1
 8000f3c:	e000      	b.n	8000f40 <HAL_GPIO_Init+0x228>
 8000f3e:	2300      	movs	r3, #0
 8000f40:	69fa      	ldr	r2, [r7, #28]
 8000f42:	f002 0203 	and.w	r2, r2, #3
 8000f46:	0092      	lsls	r2, r2, #2
 8000f48:	4093      	lsls	r3, r2
 8000f4a:	69ba      	ldr	r2, [r7, #24]
 8000f4c:	4313      	orrs	r3, r2
 8000f4e:	61bb      	str	r3, [r7, #24]
        SYSCFG->EXTICR[position >> 2U] = temp;
 8000f50:	4935      	ldr	r1, [pc, #212]	; (8001028 <HAL_GPIO_Init+0x310>)
 8000f52:	69fb      	ldr	r3, [r7, #28]
 8000f54:	089b      	lsrs	r3, r3, #2
 8000f56:	3302      	adds	r3, #2
 8000f58:	69ba      	ldr	r2, [r7, #24]
 8000f5a:	f841 2023 	str.w	r2, [r1, r3, lsl #2]

        /* Clear EXTI line configuration */
        temp = EXTI->IMR;
 8000f5e:	4b3b      	ldr	r3, [pc, #236]	; (800104c <HAL_GPIO_Init+0x334>)
 8000f60:	681b      	ldr	r3, [r3, #0]
 8000f62:	61bb      	str	r3, [r7, #24]
        temp &= ~((uint32_t)iocurrent);
 8000f64:	693b      	ldr	r3, [r7, #16]
 8000f66:	43db      	mvns	r3, r3
 8000f68:	69ba      	ldr	r2, [r7, #24]
 8000f6a:	4013      	ands	r3, r2
 8000f6c:	61bb      	str	r3, [r7, #24]
        if((GPIO_Init->Mode & EXTI_IT) != 0x00U)
 8000f6e:	683b      	ldr	r3, [r7, #0]
 8000f70:	685b      	ldr	r3, [r3, #4]
 8000f72:	f403 3380 	and.w	r3, r3, #65536	; 0x10000
 8000f76:	2b00      	cmp	r3, #0
 8000f78:	d003      	beq.n	8000f82 <HAL_GPIO_Init+0x26a>
        {
          temp |= iocurrent;
 8000f7a:	69ba      	ldr	r2, [r7, #24]
 8000f7c:	693b      	ldr	r3, [r7, #16]
 8000f7e:	4313      	orrs	r3, r2
 8000f80:	61bb      	str	r3, [r7, #24]
        }
        EXTI->IMR = temp;
 8000f82:	4a32      	ldr	r2, [pc, #200]	; (800104c <HAL_GPIO_Init+0x334>)
 8000f84:	69bb      	ldr	r3, [r7, #24]
 8000f86:	6013      	str	r3, [r2, #0]

        temp = EXTI->EMR;
 8000f88:	4b30      	ldr	r3, [pc, #192]	; (800104c <HAL_GPIO_Init+0x334>)
 8000f8a:	685b      	ldr	r3, [r3, #4]
 8000f8c:	61bb      	str	r3, [r7, #24]
        temp &= ~((uint32_t)iocurrent);
 8000f8e:	693b      	ldr	r3, [r7, #16]
 8000f90:	43db      	mvns	r3, r3
 8000f92:	69ba      	ldr	r2, [r7, #24]
 8000f94:	4013      	ands	r3, r2
 8000f96:	61bb      	str	r3, [r7, #24]
        if((GPIO_Init->Mode & EXTI_EVT) != 0x00U)
 8000f98:	683b      	ldr	r3, [r7, #0]
 8000f9a:	685b      	ldr	r3, [r3, #4]
 8000f9c:	f403 3300 	and.w	r3, r3, #131072	; 0x20000
 8000fa0:	2b00      	cmp	r3, #0
 8000fa2:	d003      	beq.n	8000fac <HAL_GPIO_Init+0x294>
        {
          temp |= iocurrent;
 8000fa4:	69ba      	ldr	r2, [r7, #24]
 8000fa6:	693b      	ldr	r3, [r7, #16]
 8000fa8:	4313      	orrs	r3, r2
 8000faa:	61bb      	str	r3, [r7, #24]
        }
        EXTI->EMR = temp;
 8000fac:	4a27      	ldr	r2, [pc, #156]	; (800104c <HAL_GPIO_Init+0x334>)
 8000fae:	69bb      	ldr	r3, [r7, #24]
 8000fb0:	6053      	str	r3, [r2, #4]

        /* Clear Rising Falling edge configuration */
        temp = EXTI->RTSR;
 8000fb2:	4b26      	ldr	r3, [pc, #152]	; (800104c <HAL_GPIO_Init+0x334>)
 8000fb4:	689b      	ldr	r3, [r3, #8]
 8000fb6:	61bb      	str	r3, [r7, #24]
        temp &= ~((uint32_t)iocurrent);
 8000fb8:	693b      	ldr	r3, [r7, #16]
 8000fba:	43db      	mvns	r3, r3
 8000fbc:	69ba      	ldr	r2, [r7, #24]
 8000fbe:	4013      	ands	r3, r2
 8000fc0:	61bb      	str	r3, [r7, #24]
        if((GPIO_Init->Mode & TRIGGER_RISING) != 0x00U)
 8000fc2:	683b      	ldr	r3, [r7, #0]
 8000fc4:	685b      	ldr	r3, [r3, #4]
 8000fc6:	f403 1380 	and.w	r3, r3, #1048576	; 0x100000
 8000fca:	2b00      	cmp	r3, #0
 8000fcc:	d003      	beq.n	8000fd6 <HAL_GPIO_Init+0x2be>
        {
          temp |= iocurrent;
 8000fce:	69ba      	ldr	r2, [r7, #24]
 8000fd0:	693b      	ldr	r3, [r7, #16]
 8000fd2:	4313      	orrs	r3, r2
 8000fd4:	61bb      	str	r3, [r7, #24]
        }
        EXTI->RTSR = temp;
 8000fd6:	4a1d      	ldr	r2, [pc, #116]	; (800104c <HAL_GPIO_Init+0x334>)
 8000fd8:	69bb      	ldr	r3, [r7, #24]
 8000fda:	6093      	str	r3, [r2, #8]

        temp = EXTI->FTSR;
 8000fdc:	4b1b      	ldr	r3, [pc, #108]	; (800104c <HAL_GPIO_Init+0x334>)
 8000fde:	68db      	ldr	r3, [r3, #12]
 8000fe0:	61bb      	str	r3, [r7, #24]
        temp &= ~((uint32_t)iocurrent);
 8000fe2:	693b      	ldr	r3, [r7, #16]
 8000fe4:	43db      	mvns	r3, r3
 8000fe6:	69ba      	ldr	r2, [r7, #24]
 8000fe8:	4013      	ands	r3, r2
 8000fea:	61bb      	str	r3, [r7, #24]
        if((GPIO_Init->Mode & TRIGGER_FALLING) != 0x00U)
 8000fec:	683b      	ldr	r3, [r7, #0]
 8000fee:	685b      	ldr	r3, [r3, #4]
 8000ff0:	f403 1300 	and.w	r3, r3, #2097152	; 0x200000
 8000ff4:	2b00      	cmp	r3, #0
 8000ff6:	d003      	beq.n	8001000 <HAL_GPIO_Init+0x2e8>
        {
          temp |= iocurrent;
 8000ff8:	69ba      	ldr	r2, [r7, #24]
 8000ffa:	693b      	ldr	r3, [r7, #16]
 8000ffc:	4313      	orrs	r3, r2
 8000ffe:	61bb      	str	r3, [r7, #24]
        }
        EXTI->FTSR = temp;
 8001000:	4a12      	ldr	r2, [pc, #72]	; (800104c <HAL_GPIO_Init+0x334>)
 8001002:	69bb      	ldr	r3, [r7, #24]
 8001004:	60d3      	str	r3, [r2, #12]
  for(position = 0U; position < GPIO_NUMBER; position++)
 8001006:	69fb      	ldr	r3, [r7, #28]
 8001008:	3301      	adds	r3, #1
 800100a:	61fb      	str	r3, [r7, #28]
 800100c:	69fb      	ldr	r3, [r7, #28]
 800100e:	2b0f      	cmp	r3, #15
 8001010:	f67f ae90 	bls.w	8000d34 <HAL_GPIO_Init+0x1c>
      }
    }
  }
}
 8001014:	bf00      	nop
 8001016:	bf00      	nop
 8001018:	3724      	adds	r7, #36	; 0x24
 800101a:	46bd      	mov	sp, r7
 800101c:	f85d 7b04 	ldr.w	r7, [sp], #4
 8001020:	4770      	bx	lr
 8001022:	bf00      	nop
 8001024:	40023800 	.word	0x40023800
 8001028:	40013800 	.word	0x40013800
 800102c:	40020000 	.word	0x40020000
 8001030:	40020400 	.word	0x40020400
 8001034:	40020800 	.word	0x40020800
 8001038:	40020c00 	.word	0x40020c00
 800103c:	40021000 	.word	0x40021000
 8001040:	40021400 	.word	0x40021400
 8001044:	40021800 	.word	0x40021800
 8001048:	40021c00 	.word	0x40021c00
 800104c:	40013c00 	.word	0x40013c00

08001050 <HAL_GPIO_WritePin>:
  *            @arg GPIO_PIN_RESET: to clear the port pin
  *            @arg GPIO_PIN_SET: to set the port pin
  * @retval None
  */
void HAL_GPIO_WritePin(GPIO_TypeDef* GPIOx, uint16_t GPIO_Pin, GPIO_PinState PinState)
{
 8001050:	b480      	push	{r7}
 8001052:	b083      	sub	sp, #12
 8001054:	af00      	add	r7, sp, #0
 8001056:	6078      	str	r0, [r7, #4]
 8001058:	460b      	mov	r3, r1
 800105a:	807b      	strh	r3, [r7, #2]
 800105c:	4613      	mov	r3, r2
 800105e:	707b      	strb	r3, [r7, #1]
  /* Check the parameters */
  assert_param(IS_GPIO_PIN(GPIO_Pin));
  assert_param(IS_GPIO_PIN_ACTION(PinState));

  if(PinState != GPIO_PIN_RESET)
 8001060:	787b      	ldrb	r3, [r7, #1]
 8001062:	2b00      	cmp	r3, #0
 8001064:	d003      	beq.n	800106e <HAL_GPIO_WritePin+0x1e>
  {
    GPIOx->BSRR = GPIO_Pin;
 8001066:	887a      	ldrh	r2, [r7, #2]
 8001068:	687b      	ldr	r3, [r7, #4]
 800106a:	619a      	str	r2, [r3, #24]
  }
  else
  {
    GPIOx->BSRR = (uint32_t)GPIO_Pin << 16U;
  }
}
 800106c:	e003      	b.n	8001076 <HAL_GPIO_WritePin+0x26>
    GPIOx->BSRR = (uint32_t)GPIO_Pin << 16U;
 800106e:	887b      	ldrh	r3, [r7, #2]
 8001070:	041a      	lsls	r2, r3, #16
 8001072:	687b      	ldr	r3, [r7, #4]
 8001074:	619a      	str	r2, [r3, #24]
}
 8001076:	bf00      	nop
 8001078:	370c      	adds	r7, #12
 800107a:	46bd      	mov	sp, r7
 800107c:	f85d 7b04 	ldr.w	r7, [sp], #4
 8001080:	4770      	bx	lr

08001082 <HAL_GPIO_TogglePin>:
  *                      x can be (A..I) to select the GPIO peripheral for STM32F40XX and STM32F427X devices.
  * @param  GPIO_Pin Specifies the pins to be toggled.
  * @retval None
  */
void HAL_GPIO_TogglePin(GPIO_TypeDef* GPIOx, uint16_t GPIO_Pin)
{
 8001082:	b480      	push	{r7}
 8001084:	b085      	sub	sp, #20
 8001086:	af00      	add	r7, sp, #0
 8001088:	6078      	str	r0, [r7, #4]
 800108a:	460b      	mov	r3, r1
 800108c:	807b      	strh	r3, [r7, #2]

  /* Check the parameters */
  assert_param(IS_GPIO_PIN(GPIO_Pin));

  /* get current Ouput Data Register value */
  odr = GPIOx->ODR;
 800108e:	687b      	ldr	r3, [r7, #4]
 8001090:	695b      	ldr	r3, [r3, #20]
 8001092:	60fb      	str	r3, [r7, #12]

  /* Set selected pins that were at low level, and reset ones that were high */
  GPIOx->BSRR = ((odr & GPIO_Pin) << GPIO_NUMBER) | (~odr & GPIO_Pin);
 8001094:	887a      	ldrh	r2, [r7, #2]
 8001096:	68fb      	ldr	r3, [r7, #12]
 8001098:	4013      	ands	r3, r2
 800109a:	041a      	lsls	r2, r3, #16
 800109c:	68fb      	ldr	r3, [r7, #12]
 800109e:	43d9      	mvns	r1, r3
 80010a0:	887b      	ldrh	r3, [r7, #2]
 80010a2:	400b      	ands	r3, r1
 80010a4:	431a      	orrs	r2, r3
 80010a6:	687b      	ldr	r3, [r7, #4]
 80010a8:	619a      	str	r2, [r3, #24]
}
 80010aa:	bf00      	nop
 80010ac:	3714      	adds	r7, #20
 80010ae:	46bd      	mov	sp, r7
 80010b0:	f85d 7b04 	ldr.w	r7, [sp], #4
 80010b4:	4770      	bx	lr
	...

080010b8 <HAL_RCC_OscConfig>:
  *         supported by this API. User should request a transition to HSE Off
  *         first and then HSE On or HSE Bypass.
  * @retval HAL status
  */
__weak HAL_StatusTypeDef HAL_RCC_OscConfig(RCC_OscInitTypeDef  *RCC_OscInitStruct)
{
 80010b8:	b580      	push	{r7, lr}
 80010ba:	b086      	sub	sp, #24
 80010bc:	af00      	add	r7, sp, #0
 80010be:	6078      	str	r0, [r7, #4]
  uint32_t tickstart, pll_config;

  /* Check Null pointer */
  if(RCC_OscInitStruct == NULL)
 80010c0:	687b      	ldr	r3, [r7, #4]
 80010c2:	2b00      	cmp	r3, #0
 80010c4:	d101      	bne.n	80010ca <HAL_RCC_OscConfig+0x12>
  {
    return HAL_ERROR;
 80010c6:	2301      	movs	r3, #1
 80010c8:	e264      	b.n	8001594 <HAL_RCC_OscConfig+0x4dc>
  }

  /* Check the parameters */
  assert_param(IS_RCC_OSCILLATORTYPE(RCC_OscInitStruct->OscillatorType));
  /*------------------------------- HSE Configuration ------------------------*/
  if(((RCC_OscInitStruct->OscillatorType) & RCC_OSCILLATORTYPE_HSE) == RCC_OSCILLATORTYPE_HSE)
 80010ca:	687b      	ldr	r3, [r7, #4]
 80010cc:	681b      	ldr	r3, [r3, #0]
 80010ce:	f003 0301 	and.w	r3, r3, #1
 80010d2:	2b00      	cmp	r3, #0
 80010d4:	d075      	beq.n	80011c2 <HAL_RCC_OscConfig+0x10a>
  {
    /* Check the parameters */
    assert_param(IS_RCC_HSE(RCC_OscInitStruct->HSEState));
    /* When the HSE is used as system clock or clock source for PLL in these cases HSE will not disabled */
    if((__HAL_RCC_GET_SYSCLK_SOURCE() == RCC_CFGR_SWS_HSE) ||\
 80010d6:	4ba3      	ldr	r3, [pc, #652]	; (8001364 <HAL_RCC_OscConfig+0x2ac>)
 80010d8:	689b      	ldr	r3, [r3, #8]
 80010da:	f003 030c 	and.w	r3, r3, #12
 80010de:	2b04      	cmp	r3, #4
 80010e0:	d00c      	beq.n	80010fc <HAL_RCC_OscConfig+0x44>
      ((__HAL_RCC_GET_SYSCLK_SOURCE() == RCC_CFGR_SWS_PLL) && ((RCC->PLLCFGR & RCC_PLLCFGR_PLLSRC) == RCC_PLLCFGR_PLLSRC_HSE)))
 80010e2:	4ba0      	ldr	r3, [pc, #640]	; (8001364 <HAL_RCC_OscConfig+0x2ac>)
 80010e4:	689b      	ldr	r3, [r3, #8]
 80010e6:	f003 030c 	and.w	r3, r3, #12
    if((__HAL_RCC_GET_SYSCLK_SOURCE() == RCC_CFGR_SWS_HSE) ||\
 80010ea:	2b08      	cmp	r3, #8
 80010ec:	d112      	bne.n	8001114 <HAL_RCC_OscConfig+0x5c>
      ((__HAL_RCC_GET_SYSCLK_SOURCE() == RCC_CFGR_SWS_PLL) && ((RCC->PLLCFGR & RCC_PLLCFGR_PLLSRC) == RCC_PLLCFGR_PLLSRC_HSE)))
 80010ee:	4b9d      	ldr	r3, [pc, #628]	; (8001364 <HAL_RCC_OscConfig+0x2ac>)
 80010f0:	685b      	ldr	r3, [r3, #4]
 80010f2:	f403 0380 	and.w	r3, r3, #4194304	; 0x400000
 80010f6:	f5b3 0f80 	cmp.w	r3, #4194304	; 0x400000
 80010fa:	d10b      	bne.n	8001114 <HAL_RCC_OscConfig+0x5c>
    {
      if((__HAL_RCC_GET_FLAG(RCC_FLAG_HSERDY) != RESET) && (RCC_OscInitStruct->HSEState == RCC_HSE_OFF))
 80010fc:	4b99      	ldr	r3, [pc, #612]	; (8001364 <HAL_RCC_OscConfig+0x2ac>)
 80010fe:	681b      	ldr	r3, [r3, #0]
 8001100:	f403 3300 	and.w	r3, r3, #131072	; 0x20000
 8001104:	2b00      	cmp	r3, #0
 8001106:	d05b      	beq.n	80011c0 <HAL_RCC_OscConfig+0x108>
 8001108:	687b      	ldr	r3, [r7, #4]
 800110a:	685b      	ldr	r3, [r3, #4]
 800110c:	2b00      	cmp	r3, #0
 800110e:	d157      	bne.n	80011c0 <HAL_RCC_OscConfig+0x108>
      {
        return HAL_ERROR;
 8001110:	2301      	movs	r3, #1
 8001112:	e23f      	b.n	8001594 <HAL_RCC_OscConfig+0x4dc>
      }
    }
    else
    {
      /* Set the new HSE configuration ---------------------------------------*/
      __HAL_RCC_HSE_CONFIG(RCC_OscInitStruct->HSEState);
 8001114:	687b      	ldr	r3, [r7, #4]
 8001116:	685b      	ldr	r3, [r3, #4]
 8001118:	f5b3 3f80 	cmp.w	r3, #65536	; 0x10000
 800111c:	d106      	bne.n	800112c <HAL_RCC_OscConfig+0x74>
 800111e:	4b91      	ldr	r3, [pc, #580]	; (8001364 <HAL_RCC_OscConfig+0x2ac>)
 8001120:	681b      	ldr	r3, [r3, #0]
 8001122:	4a90      	ldr	r2, [pc, #576]	; (8001364 <HAL_RCC_OscConfig+0x2ac>)
 8001124:	f443 3380 	orr.w	r3, r3, #65536	; 0x10000
 8001128:	6013      	str	r3, [r2, #0]
 800112a:	e01d      	b.n	8001168 <HAL_RCC_OscConfig+0xb0>
 800112c:	687b      	ldr	r3, [r7, #4]
 800112e:	685b      	ldr	r3, [r3, #4]
 8001130:	f5b3 2fa0 	cmp.w	r3, #327680	; 0x50000
 8001134:	d10c      	bne.n	8001150 <HAL_RCC_OscConfig+0x98>
 8001136:	4b8b      	ldr	r3, [pc, #556]	; (8001364 <HAL_RCC_OscConfig+0x2ac>)
 8001138:	681b      	ldr	r3, [r3, #0]
 800113a:	4a8a      	ldr	r2, [pc, #552]	; (8001364 <HAL_RCC_OscConfig+0x2ac>)
 800113c:	f443 2380 	orr.w	r3, r3, #262144	; 0x40000
 8001140:	6013      	str	r3, [r2, #0]
 8001142:	4b88      	ldr	r3, [pc, #544]	; (8001364 <HAL_RCC_OscConfig+0x2ac>)
 8001144:	681b      	ldr	r3, [r3, #0]
 8001146:	4a87      	ldr	r2, [pc, #540]	; (8001364 <HAL_RCC_OscConfig+0x2ac>)
 8001148:	f443 3380 	orr.w	r3, r3, #65536	; 0x10000
 800114c:	6013      	str	r3, [r2, #0]
 800114e:	e00b      	b.n	8001168 <HAL_RCC_OscConfig+0xb0>
 8001150:	4b84      	ldr	r3, [pc, #528]	; (8001364 <HAL_RCC_OscConfig+0x2ac>)
 8001152:	681b      	ldr	r3, [r3, #0]
 8001154:	4a83      	ldr	r2, [pc, #524]	; (8001364 <HAL_RCC_OscConfig+0x2ac>)
 8001156:	f423 3380 	bic.w	r3, r3, #65536	; 0x10000
 800115a:	6013      	str	r3, [r2, #0]
 800115c:	4b81      	ldr	r3, [pc, #516]	; (8001364 <HAL_RCC_OscConfig+0x2ac>)
 800115e:	681b      	ldr	r3, [r3, #0]
 8001160:	4a80      	ldr	r2, [pc, #512]	; (8001364 <HAL_RCC_OscConfig+0x2ac>)
 8001162:	f423 2380 	bic.w	r3, r3, #262144	; 0x40000
 8001166:	6013      	str	r3, [r2, #0]

      /* Check the HSE State */
      if((RCC_OscInitStruct->HSEState) != RCC_HSE_OFF)
 8001168:	687b      	ldr	r3, [r7, #4]
 800116a:	685b      	ldr	r3, [r3, #4]
 800116c:	2b00      	cmp	r3, #0
 800116e:	d013      	beq.n	8001198 <HAL_RCC_OscConfig+0xe0>
      {
        /* Get Start Tick */
        tickstart = HAL_GetTick();
 8001170:	f7ff fce4 	bl	8000b3c <HAL_GetTick>
 8001174:	6138      	str	r0, [r7, #16]

        /* Wait till HSE is ready */
        while(__HAL_RCC_GET_FLAG(RCC_FLAG_HSERDY) == RESET)
 8001176:	e008      	b.n	800118a <HAL_RCC_OscConfig+0xd2>
        {
          if((HAL_GetTick() - tickstart ) > HSE_TIMEOUT_VALUE)
 8001178:	f7ff fce0 	bl	8000b3c <HAL_GetTick>
 800117c:	4602      	mov	r2, r0
 800117e:	693b      	ldr	r3, [r7, #16]
 8001180:	1ad3      	subs	r3, r2, r3
 8001182:	2b64      	cmp	r3, #100	; 0x64
 8001184:	d901      	bls.n	800118a <HAL_RCC_OscConfig+0xd2>
          {
            return HAL_TIMEOUT;
 8001186:	2303      	movs	r3, #3
 8001188:	e204      	b.n	8001594 <HAL_RCC_OscConfig+0x4dc>
        while(__HAL_RCC_GET_FLAG(RCC_FLAG_HSERDY) == RESET)
 800118a:	4b76      	ldr	r3, [pc, #472]	; (8001364 <HAL_RCC_OscConfig+0x2ac>)
 800118c:	681b      	ldr	r3, [r3, #0]
 800118e:	f403 3300 	and.w	r3, r3, #131072	; 0x20000
 8001192:	2b00      	cmp	r3, #0
 8001194:	d0f0      	beq.n	8001178 <HAL_RCC_OscConfig+0xc0>
 8001196:	e014      	b.n	80011c2 <HAL_RCC_OscConfig+0x10a>
        }
      }
      else
      {
        /* Get Start Tick */
        tickstart = HAL_GetTick();
 8001198:	f7ff fcd0 	bl	8000b3c <HAL_GetTick>
 800119c:	6138      	str	r0, [r7, #16]

        /* Wait till HSE is bypassed or disabled */
        while(__HAL_RCC_GET_FLAG(RCC_FLAG_HSERDY) != RESET)
 800119e:	e008      	b.n	80011b2 <HAL_RCC_OscConfig+0xfa>
        {
          if((HAL_GetTick() - tickstart ) > HSE_TIMEOUT_VALUE)
 80011a0:	f7ff fccc 	bl	8000b3c <HAL_GetTick>
 80011a4:	4602      	mov	r2, r0
 80011a6:	693b      	ldr	r3, [r7, #16]
 80011a8:	1ad3      	subs	r3, r2, r3
 80011aa:	2b64      	cmp	r3, #100	; 0x64
 80011ac:	d901      	bls.n	80011b2 <HAL_RCC_OscConfig+0xfa>
          {
            return HAL_TIMEOUT;
 80011ae:	2303      	movs	r3, #3
 80011b0:	e1f0      	b.n	8001594 <HAL_RCC_OscConfig+0x4dc>
        while(__HAL_RCC_GET_FLAG(RCC_FLAG_HSERDY) != RESET)
 80011b2:	4b6c      	ldr	r3, [pc, #432]	; (8001364 <HAL_RCC_OscConfig+0x2ac>)
 80011b4:	681b      	ldr	r3, [r3, #0]
 80011b6:	f403 3300 	and.w	r3, r3, #131072	; 0x20000
 80011ba:	2b00      	cmp	r3, #0
 80011bc:	d1f0      	bne.n	80011a0 <HAL_RCC_OscConfig+0xe8>
 80011be:	e000      	b.n	80011c2 <HAL_RCC_OscConfig+0x10a>
      if((__HAL_RCC_GET_FLAG(RCC_FLAG_HSERDY) != RESET) && (RCC_OscInitStruct->HSEState == RCC_HSE_OFF))
 80011c0:	bf00      	nop
        }
      }
    }
  }
  /*----------------------------- HSI Configuration --------------------------*/
  if(((RCC_OscInitStruct->OscillatorType) & RCC_OSCILLATORTYPE_HSI) == RCC_OSCILLATORTYPE_HSI)
 80011c2:	687b      	ldr	r3, [r7, #4]
 80011c4:	681b      	ldr	r3, [r3, #0]
 80011c6:	f003 0302 	and.w	r3, r3, #2
 80011ca:	2b00      	cmp	r3, #0
 80011cc:	d063      	beq.n	8001296 <HAL_RCC_OscConfig+0x1de>
    /* Check the parameters */
    assert_param(IS_RCC_HSI(RCC_OscInitStruct->HSIState));
    assert_param(IS_RCC_CALIBRATION_VALUE(RCC_OscInitStruct->HSICalibrationValue));

    /* Check if HSI is used as system clock or as PLL source when PLL is selected as system clock */
    if((__HAL_RCC_GET_SYSCLK_SOURCE() == RCC_CFGR_SWS_HSI) ||\
 80011ce:	4b65      	ldr	r3, [pc, #404]	; (8001364 <HAL_RCC_OscConfig+0x2ac>)
 80011d0:	689b      	ldr	r3, [r3, #8]
 80011d2:	f003 030c 	and.w	r3, r3, #12
 80011d6:	2b00      	cmp	r3, #0
 80011d8:	d00b      	beq.n	80011f2 <HAL_RCC_OscConfig+0x13a>
      ((__HAL_RCC_GET_SYSCLK_SOURCE() == RCC_CFGR_SWS_PLL) && ((RCC->PLLCFGR & RCC_PLLCFGR_PLLSRC) == RCC_PLLCFGR_PLLSRC_HSI)))
 80011da:	4b62      	ldr	r3, [pc, #392]	; (8001364 <HAL_RCC_OscConfig+0x2ac>)
 80011dc:	689b      	ldr	r3, [r3, #8]
 80011de:	f003 030c 	and.w	r3, r3, #12
    if((__HAL_RCC_GET_SYSCLK_SOURCE() == RCC_CFGR_SWS_HSI) ||\
 80011e2:	2b08      	cmp	r3, #8
 80011e4:	d11c      	bne.n	8001220 <HAL_RCC_OscConfig+0x168>
      ((__HAL_RCC_GET_SYSCLK_SOURCE() == RCC_CFGR_SWS_PLL) && ((RCC->PLLCFGR & RCC_PLLCFGR_PLLSRC) == RCC_PLLCFGR_PLLSRC_HSI)))
 80011e6:	4b5f      	ldr	r3, [pc, #380]	; (8001364 <HAL_RCC_OscConfig+0x2ac>)
 80011e8:	685b      	ldr	r3, [r3, #4]
 80011ea:	f403 0380 	and.w	r3, r3, #4194304	; 0x400000
 80011ee:	2b00      	cmp	r3, #0
 80011f0:	d116      	bne.n	8001220 <HAL_RCC_OscConfig+0x168>
    {
      /* When HSI is used as system clock it will not disabled */
      if((__HAL_RCC_GET_FLAG(RCC_FLAG_HSIRDY) != RESET) && (RCC_OscInitStruct->HSIState != RCC_HSI_ON))
 80011f2:	4b5c      	ldr	r3, [pc, #368]	; (8001364 <HAL_RCC_OscConfig+0x2ac>)
 80011f4:	681b      	ldr	r3, [r3, #0]
 80011f6:	f003 0302 	and.w	r3, r3, #2
 80011fa:	2b00      	cmp	r3, #0
 80011fc:	d005      	beq.n	800120a <HAL_RCC_OscConfig+0x152>
 80011fe:	687b      	ldr	r3, [r7, #4]
 8001200:	68db      	ldr	r3, [r3, #12]
 8001202:	2b01      	cmp	r3, #1
 8001204:	d001      	beq.n	800120a <HAL_RCC_OscConfig+0x152>
      {
        return HAL_ERROR;
 8001206:	2301      	movs	r3, #1
 8001208:	e1c4      	b.n	8001594 <HAL_RCC_OscConfig+0x4dc>
      }
      /* Otherwise, just the calibration is allowed */
      else
      {
        /* Adjusts the Internal High Speed oscillator (HSI) calibration value.*/
        __HAL_RCC_HSI_CALIBRATIONVALUE_ADJUST(RCC_OscInitStruct->HSICalibrationValue);
 800120a:	4b56      	ldr	r3, [pc, #344]	; (8001364 <HAL_RCC_OscConfig+0x2ac>)
 800120c:	681b      	ldr	r3, [r3, #0]
 800120e:	f023 02f8 	bic.w	r2, r3, #248	; 0xf8
 8001212:	687b      	ldr	r3, [r7, #4]
 8001214:	691b      	ldr	r3, [r3, #16]
 8001216:	00db      	lsls	r3, r3, #3
 8001218:	4952      	ldr	r1, [pc, #328]	; (8001364 <HAL_RCC_OscConfig+0x2ac>)
 800121a:	4313      	orrs	r3, r2
 800121c:	600b      	str	r3, [r1, #0]
      if((__HAL_RCC_GET_FLAG(RCC_FLAG_HSIRDY) != RESET) && (RCC_OscInitStruct->HSIState != RCC_HSI_ON))
 800121e:	e03a      	b.n	8001296 <HAL_RCC_OscConfig+0x1de>
      }
    }
    else
    {
      /* Check the HSI State */
      if((RCC_OscInitStruct->HSIState)!= RCC_HSI_OFF)
 8001220:	687b      	ldr	r3, [r7, #4]
 8001222:	68db      	ldr	r3, [r3, #12]
 8001224:	2b00      	cmp	r3, #0
 8001226:	d020      	beq.n	800126a <HAL_RCC_OscConfig+0x1b2>
      {
        /* Enable the Internal High Speed oscillator (HSI). */
        __HAL_RCC_HSI_ENABLE();
 8001228:	4b4f      	ldr	r3, [pc, #316]	; (8001368 <HAL_RCC_OscConfig+0x2b0>)
 800122a:	2201      	movs	r2, #1
 800122c:	601a      	str	r2, [r3, #0]

        /* Get Start Tick*/
        tickstart = HAL_GetTick();
 800122e:	f7ff fc85 	bl	8000b3c <HAL_GetTick>
 8001232:	6138      	str	r0, [r7, #16]

        /* Wait till HSI is ready */
        while(__HAL_RCC_GET_FLAG(RCC_FLAG_HSIRDY) == RESET)
 8001234:	e008      	b.n	8001248 <HAL_RCC_OscConfig+0x190>
        {
          if((HAL_GetTick() - tickstart ) > HSI_TIMEOUT_VALUE)
 8001236:	f7ff fc81 	bl	8000b3c <HAL_GetTick>
 800123a:	4602      	mov	r2, r0
 800123c:	693b      	ldr	r3, [r7, #16]
 800123e:	1ad3      	subs	r3, r2, r3
 8001240:	2b02      	cmp	r3, #2
 8001242:	d901      	bls.n	8001248 <HAL_RCC_OscConfig+0x190>
          {
            return HAL_TIMEOUT;
 8001244:	2303      	movs	r3, #3
 8001246:	e1a5      	b.n	8001594 <HAL_RCC_OscConfig+0x4dc>
        while(__HAL_RCC_GET_FLAG(RCC_FLAG_HSIRDY) == RESET)
 8001248:	4b46      	ldr	r3, [pc, #280]	; (8001364 <HAL_RCC_OscConfig+0x2ac>)
 800124a:	681b      	ldr	r3, [r3, #0]
 800124c:	f003 0302 	and.w	r3, r3, #2
 8001250:	2b00      	cmp	r3, #0
 8001252:	d0f0      	beq.n	8001236 <HAL_RCC_OscConfig+0x17e>
          }
        }

        /* Adjusts the Internal High Speed oscillator (HSI) calibration value. */
        __HAL_RCC_HSI_CALIBRATIONVALUE_ADJUST(RCC_OscInitStruct->HSICalibrationValue);
 8001254:	4b43      	ldr	r3, [pc, #268]	; (8001364 <HAL_RCC_OscConfig+0x2ac>)
 8001256:	681b      	ldr	r3, [r3, #0]
 8001258:	f023 02f8 	bic.w	r2, r3, #248	; 0xf8
 800125c:	687b      	ldr	r3, [r7, #4]
 800125e:	691b      	ldr	r3, [r3, #16]
 8001260:	00db      	lsls	r3, r3, #3
 8001262:	4940      	ldr	r1, [pc, #256]	; (8001364 <HAL_RCC_OscConfig+0x2ac>)
 8001264:	4313      	orrs	r3, r2
 8001266:	600b      	str	r3, [r1, #0]
 8001268:	e015      	b.n	8001296 <HAL_RCC_OscConfig+0x1de>
      }
      else
      {
        /* Disable the Internal High Speed oscillator (HSI). */
        __HAL_RCC_HSI_DISABLE();
 800126a:	4b3f      	ldr	r3, [pc, #252]	; (8001368 <HAL_RCC_OscConfig+0x2b0>)
 800126c:	2200      	movs	r2, #0
 800126e:	601a      	str	r2, [r3, #0]

        /* Get Start Tick*/
        tickstart = HAL_GetTick();
 8001270:	f7ff fc64 	bl	8000b3c <HAL_GetTick>
 8001274:	6138      	str	r0, [r7, #16]

        /* Wait till HSI is ready */
        while(__HAL_RCC_GET_FLAG(RCC_FLAG_HSIRDY) != RESET)
 8001276:	e008      	b.n	800128a <HAL_RCC_OscConfig+0x1d2>
        {
          if((HAL_GetTick() - tickstart ) > HSI_TIMEOUT_VALUE)
 8001278:	f7ff fc60 	bl	8000b3c <HAL_GetTick>
 800127c:	4602      	mov	r2, r0
 800127e:	693b      	ldr	r3, [r7, #16]
 8001280:	1ad3      	subs	r3, r2, r3
 8001282:	2b02      	cmp	r3, #2
 8001284:	d901      	bls.n	800128a <HAL_RCC_OscConfig+0x1d2>
          {
            return HAL_TIMEOUT;
 8001286:	2303      	movs	r3, #3
 8001288:	e184      	b.n	8001594 <HAL_RCC_OscConfig+0x4dc>
        while(__HAL_RCC_GET_FLAG(RCC_FLAG_HSIRDY) != RESET)
 800128a:	4b36      	ldr	r3, [pc, #216]	; (8001364 <HAL_RCC_OscConfig+0x2ac>)
 800128c:	681b      	ldr	r3, [r3, #0]
 800128e:	f003 0302 	and.w	r3, r3, #2
 8001292:	2b00      	cmp	r3, #0
 8001294:	d1f0      	bne.n	8001278 <HAL_RCC_OscConfig+0x1c0>
        }
      }
    }
  }
  /*------------------------------ LSI Configuration -------------------------*/
  if(((RCC_OscInitStruct->OscillatorType) & RCC_OSCILLATORTYPE_LSI) == RCC_OSCILLATORTYPE_LSI)
 8001296:	687b      	ldr	r3, [r7, #4]
 8001298:	681b      	ldr	r3, [r3, #0]
 800129a:	f003 0308 	and.w	r3, r3, #8
 800129e:	2b00      	cmp	r3, #0
 80012a0:	d030      	beq.n	8001304 <HAL_RCC_OscConfig+0x24c>
  {
    /* Check the parameters */
    assert_param(IS_RCC_LSI(RCC_OscInitStruct->LSIState));

    /* Check the LSI State */
    if((RCC_OscInitStruct->LSIState)!= RCC_LSI_OFF)
 80012a2:	687b      	ldr	r3, [r7, #4]
 80012a4:	695b      	ldr	r3, [r3, #20]
 80012a6:	2b00      	cmp	r3, #0
 80012a8:	d016      	beq.n	80012d8 <HAL_RCC_OscConfig+0x220>
    {
      /* Enable the Internal Low Speed oscillator (LSI). */
      __HAL_RCC_LSI_ENABLE();
 80012aa:	4b30      	ldr	r3, [pc, #192]	; (800136c <HAL_RCC_OscConfig+0x2b4>)
 80012ac:	2201      	movs	r2, #1
 80012ae:	601a      	str	r2, [r3, #0]

      /* Get Start Tick*/
      tickstart = HAL_GetTick();
 80012b0:	f7ff fc44 	bl	8000b3c <HAL_GetTick>
 80012b4:	6138      	str	r0, [r7, #16]

      /* Wait till LSI is ready */
      while(__HAL_RCC_GET_FLAG(RCC_FLAG_LSIRDY) == RESET)
 80012b6:	e008      	b.n	80012ca <HAL_RCC_OscConfig+0x212>
      {
        if((HAL_GetTick() - tickstart ) > LSI_TIMEOUT_VALUE)
 80012b8:	f7ff fc40 	bl	8000b3c <HAL_GetTick>
 80012bc:	4602      	mov	r2, r0
 80012be:	693b      	ldr	r3, [r7, #16]
 80012c0:	1ad3      	subs	r3, r2, r3
 80012c2:	2b02      	cmp	r3, #2
 80012c4:	d901      	bls.n	80012ca <HAL_RCC_OscConfig+0x212>
        {
          return HAL_TIMEOUT;
 80012c6:	2303      	movs	r3, #3
 80012c8:	e164      	b.n	8001594 <HAL_RCC_OscConfig+0x4dc>
      while(__HAL_RCC_GET_FLAG(RCC_FLAG_LSIRDY) == RESET)
 80012ca:	4b26      	ldr	r3, [pc, #152]	; (8001364 <HAL_RCC_OscConfig+0x2ac>)
 80012cc:	6f5b      	ldr	r3, [r3, #116]	; 0x74
 80012ce:	f003 0302 	and.w	r3, r3, #2
 80012d2:	2b00      	cmp	r3, #0
 80012d4:	d0f0      	beq.n	80012b8 <HAL_RCC_OscConfig+0x200>
 80012d6:	e015      	b.n	8001304 <HAL_RCC_OscConfig+0x24c>
      }
    }
    else
    {
      /* Disable the Internal Low Speed oscillator (LSI). */
      __HAL_RCC_LSI_DISABLE();
 80012d8:	4b24      	ldr	r3, [pc, #144]	; (800136c <HAL_RCC_OscConfig+0x2b4>)
 80012da:	2200      	movs	r2, #0
 80012dc:	601a      	str	r2, [r3, #0]

      /* Get Start Tick */
      tickstart = HAL_GetTick();
 80012de:	f7ff fc2d 	bl	8000b3c <HAL_GetTick>
 80012e2:	6138      	str	r0, [r7, #16]

      /* Wait till LSI is ready */
      while(__HAL_RCC_GET_FLAG(RCC_FLAG_LSIRDY) != RESET)
 80012e4:	e008      	b.n	80012f8 <HAL_RCC_OscConfig+0x240>
      {
        if((HAL_GetTick() - tickstart ) > LSI_TIMEOUT_VALUE)
 80012e6:	f7ff fc29 	bl	8000b3c <HAL_GetTick>
 80012ea:	4602      	mov	r2, r0
 80012ec:	693b      	ldr	r3, [r7, #16]
 80012ee:	1ad3      	subs	r3, r2, r3
 80012f0:	2b02      	cmp	r3, #2
 80012f2:	d901      	bls.n	80012f8 <HAL_RCC_OscConfig+0x240>
        {
          return HAL_TIMEOUT;
 80012f4:	2303      	movs	r3, #3
 80012f6:	e14d      	b.n	8001594 <HAL_RCC_OscConfig+0x4dc>
      while(__HAL_RCC_GET_FLAG(RCC_FLAG_LSIRDY) != RESET)
 80012f8:	4b1a      	ldr	r3, [pc, #104]	; (8001364 <HAL_RCC_OscConfig+0x2ac>)
 80012fa:	6f5b      	ldr	r3, [r3, #116]	; 0x74
 80012fc:	f003 0302 	and.w	r3, r3, #2
 8001300:	2b00      	cmp	r3, #0
 8001302:	d1f0      	bne.n	80012e6 <HAL_RCC_OscConfig+0x22e>
        }
      }
    }
  }
  /*------------------------------ LSE Configuration -------------------------*/
  if(((RCC_OscInitStruct->OscillatorType) & RCC_OSCILLATORTYPE_LSE) == RCC_OSCILLATORTYPE_LSE)
 8001304:	687b      	ldr	r3, [r7, #4]
 8001306:	681b      	ldr	r3, [r3, #0]
 8001308:	f003 0304 	and.w	r3, r3, #4
 800130c:	2b00      	cmp	r3, #0
 800130e:	f000 80a0 	beq.w	8001452 <HAL_RCC_OscConfig+0x39a>
  {
    FlagStatus       pwrclkchanged = RESET;
 8001312:	2300      	movs	r3, #0
 8001314:	75fb      	strb	r3, [r7, #23]
    /* Check the parameters */
    assert_param(IS_RCC_LSE(RCC_OscInitStruct->LSEState));

    /* Update LSE configuration in Backup Domain control register    */
    /* Requires to enable write access to Backup Domain of necessary */
    if(__HAL_RCC_PWR_IS_CLK_DISABLED())
 8001316:	4b13      	ldr	r3, [pc, #76]	; (8001364 <HAL_RCC_OscConfig+0x2ac>)
 8001318:	6c1b      	ldr	r3, [r3, #64]	; 0x40
 800131a:	f003 5380 	and.w	r3, r3, #268435456	; 0x10000000
 800131e:	2b00      	cmp	r3, #0
 8001320:	d10f      	bne.n	8001342 <HAL_RCC_OscConfig+0x28a>
    {
      __HAL_RCC_PWR_CLK_ENABLE();
 8001322:	2300      	movs	r3, #0
 8001324:	60bb      	str	r3, [r7, #8]
 8001326:	4b0f      	ldr	r3, [pc, #60]	; (8001364 <HAL_RCC_OscConfig+0x2ac>)
 8001328:	6c1b      	ldr	r3, [r3, #64]	; 0x40
 800132a:	4a0e      	ldr	r2, [pc, #56]	; (8001364 <HAL_RCC_OscConfig+0x2ac>)
 800132c:	f043 5380 	orr.w	r3, r3, #268435456	; 0x10000000
 8001330:	6413      	str	r3, [r2, #64]	; 0x40
 8001332:	4b0c      	ldr	r3, [pc, #48]	; (8001364 <HAL_RCC_OscConfig+0x2ac>)
 8001334:	6c1b      	ldr	r3, [r3, #64]	; 0x40
 8001336:	f003 5380 	and.w	r3, r3, #268435456	; 0x10000000
 800133a:	60bb      	str	r3, [r7, #8]
 800133c:	68bb      	ldr	r3, [r7, #8]
      pwrclkchanged = SET;
 800133e:	2301      	movs	r3, #1
 8001340:	75fb      	strb	r3, [r7, #23]
    }

    if(HAL_IS_BIT_CLR(PWR->CR, PWR_CR_DBP))
 8001342:	4b0b      	ldr	r3, [pc, #44]	; (8001370 <HAL_RCC_OscConfig+0x2b8>)
 8001344:	681b      	ldr	r3, [r3, #0]
 8001346:	f403 7380 	and.w	r3, r3, #256	; 0x100
 800134a:	2b00      	cmp	r3, #0
 800134c:	d121      	bne.n	8001392 <HAL_RCC_OscConfig+0x2da>
    {
      /* Enable write access to Backup domain */
      SET_BIT(PWR->CR, PWR_CR_DBP);
 800134e:	4b08      	ldr	r3, [pc, #32]	; (8001370 <HAL_RCC_OscConfig+0x2b8>)
 8001350:	681b      	ldr	r3, [r3, #0]
 8001352:	4a07      	ldr	r2, [pc, #28]	; (8001370 <HAL_RCC_OscConfig+0x2b8>)
 8001354:	f443 7380 	orr.w	r3, r3, #256	; 0x100
 8001358:	6013      	str	r3, [r2, #0]

      /* Wait for Backup domain Write protection disable */
      tickstart = HAL_GetTick();
 800135a:	f7ff fbef 	bl	8000b3c <HAL_GetTick>
 800135e:	6138      	str	r0, [r7, #16]

      while(HAL_IS_BIT_CLR(PWR->CR, PWR_CR_DBP))
 8001360:	e011      	b.n	8001386 <HAL_RCC_OscConfig+0x2ce>
 8001362:	bf00      	nop
 8001364:	40023800 	.word	0x40023800
 8001368:	42470000 	.word	0x42470000
 800136c:	42470e80 	.word	0x42470e80
 8001370:	40007000 	.word	0x40007000
      {
        if((HAL_GetTick() - tickstart) > RCC_DBP_TIMEOUT_VALUE)
 8001374:	f7ff fbe2 	bl	8000b3c <HAL_GetTick>
 8001378:	4602      	mov	r2, r0
 800137a:	693b      	ldr	r3, [r7, #16]
 800137c:	1ad3      	subs	r3, r2, r3
 800137e:	2b02      	cmp	r3, #2
 8001380:	d901      	bls.n	8001386 <HAL_RCC_OscConfig+0x2ce>
        {
          return HAL_TIMEOUT;
 8001382:	2303      	movs	r3, #3
 8001384:	e106      	b.n	8001594 <HAL_RCC_OscConfig+0x4dc>
      while(HAL_IS_BIT_CLR(PWR->CR, PWR_CR_DBP))
 8001386:	4b85      	ldr	r3, [pc, #532]	; (800159c <HAL_RCC_OscConfig+0x4e4>)
 8001388:	681b      	ldr	r3, [r3, #0]
 800138a:	f403 7380 	and.w	r3, r3, #256	; 0x100
 800138e:	2b00      	cmp	r3, #0
 8001390:	d0f0      	beq.n	8001374 <HAL_RCC_OscConfig+0x2bc>
        }
      }
    }

    /* Set the new LSE configuration -----------------------------------------*/
    __HAL_RCC_LSE_CONFIG(RCC_OscInitStruct->LSEState);
 8001392:	687b      	ldr	r3, [r7, #4]
 8001394:	689b      	ldr	r3, [r3, #8]
 8001396:	2b01      	cmp	r3, #1
 8001398:	d106      	bne.n	80013a8 <HAL_RCC_OscConfig+0x2f0>
 800139a:	4b81      	ldr	r3, [pc, #516]	; (80015a0 <HAL_RCC_OscConfig+0x4e8>)
 800139c:	6f1b      	ldr	r3, [r3, #112]	; 0x70
 800139e:	4a80      	ldr	r2, [pc, #512]	; (80015a0 <HAL_RCC_OscConfig+0x4e8>)
 80013a0:	f043 0301 	orr.w	r3, r3, #1
 80013a4:	6713      	str	r3, [r2, #112]	; 0x70
 80013a6:	e01c      	b.n	80013e2 <HAL_RCC_OscConfig+0x32a>
 80013a8:	687b      	ldr	r3, [r7, #4]
 80013aa:	689b      	ldr	r3, [r3, #8]
 80013ac:	2b05      	cmp	r3, #5
 80013ae:	d10c      	bne.n	80013ca <HAL_RCC_OscConfig+0x312>
 80013b0:	4b7b      	ldr	r3, [pc, #492]	; (80015a0 <HAL_RCC_OscConfig+0x4e8>)
 80013b2:	6f1b      	ldr	r3, [r3, #112]	; 0x70
 80013b4:	4a7a      	ldr	r2, [pc, #488]	; (80015a0 <HAL_RCC_OscConfig+0x4e8>)
 80013b6:	f043 0304 	orr.w	r3, r3, #4
 80013ba:	6713      	str	r3, [r2, #112]	; 0x70
 80013bc:	4b78      	ldr	r3, [pc, #480]	; (80015a0 <HAL_RCC_OscConfig+0x4e8>)
 80013be:	6f1b      	ldr	r3, [r3, #112]	; 0x70
 80013c0:	4a77      	ldr	r2, [pc, #476]	; (80015a0 <HAL_RCC_OscConfig+0x4e8>)
 80013c2:	f043 0301 	orr.w	r3, r3, #1
 80013c6:	6713      	str	r3, [r2, #112]	; 0x70
 80013c8:	e00b      	b.n	80013e2 <HAL_RCC_OscConfig+0x32a>
 80013ca:	4b75      	ldr	r3, [pc, #468]	; (80015a0 <HAL_RCC_OscConfig+0x4e8>)
 80013cc:	6f1b      	ldr	r3, [r3, #112]	; 0x70
 80013ce:	4a74      	ldr	r2, [pc, #464]	; (80015a0 <HAL_RCC_OscConfig+0x4e8>)
 80013d0:	f023 0301 	bic.w	r3, r3, #1
 80013d4:	6713      	str	r3, [r2, #112]	; 0x70
 80013d6:	4b72      	ldr	r3, [pc, #456]	; (80015a0 <HAL_RCC_OscConfig+0x4e8>)
 80013d8:	6f1b      	ldr	r3, [r3, #112]	; 0x70
 80013da:	4a71      	ldr	r2, [pc, #452]	; (80015a0 <HAL_RCC_OscConfig+0x4e8>)
 80013dc:	f023 0304 	bic.w	r3, r3, #4
 80013e0:	6713      	str	r3, [r2, #112]	; 0x70
    /* Check the LSE State */
    if((RCC_OscInitStruct->LSEState) != RCC_LSE_OFF)
 80013e2:	687b      	ldr	r3, [r7, #4]
 80013e4:	689b      	ldr	r3, [r3, #8]
 80013e6:	2b00      	cmp	r3, #0
 80013e8:	d015      	beq.n	8001416 <HAL_RCC_OscConfig+0x35e>
    {
      /* Get Start Tick*/
      tickstart = HAL_GetTick();
 80013ea:	f7ff fba7 	bl	8000b3c <HAL_GetTick>
 80013ee:	6138      	str	r0, [r7, #16]

      /* Wait till LSE is ready */
      while(__HAL_RCC_GET_FLAG(RCC_FLAG_LSERDY) == RESET)
 80013f0:	e00a      	b.n	8001408 <HAL_RCC_OscConfig+0x350>
      {
        if((HAL_GetTick() - tickstart ) > RCC_LSE_TIMEOUT_VALUE)
 80013f2:	f7ff fba3 	bl	8000b3c <HAL_GetTick>
 80013f6:	4602      	mov	r2, r0
 80013f8:	693b      	ldr	r3, [r7, #16]
 80013fa:	1ad3      	subs	r3, r2, r3
 80013fc:	f241 3288 	movw	r2, #5000	; 0x1388
 8001400:	4293      	cmp	r3, r2
 8001402:	d901      	bls.n	8001408 <HAL_RCC_OscConfig+0x350>
        {
          return HAL_TIMEOUT;
 8001404:	2303      	movs	r3, #3
 8001406:	e0c5      	b.n	8001594 <HAL_RCC_OscConfig+0x4dc>
      while(__HAL_RCC_GET_FLAG(RCC_FLAG_LSERDY) == RESET)
 8001408:	4b65      	ldr	r3, [pc, #404]	; (80015a0 <HAL_RCC_OscConfig+0x4e8>)
 800140a:	6f1b      	ldr	r3, [r3, #112]	; 0x70
 800140c:	f003 0302 	and.w	r3, r3, #2
 8001410:	2b00      	cmp	r3, #0
 8001412:	d0ee      	beq.n	80013f2 <HAL_RCC_OscConfig+0x33a>
 8001414:	e014      	b.n	8001440 <HAL_RCC_OscConfig+0x388>
      }
    }
    else
    {
      /* Get Start Tick */
      tickstart = HAL_GetTick();
 8001416:	f7ff fb91 	bl	8000b3c <HAL_GetTick>
 800141a:	6138      	str	r0, [r7, #16]

      /* Wait till LSE is ready */
      while(__HAL_RCC_GET_FLAG(RCC_FLAG_LSERDY) != RESET)
 800141c:	e00a      	b.n	8001434 <HAL_RCC_OscConfig+0x37c>
      {
        if((HAL_GetTick() - tickstart ) > RCC_LSE_TIMEOUT_VALUE)
 800141e:	f7ff fb8d 	bl	8000b3c <HAL_GetTick>
 8001422:	4602      	mov	r2, r0
 8001424:	693b      	ldr	r3, [r7, #16]
 8001426:	1ad3      	subs	r3, r2, r3
 8001428:	f241 3288 	movw	r2, #5000	; 0x1388
 800142c:	4293      	cmp	r3, r2
 800142e:	d901      	bls.n	8001434 <HAL_RCC_OscConfig+0x37c>
        {
          return HAL_TIMEOUT;
 8001430:	2303      	movs	r3, #3
 8001432:	e0af      	b.n	8001594 <HAL_RCC_OscConfig+0x4dc>
      while(__HAL_RCC_GET_FLAG(RCC_FLAG_LSERDY) != RESET)
 8001434:	4b5a      	ldr	r3, [pc, #360]	; (80015a0 <HAL_RCC_OscConfig+0x4e8>)
 8001436:	6f1b      	ldr	r3, [r3, #112]	; 0x70
 8001438:	f003 0302 	and.w	r3, r3, #2
 800143c:	2b00      	cmp	r3, #0
 800143e:	d1ee      	bne.n	800141e <HAL_RCC_OscConfig+0x366>
        }
      }
    }

    /* Restore clock configuration if changed */
    if(pwrclkchanged == SET)
 8001440:	7dfb      	ldrb	r3, [r7, #23]
 8001442:	2b01      	cmp	r3, #1
 8001444:	d105      	bne.n	8001452 <HAL_RCC_OscConfig+0x39a>
    {
      __HAL_RCC_PWR_CLK_DISABLE();
 8001446:	4b56      	ldr	r3, [pc, #344]	; (80015a0 <HAL_RCC_OscConfig+0x4e8>)
 8001448:	6c1b      	ldr	r3, [r3, #64]	; 0x40
 800144a:	4a55      	ldr	r2, [pc, #340]	; (80015a0 <HAL_RCC_OscConfig+0x4e8>)
 800144c:	f023 5380 	bic.w	r3, r3, #268435456	; 0x10000000
 8001450:	6413      	str	r3, [r2, #64]	; 0x40
    }
  }
  /*-------------------------------- PLL Configuration -----------------------*/
  /* Check the parameters */
  assert_param(IS_RCC_PLL(RCC_OscInitStruct->PLL.PLLState));
  if ((RCC_OscInitStruct->PLL.PLLState) != RCC_PLL_NONE)
 8001452:	687b      	ldr	r3, [r7, #4]
 8001454:	699b      	ldr	r3, [r3, #24]
 8001456:	2b00      	cmp	r3, #0
 8001458:	f000 809b 	beq.w	8001592 <HAL_RCC_OscConfig+0x4da>
  {
    /* Check if the PLL is used as system clock or not */
    if(__HAL_RCC_GET_SYSCLK_SOURCE() != RCC_CFGR_SWS_PLL)
 800145c:	4b50      	ldr	r3, [pc, #320]	; (80015a0 <HAL_RCC_OscConfig+0x4e8>)
 800145e:	689b      	ldr	r3, [r3, #8]
 8001460:	f003 030c 	and.w	r3, r3, #12
 8001464:	2b08      	cmp	r3, #8
 8001466:	d05c      	beq.n	8001522 <HAL_RCC_OscConfig+0x46a>
    {
      if((RCC_OscInitStruct->PLL.PLLState) == RCC_PLL_ON)
 8001468:	687b      	ldr	r3, [r7, #4]
 800146a:	699b      	ldr	r3, [r3, #24]
 800146c:	2b02      	cmp	r3, #2
 800146e:	d141      	bne.n	80014f4 <HAL_RCC_OscConfig+0x43c>
        assert_param(IS_RCC_PLLN_VALUE(RCC_OscInitStruct->PLL.PLLN));
        assert_param(IS_RCC_PLLP_VALUE(RCC_OscInitStruct->PLL.PLLP));
        assert_param(IS_RCC_PLLQ_VALUE(RCC_OscInitStruct->PLL.PLLQ));

        /* Disable the main PLL. */
        __HAL_RCC_PLL_DISABLE();
 8001470:	4b4c      	ldr	r3, [pc, #304]	; (80015a4 <HAL_RCC_OscConfig+0x4ec>)
 8001472:	2200      	movs	r2, #0
 8001474:	601a      	str	r2, [r3, #0]

        /* Get Start Tick */
        tickstart = HAL_GetTick();
 8001476:	f7ff fb61 	bl	8000b3c <HAL_GetTick>
 800147a:	6138      	str	r0, [r7, #16]

        /* Wait till PLL is ready */
        while(__HAL_RCC_GET_FLAG(RCC_FLAG_PLLRDY) != RESET)
 800147c:	e008      	b.n	8001490 <HAL_RCC_OscConfig+0x3d8>
        {
          if((HAL_GetTick() - tickstart ) > PLL_TIMEOUT_VALUE)
 800147e:	f7ff fb5d 	bl	8000b3c <HAL_GetTick>
 8001482:	4602      	mov	r2, r0
 8001484:	693b      	ldr	r3, [r7, #16]
 8001486:	1ad3      	subs	r3, r2, r3
 8001488:	2b02      	cmp	r3, #2
 800148a:	d901      	bls.n	8001490 <HAL_RCC_OscConfig+0x3d8>
          {
            return HAL_TIMEOUT;
 800148c:	2303      	movs	r3, #3
 800148e:	e081      	b.n	8001594 <HAL_RCC_OscConfig+0x4dc>
        while(__HAL_RCC_GET_FLAG(RCC_FLAG_PLLRDY) != RESET)
 8001490:	4b43      	ldr	r3, [pc, #268]	; (80015a0 <HAL_RCC_OscConfig+0x4e8>)
 8001492:	681b      	ldr	r3, [r3, #0]
 8001494:	f003 7300 	and.w	r3, r3, #33554432	; 0x2000000
 8001498:	2b00      	cmp	r3, #0
 800149a:	d1f0      	bne.n	800147e <HAL_RCC_OscConfig+0x3c6>
          }
        }

        /* Configure the main PLL clock source, multiplication and division factors. */
        WRITE_REG(RCC->PLLCFGR, (RCC_OscInitStruct->PLL.PLLSource                                            | \
 800149c:	687b      	ldr	r3, [r7, #4]
 800149e:	69da      	ldr	r2, [r3, #28]
 80014a0:	687b      	ldr	r3, [r7, #4]
 80014a2:	6a1b      	ldr	r3, [r3, #32]
 80014a4:	431a      	orrs	r2, r3
 80014a6:	687b      	ldr	r3, [r7, #4]
 80014a8:	6a5b      	ldr	r3, [r3, #36]	; 0x24
 80014aa:	019b      	lsls	r3, r3, #6
 80014ac:	431a      	orrs	r2, r3
 80014ae:	687b      	ldr	r3, [r7, #4]
 80014b0:	6a9b      	ldr	r3, [r3, #40]	; 0x28
 80014b2:	085b      	lsrs	r3, r3, #1
 80014b4:	3b01      	subs	r3, #1
 80014b6:	041b      	lsls	r3, r3, #16
 80014b8:	431a      	orrs	r2, r3
 80014ba:	687b      	ldr	r3, [r7, #4]
 80014bc:	6adb      	ldr	r3, [r3, #44]	; 0x2c
 80014be:	061b      	lsls	r3, r3, #24
 80014c0:	4937      	ldr	r1, [pc, #220]	; (80015a0 <HAL_RCC_OscConfig+0x4e8>)
 80014c2:	4313      	orrs	r3, r2
 80014c4:	604b      	str	r3, [r1, #4]
                                 RCC_OscInitStruct->PLL.PLLM                                                 | \
                                 (RCC_OscInitStruct->PLL.PLLN << RCC_PLLCFGR_PLLN_Pos)             | \
                                 (((RCC_OscInitStruct->PLL.PLLP >> 1U) - 1U) << RCC_PLLCFGR_PLLP_Pos) | \
                                 (RCC_OscInitStruct->PLL.PLLQ << RCC_PLLCFGR_PLLQ_Pos)));
        /* Enable the main PLL. */
        __HAL_RCC_PLL_ENABLE();
 80014c6:	4b37      	ldr	r3, [pc, #220]	; (80015a4 <HAL_RCC_OscConfig+0x4ec>)
 80014c8:	2201      	movs	r2, #1
 80014ca:	601a      	str	r2, [r3, #0]

        /* Get Start Tick */
        tickstart = HAL_GetTick();
 80014cc:	f7ff fb36 	bl	8000b3c <HAL_GetTick>
 80014d0:	6138      	str	r0, [r7, #16]

        /* Wait till PLL is ready */
        while(__HAL_RCC_GET_FLAG(RCC_FLAG_PLLRDY) == RESET)
 80014d2:	e008      	b.n	80014e6 <HAL_RCC_OscConfig+0x42e>
        {
          if((HAL_GetTick() - tickstart ) > PLL_TIMEOUT_VALUE)
 80014d4:	f7ff fb32 	bl	8000b3c <HAL_GetTick>
 80014d8:	4602      	mov	r2, r0
 80014da:	693b      	ldr	r3, [r7, #16]
 80014dc:	1ad3      	subs	r3, r2, r3
 80014de:	2b02      	cmp	r3, #2
 80014e0:	d901      	bls.n	80014e6 <HAL_RCC_OscConfig+0x42e>
          {
            return HAL_TIMEOUT;
 80014e2:	2303      	movs	r3, #3
 80014e4:	e056      	b.n	8001594 <HAL_RCC_OscConfig+0x4dc>
        while(__HAL_RCC_GET_FLAG(RCC_FLAG_PLLRDY) == RESET)
 80014e6:	4b2e      	ldr	r3, [pc, #184]	; (80015a0 <HAL_RCC_OscConfig+0x4e8>)
 80014e8:	681b      	ldr	r3, [r3, #0]
 80014ea:	f003 7300 	and.w	r3, r3, #33554432	; 0x2000000
 80014ee:	2b00      	cmp	r3, #0
 80014f0:	d0f0      	beq.n	80014d4 <HAL_RCC_OscConfig+0x41c>
 80014f2:	e04e      	b.n	8001592 <HAL_RCC_OscConfig+0x4da>
        }
      }
      else
      {
        /* Disable the main PLL. */
        __HAL_RCC_PLL_DISABLE();
 80014f4:	4b2b      	ldr	r3, [pc, #172]	; (80015a4 <HAL_RCC_OscConfig+0x4ec>)
 80014f6:	2200      	movs	r2, #0
 80014f8:	601a      	str	r2, [r3, #0]

        /* Get Start Tick */
        tickstart = HAL_GetTick();
 80014fa:	f7ff fb1f 	bl	8000b3c <HAL_GetTick>
 80014fe:	6138      	str	r0, [r7, #16]

        /* Wait till PLL is ready */
        while(__HAL_RCC_GET_FLAG(RCC_FLAG_PLLRDY) != RESET)
 8001500:	e008      	b.n	8001514 <HAL_RCC_OscConfig+0x45c>
        {
          if((HAL_GetTick() - tickstart ) > PLL_TIMEOUT_VALUE)
 8001502:	f7ff fb1b 	bl	8000b3c <HAL_GetTick>
 8001506:	4602      	mov	r2, r0
 8001508:	693b      	ldr	r3, [r7, #16]
 800150a:	1ad3      	subs	r3, r2, r3
 800150c:	2b02      	cmp	r3, #2
 800150e:	d901      	bls.n	8001514 <HAL_RCC_OscConfig+0x45c>
          {
            return HAL_TIMEOUT;
 8001510:	2303      	movs	r3, #3
 8001512:	e03f      	b.n	8001594 <HAL_RCC_OscConfig+0x4dc>
        while(__HAL_RCC_GET_FLAG(RCC_FLAG_PLLRDY) != RESET)
 8001514:	4b22      	ldr	r3, [pc, #136]	; (80015a0 <HAL_RCC_OscConfig+0x4e8>)
 8001516:	681b      	ldr	r3, [r3, #0]
 8001518:	f003 7300 	and.w	r3, r3, #33554432	; 0x2000000
 800151c:	2b00      	cmp	r3, #0
 800151e:	d1f0      	bne.n	8001502 <HAL_RCC_OscConfig+0x44a>
 8001520:	e037      	b.n	8001592 <HAL_RCC_OscConfig+0x4da>
      }
    }
    else
    {
      /* Check if there is a request to disable the PLL used as System clock source */
      if((RCC_OscInitStruct->PLL.PLLState) == RCC_PLL_OFF)
 8001522:	687b      	ldr	r3, [r7, #4]
 8001524:	699b      	ldr	r3, [r3, #24]
 8001526:	2b01      	cmp	r3, #1
 8001528:	d101      	bne.n	800152e <HAL_RCC_OscConfig+0x476>
      {
        return HAL_ERROR;
 800152a:	2301      	movs	r3, #1
 800152c:	e032      	b.n	8001594 <HAL_RCC_OscConfig+0x4dc>
      }
      else
      {
        /* Do not return HAL_ERROR if request repeats the current configuration */
        pll_config = RCC->PLLCFGR;
 800152e:	4b1c      	ldr	r3, [pc, #112]	; (80015a0 <HAL_RCC_OscConfig+0x4e8>)
 8001530:	685b      	ldr	r3, [r3, #4]
 8001532:	60fb      	str	r3, [r7, #12]
            (READ_BIT(pll_config, RCC_PLLCFGR_PLLN) != (RCC_OscInitStruct->PLL.PLLN) << RCC_PLLCFGR_PLLN_Pos) ||
            (READ_BIT(pll_config, RCC_PLLCFGR_PLLP) != (((RCC_OscInitStruct->PLL.PLLP >> 1U) - 1U)) << RCC_PLLCFGR_PLLP_Pos) ||
            (READ_BIT(pll_config, RCC_PLLCFGR_PLLQ) != (RCC_OscInitStruct->PLL.PLLQ << RCC_PLLCFGR_PLLQ_Pos)) ||
            (READ_BIT(pll_config, RCC_PLLCFGR_PLLR) != (RCC_OscInitStruct->PLL.PLLR << RCC_PLLCFGR_PLLR_Pos)))
#else
        if (((RCC_OscInitStruct->PLL.PLLState) == RCC_PLL_OFF) ||
 8001534:	687b      	ldr	r3, [r7, #4]
 8001536:	699b      	ldr	r3, [r3, #24]
 8001538:	2b01      	cmp	r3, #1
 800153a:	d028      	beq.n	800158e <HAL_RCC_OscConfig+0x4d6>
            (READ_BIT(pll_config, RCC_PLLCFGR_PLLSRC) != RCC_OscInitStruct->PLL.PLLSource) ||
 800153c:	68fb      	ldr	r3, [r7, #12]
 800153e:	f403 0280 	and.w	r2, r3, #4194304	; 0x400000
 8001542:	687b      	ldr	r3, [r7, #4]
 8001544:	69db      	ldr	r3, [r3, #28]
        if (((RCC_OscInitStruct->PLL.PLLState) == RCC_PLL_OFF) ||
 8001546:	429a      	cmp	r2, r3
 8001548:	d121      	bne.n	800158e <HAL_RCC_OscConfig+0x4d6>
            (READ_BIT(pll_config, RCC_PLLCFGR_PLLM) != (RCC_OscInitStruct->PLL.PLLM) << RCC_PLLCFGR_PLLM_Pos) ||
 800154a:	68fb      	ldr	r3, [r7, #12]
 800154c:	f003 023f 	and.w	r2, r3, #63	; 0x3f
 8001550:	687b      	ldr	r3, [r7, #4]
 8001552:	6a1b      	ldr	r3, [r3, #32]
            (READ_BIT(pll_config, RCC_PLLCFGR_PLLSRC) != RCC_OscInitStruct->PLL.PLLSource) ||
 8001554:	429a      	cmp	r2, r3
 8001556:	d11a      	bne.n	800158e <HAL_RCC_OscConfig+0x4d6>
            (READ_BIT(pll_config, RCC_PLLCFGR_PLLN) != (RCC_OscInitStruct->PLL.PLLN) << RCC_PLLCFGR_PLLN_Pos) ||
 8001558:	68fa      	ldr	r2, [r7, #12]
 800155a:	f647 73c0 	movw	r3, #32704	; 0x7fc0
 800155e:	4013      	ands	r3, r2
 8001560:	687a      	ldr	r2, [r7, #4]
 8001562:	6a52      	ldr	r2, [r2, #36]	; 0x24
 8001564:	0192      	lsls	r2, r2, #6
            (READ_BIT(pll_config, RCC_PLLCFGR_PLLM) != (RCC_OscInitStruct->PLL.PLLM) << RCC_PLLCFGR_PLLM_Pos) ||
 8001566:	4293      	cmp	r3, r2
 8001568:	d111      	bne.n	800158e <HAL_RCC_OscConfig+0x4d6>
            (READ_BIT(pll_config, RCC_PLLCFGR_PLLP) != (((RCC_OscInitStruct->PLL.PLLP >> 1U) - 1U)) << RCC_PLLCFGR_PLLP_Pos) ||
 800156a:	68fb      	ldr	r3, [r7, #12]
 800156c:	f403 3240 	and.w	r2, r3, #196608	; 0x30000
 8001570:	687b      	ldr	r3, [r7, #4]
 8001572:	6a9b      	ldr	r3, [r3, #40]	; 0x28
 8001574:	085b      	lsrs	r3, r3, #1
 8001576:	3b01      	subs	r3, #1
 8001578:	041b      	lsls	r3, r3, #16
            (READ_BIT(pll_config, RCC_PLLCFGR_PLLN) != (RCC_OscInitStruct->PLL.PLLN) << RCC_PLLCFGR_PLLN_Pos) ||
 800157a:	429a      	cmp	r2, r3
 800157c:	d107      	bne.n	800158e <HAL_RCC_OscConfig+0x4d6>
            (READ_BIT(pll_config, RCC_PLLCFGR_PLLQ) != (RCC_OscInitStruct->PLL.PLLQ << RCC_PLLCFGR_PLLQ_Pos)))
 800157e:	68fb      	ldr	r3, [r7, #12]
 8001580:	f003 6270 	and.w	r2, r3, #251658240	; 0xf000000
 8001584:	687b      	ldr	r3, [r7, #4]
 8001586:	6adb      	ldr	r3, [r3, #44]	; 0x2c
 8001588:	061b      	lsls	r3, r3, #24
            (READ_BIT(pll_config, RCC_PLLCFGR_PLLP) != (((RCC_OscInitStruct->PLL.PLLP >> 1U) - 1U)) << RCC_PLLCFGR_PLLP_Pos) ||
 800158a:	429a      	cmp	r2, r3
 800158c:	d001      	beq.n	8001592 <HAL_RCC_OscConfig+0x4da>
#endif
        {
          return HAL_ERROR;
 800158e:	2301      	movs	r3, #1
 8001590:	e000      	b.n	8001594 <HAL_RCC_OscConfig+0x4dc>
        }
      }
    }
  }
  return HAL_OK;
 8001592:	2300      	movs	r3, #0
}
 8001594:	4618      	mov	r0, r3
 8001596:	3718      	adds	r7, #24
 8001598:	46bd      	mov	sp, r7
 800159a:	bd80      	pop	{r7, pc}
 800159c:	40007000 	.word	0x40007000
 80015a0:	40023800 	.word	0x40023800
 80015a4:	42470060 	.word	0x42470060

080015a8 <HAL_RCC_ClockConfig>:
  *         HPRE[3:0] bits to ensure that HCLK not exceed the maximum allowed frequency
  *         (for more details refer to section above "Initialization/de-initialization functions")
  * @retval None
  */
HAL_StatusTypeDef HAL_RCC_ClockConfig(RCC_ClkInitTypeDef  *RCC_ClkInitStruct, uint32_t FLatency)
{
 80015a8:	b580      	push	{r7, lr}
 80015aa:	b084      	sub	sp, #16
 80015ac:	af00      	add	r7, sp, #0
 80015ae:	6078      	str	r0, [r7, #4]
 80015b0:	6039      	str	r1, [r7, #0]
  uint32_t tickstart;

  /* Check Null pointer */
  if(RCC_ClkInitStruct == NULL)
 80015b2:	687b      	ldr	r3, [r7, #4]
 80015b4:	2b00      	cmp	r3, #0
 80015b6:	d101      	bne.n	80015bc <HAL_RCC_ClockConfig+0x14>
  {
    return HAL_ERROR;
 80015b8:	2301      	movs	r3, #1
 80015ba:	e0cc      	b.n	8001756 <HAL_RCC_ClockConfig+0x1ae>
  /* To correctly read data from FLASH memory, the number of wait states (LATENCY)
    must be correctly programmed according to the frequency of the CPU clock
    (HCLK) and the supply voltage of the device. */

  /* Increasing the number of wait states because of higher CPU frequency */
  if(FLatency > __HAL_FLASH_GET_LATENCY())
 80015bc:	4b68      	ldr	r3, [pc, #416]	; (8001760 <HAL_RCC_ClockConfig+0x1b8>)
 80015be:	681b      	ldr	r3, [r3, #0]
 80015c0:	f003 0307 	and.w	r3, r3, #7
 80015c4:	683a      	ldr	r2, [r7, #0]
 80015c6:	429a      	cmp	r2, r3
 80015c8:	d90c      	bls.n	80015e4 <HAL_RCC_ClockConfig+0x3c>
  {
    /* Program the new number of wait states to the LATENCY bits in the FLASH_ACR register */
    __HAL_FLASH_SET_LATENCY(FLatency);
 80015ca:	4b65      	ldr	r3, [pc, #404]	; (8001760 <HAL_RCC_ClockConfig+0x1b8>)
 80015cc:	683a      	ldr	r2, [r7, #0]
 80015ce:	b2d2      	uxtb	r2, r2
 80015d0:	701a      	strb	r2, [r3, #0]

    /* Check that the new number of wait states is taken into account to access the Flash
    memory by reading the FLASH_ACR register */
    if(__HAL_FLASH_GET_LATENCY() != FLatency)
 80015d2:	4b63      	ldr	r3, [pc, #396]	; (8001760 <HAL_RCC_ClockConfig+0x1b8>)
 80015d4:	681b      	ldr	r3, [r3, #0]
 80015d6:	f003 0307 	and.w	r3, r3, #7
 80015da:	683a      	ldr	r2, [r7, #0]
 80015dc:	429a      	cmp	r2, r3
 80015de:	d001      	beq.n	80015e4 <HAL_RCC_ClockConfig+0x3c>
    {
      return HAL_ERROR;
 80015e0:	2301      	movs	r3, #1
 80015e2:	e0b8      	b.n	8001756 <HAL_RCC_ClockConfig+0x1ae>
    }
  }

  /*-------------------------- HCLK Configuration --------------------------*/
  if(((RCC_ClkInitStruct->ClockType) & RCC_CLOCKTYPE_HCLK) == RCC_CLOCKTYPE_HCLK)
 80015e4:	687b      	ldr	r3, [r7, #4]
 80015e6:	681b      	ldr	r3, [r3, #0]
 80015e8:	f003 0302 	and.w	r3, r3, #2
 80015ec:	2b00      	cmp	r3, #0
 80015ee:	d020      	beq.n	8001632 <HAL_RCC_ClockConfig+0x8a>
  {
    /* Set the highest APBx dividers in order to ensure that we do not go through
       a non-spec phase whatever we decrease or increase HCLK. */
    if(((RCC_ClkInitStruct->ClockType) & RCC_CLOCKTYPE_PCLK1) == RCC_CLOCKTYPE_PCLK1)
 80015f0:	687b      	ldr	r3, [r7, #4]
 80015f2:	681b      	ldr	r3, [r3, #0]
 80015f4:	f003 0304 	and.w	r3, r3, #4
 80015f8:	2b00      	cmp	r3, #0
 80015fa:	d005      	beq.n	8001608 <HAL_RCC_ClockConfig+0x60>
    {
      MODIFY_REG(RCC->CFGR, RCC_CFGR_PPRE1, RCC_HCLK_DIV16);
 80015fc:	4b59      	ldr	r3, [pc, #356]	; (8001764 <HAL_RCC_ClockConfig+0x1bc>)
 80015fe:	689b      	ldr	r3, [r3, #8]
 8001600:	4a58      	ldr	r2, [pc, #352]	; (8001764 <HAL_RCC_ClockConfig+0x1bc>)
 8001602:	f443 53e0 	orr.w	r3, r3, #7168	; 0x1c00
 8001606:	6093      	str	r3, [r2, #8]
    }

    if(((RCC_ClkInitStruct->ClockType) & RCC_CLOCKTYPE_PCLK2) == RCC_CLOCKTYPE_PCLK2)
 8001608:	687b      	ldr	r3, [r7, #4]
 800160a:	681b      	ldr	r3, [r3, #0]
 800160c:	f003 0308 	and.w	r3, r3, #8
 8001610:	2b00      	cmp	r3, #0
 8001612:	d005      	beq.n	8001620 <HAL_RCC_ClockConfig+0x78>
    {
      MODIFY_REG(RCC->CFGR, RCC_CFGR_PPRE2, (RCC_HCLK_DIV16 << 3));
 8001614:	4b53      	ldr	r3, [pc, #332]	; (8001764 <HAL_RCC_ClockConfig+0x1bc>)
 8001616:	689b      	ldr	r3, [r3, #8]
 8001618:	4a52      	ldr	r2, [pc, #328]	; (8001764 <HAL_RCC_ClockConfig+0x1bc>)
 800161a:	f443 4360 	orr.w	r3, r3, #57344	; 0xe000
 800161e:	6093      	str	r3, [r2, #8]
    }

    assert_param(IS_RCC_HCLK(RCC_ClkInitStruct->AHBCLKDivider));
    MODIFY_REG(RCC->CFGR, RCC_CFGR_HPRE, RCC_ClkInitStruct->AHBCLKDivider);
 8001620:	4b50      	ldr	r3, [pc, #320]	; (8001764 <HAL_RCC_ClockConfig+0x1bc>)
 8001622:	689b      	ldr	r3, [r3, #8]
 8001624:	f023 02f0 	bic.w	r2, r3, #240	; 0xf0
 8001628:	687b      	ldr	r3, [r7, #4]
 800162a:	689b      	ldr	r3, [r3, #8]
 800162c:	494d      	ldr	r1, [pc, #308]	; (8001764 <HAL_RCC_ClockConfig+0x1bc>)
 800162e:	4313      	orrs	r3, r2
 8001630:	608b      	str	r3, [r1, #8]
  }

  /*------------------------- SYSCLK Configuration ---------------------------*/
  if(((RCC_ClkInitStruct->ClockType) & RCC_CLOCKTYPE_SYSCLK) == RCC_CLOCKTYPE_SYSCLK)
 8001632:	687b      	ldr	r3, [r7, #4]
 8001634:	681b      	ldr	r3, [r3, #0]
 8001636:	f003 0301 	and.w	r3, r3, #1
 800163a:	2b00      	cmp	r3, #0
 800163c:	d044      	beq.n	80016c8 <HAL_RCC_ClockConfig+0x120>
  {
    assert_param(IS_RCC_SYSCLKSOURCE(RCC_ClkInitStruct->SYSCLKSource));

    /* HSE is selected as System Clock Source */
    if(RCC_ClkInitStruct->SYSCLKSource == RCC_SYSCLKSOURCE_HSE)
 800163e:	687b      	ldr	r3, [r7, #4]
 8001640:	685b      	ldr	r3, [r3, #4]
 8001642:	2b01      	cmp	r3, #1
 8001644:	d107      	bne.n	8001656 <HAL_RCC_ClockConfig+0xae>
    {
      /* Check the HSE ready flag */
      if(__HAL_RCC_GET_FLAG(RCC_FLAG_HSERDY) == RESET)
 8001646:	4b47      	ldr	r3, [pc, #284]	; (8001764 <HAL_RCC_ClockConfig+0x1bc>)
 8001648:	681b      	ldr	r3, [r3, #0]
 800164a:	f403 3300 	and.w	r3, r3, #131072	; 0x20000
 800164e:	2b00      	cmp	r3, #0
 8001650:	d119      	bne.n	8001686 <HAL_RCC_ClockConfig+0xde>
      {
        return HAL_ERROR;
 8001652:	2301      	movs	r3, #1
 8001654:	e07f      	b.n	8001756 <HAL_RCC_ClockConfig+0x1ae>
      }
    }
    /* PLL is selected as System Clock Source */
    else if((RCC_ClkInitStruct->SYSCLKSource == RCC_SYSCLKSOURCE_PLLCLK)   ||
 8001656:	687b      	ldr	r3, [r7, #4]
 8001658:	685b      	ldr	r3, [r3, #4]
 800165a:	2b02      	cmp	r3, #2
 800165c:	d003      	beq.n	8001666 <HAL_RCC_ClockConfig+0xbe>
            (RCC_ClkInitStruct->SYSCLKSource == RCC_SYSCLKSOURCE_PLLRCLK))
 800165e:	687b      	ldr	r3, [r7, #4]
 8001660:	685b      	ldr	r3, [r3, #4]
    else if((RCC_ClkInitStruct->SYSCLKSource == RCC_SYSCLKSOURCE_PLLCLK)   ||
 8001662:	2b03      	cmp	r3, #3
 8001664:	d107      	bne.n	8001676 <HAL_RCC_ClockConfig+0xce>
    {
      /* Check the PLL ready flag */
      if(__HAL_RCC_GET_FLAG(RCC_FLAG_PLLRDY) == RESET)
 8001666:	4b3f      	ldr	r3, [pc, #252]	; (8001764 <HAL_RCC_ClockConfig+0x1bc>)
 8001668:	681b      	ldr	r3, [r3, #0]
 800166a:	f003 7300 	and.w	r3, r3, #33554432	; 0x2000000
 800166e:	2b00      	cmp	r3, #0
 8001670:	d109      	bne.n	8001686 <HAL_RCC_ClockConfig+0xde>
      {
        return HAL_ERROR;
 8001672:	2301      	movs	r3, #1
 8001674:	e06f      	b.n	8001756 <HAL_RCC_ClockConfig+0x1ae>
    }
    /* HSI is selected as System Clock Source */
    else
    {
      /* Check the HSI ready flag */
      if(__HAL_RCC_GET_FLAG(RCC_FLAG_HSIRDY) == RESET)
 8001676:	4b3b      	ldr	r3, [pc, #236]	; (8001764 <HAL_RCC_ClockConfig+0x1bc>)
 8001678:	681b      	ldr	r3, [r3, #0]
 800167a:	f003 0302 	and.w	r3, r3, #2
 800167e:	2b00      	cmp	r3, #0
 8001680:	d101      	bne.n	8001686 <HAL_RCC_ClockConfig+0xde>
      {
        return HAL_ERROR;
 8001682:	2301      	movs	r3, #1
 8001684:	e067      	b.n	8001756 <HAL_RCC_ClockConfig+0x1ae>
      }
    }

    __HAL_RCC_SYSCLK_CONFIG(RCC_ClkInitStruct->SYSCLKSource);
 8001686:	4b37      	ldr	r3, [pc, #220]	; (8001764 <HAL_RCC_ClockConfig+0x1bc>)
 8001688:	689b      	ldr	r3, [r3, #8]
 800168a:	f023 0203 	bic.w	r2, r3, #3
 800168e:	687b      	ldr	r3, [r7, #4]
 8001690:	685b      	ldr	r3, [r3, #4]
 8001692:	4934      	ldr	r1, [pc, #208]	; (8001764 <HAL_RCC_ClockConfig+0x1bc>)
 8001694:	4313      	orrs	r3, r2
 8001696:	608b      	str	r3, [r1, #8]

    /* Get Start Tick */
    tickstart = HAL_GetTick();
 8001698:	f7ff fa50 	bl	8000b3c <HAL_GetTick>
 800169c:	60f8      	str	r0, [r7, #12]

    while (__HAL_RCC_GET_SYSCLK_SOURCE() != (RCC_ClkInitStruct->SYSCLKSource << RCC_CFGR_SWS_Pos))
 800169e:	e00a      	b.n	80016b6 <HAL_RCC_ClockConfig+0x10e>
    {
      if ((HAL_GetTick() - tickstart) > CLOCKSWITCH_TIMEOUT_VALUE)
 80016a0:	f7ff fa4c 	bl	8000b3c <HAL_GetTick>
 80016a4:	4602      	mov	r2, r0
 80016a6:	68fb      	ldr	r3, [r7, #12]
 80016a8:	1ad3      	subs	r3, r2, r3
 80016aa:	f241 3288 	movw	r2, #5000	; 0x1388
 80016ae:	4293      	cmp	r3, r2
 80016b0:	d901      	bls.n	80016b6 <HAL_RCC_ClockConfig+0x10e>
      {
        return HAL_TIMEOUT;
 80016b2:	2303      	movs	r3, #3
 80016b4:	e04f      	b.n	8001756 <HAL_RCC_ClockConfig+0x1ae>
    while (__HAL_RCC_GET_SYSCLK_SOURCE() != (RCC_ClkInitStruct->SYSCLKSource << RCC_CFGR_SWS_Pos))
 80016b6:	4b2b      	ldr	r3, [pc, #172]	; (8001764 <HAL_RCC_ClockConfig+0x1bc>)
 80016b8:	689b      	ldr	r3, [r3, #8]
 80016ba:	f003 020c 	and.w	r2, r3, #12
 80016be:	687b      	ldr	r3, [r7, #4]
 80016c0:	685b      	ldr	r3, [r3, #4]
 80016c2:	009b      	lsls	r3, r3, #2
 80016c4:	429a      	cmp	r2, r3
 80016c6:	d1eb      	bne.n	80016a0 <HAL_RCC_ClockConfig+0xf8>
      }
    }
  }

  /* Decreasing the number of wait states because of lower CPU frequency */
  if(FLatency < __HAL_FLASH_GET_LATENCY())
 80016c8:	4b25      	ldr	r3, [pc, #148]	; (8001760 <HAL_RCC_ClockConfig+0x1b8>)
 80016ca:	681b      	ldr	r3, [r3, #0]
 80016cc:	f003 0307 	and.w	r3, r3, #7
 80016d0:	683a      	ldr	r2, [r7, #0]
 80016d2:	429a      	cmp	r2, r3
 80016d4:	d20c      	bcs.n	80016f0 <HAL_RCC_ClockConfig+0x148>
  {
     /* Program the new number of wait states to the LATENCY bits in the FLASH_ACR register */
    __HAL_FLASH_SET_LATENCY(FLatency);
 80016d6:	4b22      	ldr	r3, [pc, #136]	; (8001760 <HAL_RCC_ClockConfig+0x1b8>)
 80016d8:	683a      	ldr	r2, [r7, #0]
 80016da:	b2d2      	uxtb	r2, r2
 80016dc:	701a      	strb	r2, [r3, #0]

    /* Check that the new number of wait states is taken into account to access the Flash
    memory by reading the FLASH_ACR register */
    if(__HAL_FLASH_GET_LATENCY() != FLatency)
 80016de:	4b20      	ldr	r3, [pc, #128]	; (8001760 <HAL_RCC_ClockConfig+0x1b8>)
 80016e0:	681b      	ldr	r3, [r3, #0]
 80016e2:	f003 0307 	and.w	r3, r3, #7
 80016e6:	683a      	ldr	r2, [r7, #0]
 80016e8:	429a      	cmp	r2, r3
 80016ea:	d001      	beq.n	80016f0 <HAL_RCC_ClockConfig+0x148>
    {
      return HAL_ERROR;
 80016ec:	2301      	movs	r3, #1
 80016ee:	e032      	b.n	8001756 <HAL_RCC_ClockConfig+0x1ae>
    }
  }

  /*-------------------------- PCLK1 Configuration ---------------------------*/
  if(((RCC_ClkInitStruct->ClockType) & RCC_CLOCKTYPE_PCLK1) == RCC_CLOCKTYPE_PCLK1)
 80016f0:	687b      	ldr	r3, [r7, #4]
 80016f2:	681b      	ldr	r3, [r3, #0]
 80016f4:	f003 0304 	and.w	r3, r3, #4
 80016f8:	2b00      	cmp	r3, #0
 80016fa:	d008      	beq.n	800170e <HAL_RCC_ClockConfig+0x166>
  {
    assert_param(IS_RCC_PCLK(RCC_ClkInitStruct->APB1CLKDivider));
    MODIFY_REG(RCC->CFGR, RCC_CFGR_PPRE1, RCC_ClkInitStruct->APB1CLKDivider);
 80016fc:	4b19      	ldr	r3, [pc, #100]	; (8001764 <HAL_RCC_ClockConfig+0x1bc>)
 80016fe:	689b      	ldr	r3, [r3, #8]
 8001700:	f423 52e0 	bic.w	r2, r3, #7168	; 0x1c00
 8001704:	687b      	ldr	r3, [r7, #4]
 8001706:	68db      	ldr	r3, [r3, #12]
 8001708:	4916      	ldr	r1, [pc, #88]	; (8001764 <HAL_RCC_ClockConfig+0x1bc>)
 800170a:	4313      	orrs	r3, r2
 800170c:	608b      	str	r3, [r1, #8]
  }

  /*-------------------------- PCLK2 Configuration ---------------------------*/
  if(((RCC_ClkInitStruct->ClockType) & RCC_CLOCKTYPE_PCLK2) == RCC_CLOCKTYPE_PCLK2)
 800170e:	687b      	ldr	r3, [r7, #4]
 8001710:	681b      	ldr	r3, [r3, #0]
 8001712:	f003 0308 	and.w	r3, r3, #8
 8001716:	2b00      	cmp	r3, #0
 8001718:	d009      	beq.n	800172e <HAL_RCC_ClockConfig+0x186>
  {
    assert_param(IS_RCC_PCLK(RCC_ClkInitStruct->APB2CLKDivider));
    MODIFY_REG(RCC->CFGR, RCC_CFGR_PPRE2, ((RCC_ClkInitStruct->APB2CLKDivider) << 3U));
 800171a:	4b12      	ldr	r3, [pc, #72]	; (8001764 <HAL_RCC_ClockConfig+0x1bc>)
 800171c:	689b      	ldr	r3, [r3, #8]
 800171e:	f423 4260 	bic.w	r2, r3, #57344	; 0xe000
 8001722:	687b      	ldr	r3, [r7, #4]
 8001724:	691b      	ldr	r3, [r3, #16]
 8001726:	00db      	lsls	r3, r3, #3
 8001728:	490e      	ldr	r1, [pc, #56]	; (8001764 <HAL_RCC_ClockConfig+0x1bc>)
 800172a:	4313      	orrs	r3, r2
 800172c:	608b      	str	r3, [r1, #8]
  }

  /* Update the SystemCoreClock global variable */
  SystemCoreClock = HAL_RCC_GetSysClockFreq() >> AHBPrescTable[(RCC->CFGR & RCC_CFGR_HPRE)>> RCC_CFGR_HPRE_Pos];
 800172e:	f000 f821 	bl	8001774 <HAL_RCC_GetSysClockFreq>
 8001732:	4602      	mov	r2, r0
 8001734:	4b0b      	ldr	r3, [pc, #44]	; (8001764 <HAL_RCC_ClockConfig+0x1bc>)
 8001736:	689b      	ldr	r3, [r3, #8]
 8001738:	091b      	lsrs	r3, r3, #4
 800173a:	f003 030f 	and.w	r3, r3, #15
 800173e:	490a      	ldr	r1, [pc, #40]	; (8001768 <HAL_RCC_ClockConfig+0x1c0>)
 8001740:	5ccb      	ldrb	r3, [r1, r3]
 8001742:	fa22 f303 	lsr.w	r3, r2, r3
 8001746:	4a09      	ldr	r2, [pc, #36]	; (800176c <HAL_RCC_ClockConfig+0x1c4>)
 8001748:	6013      	str	r3, [r2, #0]

  /* Configure the source of time base considering new system clocks settings */
  HAL_InitTick (uwTickPrio);
 800174a:	4b09      	ldr	r3, [pc, #36]	; (8001770 <HAL_RCC_ClockConfig+0x1c8>)
 800174c:	681b      	ldr	r3, [r3, #0]
 800174e:	4618      	mov	r0, r3
 8001750:	f7ff f90a 	bl	8000968 <HAL_InitTick>

  return HAL_OK;
 8001754:	2300      	movs	r3, #0
}
 8001756:	4618      	mov	r0, r3
 8001758:	3710      	adds	r7, #16
 800175a:	46bd      	mov	sp, r7
 800175c:	bd80      	pop	{r7, pc}
 800175e:	bf00      	nop
 8001760:	40023c00 	.word	0x40023c00
 8001764:	40023800 	.word	0x40023800
 8001768:	08003c74 	.word	0x08003c74
 800176c:	20000000 	.word	0x20000000
 8001770:	20000004 	.word	0x20000004

08001774 <HAL_RCC_GetSysClockFreq>:
  *
  *
  * @retval SYSCLK frequency
  */
__weak uint32_t HAL_RCC_GetSysClockFreq(void)
{
 8001774:	e92d 43b0 	stmdb	sp!, {r4, r5, r7, r8, r9, lr}
 8001778:	b084      	sub	sp, #16
 800177a:	af00      	add	r7, sp, #0
  uint32_t pllm = 0U, pllvco = 0U, pllp = 0U;
 800177c:	2300      	movs	r3, #0
 800177e:	607b      	str	r3, [r7, #4]
 8001780:	2300      	movs	r3, #0
 8001782:	60fb      	str	r3, [r7, #12]
 8001784:	2300      	movs	r3, #0
 8001786:	603b      	str	r3, [r7, #0]
  uint32_t sysclockfreq = 0U;
 8001788:	2300      	movs	r3, #0
 800178a:	60bb      	str	r3, [r7, #8]

  /* Get SYSCLK source -------------------------------------------------------*/
  switch (RCC->CFGR & RCC_CFGR_SWS)
 800178c:	4b67      	ldr	r3, [pc, #412]	; (800192c <HAL_RCC_GetSysClockFreq+0x1b8>)
 800178e:	689b      	ldr	r3, [r3, #8]
 8001790:	f003 030c 	and.w	r3, r3, #12
 8001794:	2b08      	cmp	r3, #8
 8001796:	d00d      	beq.n	80017b4 <HAL_RCC_GetSysClockFreq+0x40>
 8001798:	2b08      	cmp	r3, #8
 800179a:	f200 80bd 	bhi.w	8001918 <HAL_RCC_GetSysClockFreq+0x1a4>
 800179e:	2b00      	cmp	r3, #0
 80017a0:	d002      	beq.n	80017a8 <HAL_RCC_GetSysClockFreq+0x34>
 80017a2:	2b04      	cmp	r3, #4
 80017a4:	d003      	beq.n	80017ae <HAL_RCC_GetSysClockFreq+0x3a>
 80017a6:	e0b7      	b.n	8001918 <HAL_RCC_GetSysClockFreq+0x1a4>
  {
    case RCC_CFGR_SWS_HSI:  /* HSI used as system clock source */
    {
      sysclockfreq = HSI_VALUE;
 80017a8:	4b61      	ldr	r3, [pc, #388]	; (8001930 <HAL_RCC_GetSysClockFreq+0x1bc>)
 80017aa:	60bb      	str	r3, [r7, #8]
       break;
 80017ac:	e0b7      	b.n	800191e <HAL_RCC_GetSysClockFreq+0x1aa>
    }
    case RCC_CFGR_SWS_HSE:  /* HSE used as system clock  source */
    {
      sysclockfreq = HSE_VALUE;
 80017ae:	4b61      	ldr	r3, [pc, #388]	; (8001934 <HAL_RCC_GetSysClockFreq+0x1c0>)
 80017b0:	60bb      	str	r3, [r7, #8]
      break;
 80017b2:	e0b4      	b.n	800191e <HAL_RCC_GetSysClockFreq+0x1aa>
    }
    case RCC_CFGR_SWS_PLL:  /* PLL used as system clock  source */
    {
      /* PLL_VCO = (HSE_VALUE or HSI_VALUE / PLLM) * PLLN
      SYSCLK = PLL_VCO / PLLP */
      pllm = RCC->PLLCFGR & RCC_PLLCFGR_PLLM;
 80017b4:	4b5d      	ldr	r3, [pc, #372]	; (800192c <HAL_RCC_GetSysClockFreq+0x1b8>)
 80017b6:	685b      	ldr	r3, [r3, #4]
 80017b8:	f003 033f 	and.w	r3, r3, #63	; 0x3f
 80017bc:	607b      	str	r3, [r7, #4]
      if(__HAL_RCC_GET_PLL_OSCSOURCE() != RCC_PLLSOURCE_HSI)
 80017be:	4b5b      	ldr	r3, [pc, #364]	; (800192c <HAL_RCC_GetSysClockFreq+0x1b8>)
 80017c0:	685b      	ldr	r3, [r3, #4]
 80017c2:	f403 0380 	and.w	r3, r3, #4194304	; 0x400000
 80017c6:	2b00      	cmp	r3, #0
 80017c8:	d04d      	beq.n	8001866 <HAL_RCC_GetSysClockFreq+0xf2>
      {
        /* HSE used as PLL clock source */
        pllvco = (uint32_t) ((((uint64_t) HSE_VALUE * ((uint64_t) ((RCC->PLLCFGR & RCC_PLLCFGR_PLLN) >> RCC_PLLCFGR_PLLN_Pos)))) / (uint64_t)pllm);
 80017ca:	4b58      	ldr	r3, [pc, #352]	; (800192c <HAL_RCC_GetSysClockFreq+0x1b8>)
 80017cc:	685b      	ldr	r3, [r3, #4]
 80017ce:	099b      	lsrs	r3, r3, #6
 80017d0:	461a      	mov	r2, r3
 80017d2:	f04f 0300 	mov.w	r3, #0
 80017d6:	f240 10ff 	movw	r0, #511	; 0x1ff
 80017da:	f04f 0100 	mov.w	r1, #0
 80017de:	ea02 0800 	and.w	r8, r2, r0
 80017e2:	ea03 0901 	and.w	r9, r3, r1
 80017e6:	4640      	mov	r0, r8
 80017e8:	4649      	mov	r1, r9
 80017ea:	f04f 0200 	mov.w	r2, #0
 80017ee:	f04f 0300 	mov.w	r3, #0
 80017f2:	014b      	lsls	r3, r1, #5
 80017f4:	ea43 63d0 	orr.w	r3, r3, r0, lsr #27
 80017f8:	0142      	lsls	r2, r0, #5
 80017fa:	4610      	mov	r0, r2
 80017fc:	4619      	mov	r1, r3
 80017fe:	ebb0 0008 	subs.w	r0, r0, r8
 8001802:	eb61 0109 	sbc.w	r1, r1, r9
 8001806:	f04f 0200 	mov.w	r2, #0
 800180a:	f04f 0300 	mov.w	r3, #0
 800180e:	018b      	lsls	r3, r1, #6
 8001810:	ea43 6390 	orr.w	r3, r3, r0, lsr #26
 8001814:	0182      	lsls	r2, r0, #6
 8001816:	1a12      	subs	r2, r2, r0
 8001818:	eb63 0301 	sbc.w	r3, r3, r1
 800181c:	f04f 0000 	mov.w	r0, #0
 8001820:	f04f 0100 	mov.w	r1, #0
 8001824:	00d9      	lsls	r1, r3, #3
 8001826:	ea41 7152 	orr.w	r1, r1, r2, lsr #29
 800182a:	00d0      	lsls	r0, r2, #3
 800182c:	4602      	mov	r2, r0
 800182e:	460b      	mov	r3, r1
 8001830:	eb12 0208 	adds.w	r2, r2, r8
 8001834:	eb43 0309 	adc.w	r3, r3, r9
 8001838:	f04f 0000 	mov.w	r0, #0
 800183c:	f04f 0100 	mov.w	r1, #0
 8001840:	0259      	lsls	r1, r3, #9
 8001842:	ea41 51d2 	orr.w	r1, r1, r2, lsr #23
 8001846:	0250      	lsls	r0, r2, #9
 8001848:	4602      	mov	r2, r0
 800184a:	460b      	mov	r3, r1
 800184c:	4610      	mov	r0, r2
 800184e:	4619      	mov	r1, r3
 8001850:	687b      	ldr	r3, [r7, #4]
 8001852:	461a      	mov	r2, r3
 8001854:	f04f 0300 	mov.w	r3, #0
 8001858:	f7fe fcc2 	bl	80001e0 <__aeabi_uldivmod>
 800185c:	4602      	mov	r2, r0
 800185e:	460b      	mov	r3, r1
 8001860:	4613      	mov	r3, r2
 8001862:	60fb      	str	r3, [r7, #12]
 8001864:	e04a      	b.n	80018fc <HAL_RCC_GetSysClockFreq+0x188>
      }
      else
      {
        /* HSI used as PLL clock source */
        pllvco = (uint32_t) ((((uint64_t) HSI_VALUE * ((uint64_t) ((RCC->PLLCFGR & RCC_PLLCFGR_PLLN) >> RCC_PLLCFGR_PLLN_Pos)))) / (uint64_t)pllm);
 8001866:	4b31      	ldr	r3, [pc, #196]	; (800192c <HAL_RCC_GetSysClockFreq+0x1b8>)
 8001868:	685b      	ldr	r3, [r3, #4]
 800186a:	099b      	lsrs	r3, r3, #6
 800186c:	461a      	mov	r2, r3
 800186e:	f04f 0300 	mov.w	r3, #0
 8001872:	f240 10ff 	movw	r0, #511	; 0x1ff
 8001876:	f04f 0100 	mov.w	r1, #0
 800187a:	ea02 0400 	and.w	r4, r2, r0
 800187e:	ea03 0501 	and.w	r5, r3, r1
 8001882:	4620      	mov	r0, r4
 8001884:	4629      	mov	r1, r5
 8001886:	f04f 0200 	mov.w	r2, #0
 800188a:	f04f 0300 	mov.w	r3, #0
 800188e:	014b      	lsls	r3, r1, #5
 8001890:	ea43 63d0 	orr.w	r3, r3, r0, lsr #27
 8001894:	0142      	lsls	r2, r0, #5
 8001896:	4610      	mov	r0, r2
 8001898:	4619      	mov	r1, r3
 800189a:	1b00      	subs	r0, r0, r4
 800189c:	eb61 0105 	sbc.w	r1, r1, r5
 80018a0:	f04f 0200 	mov.w	r2, #0
 80018a4:	f04f 0300 	mov.w	r3, #0
 80018a8:	018b      	lsls	r3, r1, #6
 80018aa:	ea43 6390 	orr.w	r3, r3, r0, lsr #26
 80018ae:	0182      	lsls	r2, r0, #6
 80018b0:	1a12      	subs	r2, r2, r0
 80018b2:	eb63 0301 	sbc.w	r3, r3, r1
 80018b6:	f04f 0000 	mov.w	r0, #0
 80018ba:	f04f 0100 	mov.w	r1, #0
 80018be:	00d9      	lsls	r1, r3, #3
 80018c0:	ea41 7152 	orr.w	r1, r1, r2, lsr #29
 80018c4:	00d0      	lsls	r0, r2, #3
 80018c6:	4602      	mov	r2, r0
 80018c8:	460b      	mov	r3, r1
 80018ca:	1912      	adds	r2, r2, r4
 80018cc:	eb45 0303 	adc.w	r3, r5, r3
 80018d0:	f04f 0000 	mov.w	r0, #0
 80018d4:	f04f 0100 	mov.w	r1, #0
 80018d8:	0299      	lsls	r1, r3, #10
 80018da:	ea41 5192 	orr.w	r1, r1, r2, lsr #22
 80018de:	0290      	lsls	r0, r2, #10
 80018e0:	4602      	mov	r2, r0
 80018e2:	460b      	mov	r3, r1
 80018e4:	4610      	mov	r0, r2
 80018e6:	4619      	mov	r1, r3
 80018e8:	687b      	ldr	r3, [r7, #4]
 80018ea:	461a      	mov	r2, r3
 80018ec:	f04f 0300 	mov.w	r3, #0
 80018f0:	f7fe fc76 	bl	80001e0 <__aeabi_uldivmod>
 80018f4:	4602      	mov	r2, r0
 80018f6:	460b      	mov	r3, r1
 80018f8:	4613      	mov	r3, r2
 80018fa:	60fb      	str	r3, [r7, #12]
      }
      pllp = ((((RCC->PLLCFGR & RCC_PLLCFGR_PLLP) >> RCC_PLLCFGR_PLLP_Pos) + 1U) *2U);
 80018fc:	4b0b      	ldr	r3, [pc, #44]	; (800192c <HAL_RCC_GetSysClockFreq+0x1b8>)
 80018fe:	685b      	ldr	r3, [r3, #4]
 8001900:	0c1b      	lsrs	r3, r3, #16
 8001902:	f003 0303 	and.w	r3, r3, #3
 8001906:	3301      	adds	r3, #1
 8001908:	005b      	lsls	r3, r3, #1
 800190a:	603b      	str	r3, [r7, #0]

      sysclockfreq = pllvco/pllp;
 800190c:	68fa      	ldr	r2, [r7, #12]
 800190e:	683b      	ldr	r3, [r7, #0]
 8001910:	fbb2 f3f3 	udiv	r3, r2, r3
 8001914:	60bb      	str	r3, [r7, #8]
      break;
 8001916:	e002      	b.n	800191e <HAL_RCC_GetSysClockFreq+0x1aa>
    }
    default:
    {
      sysclockfreq = HSI_VALUE;
 8001918:	4b05      	ldr	r3, [pc, #20]	; (8001930 <HAL_RCC_GetSysClockFreq+0x1bc>)
 800191a:	60bb      	str	r3, [r7, #8]
      break;
 800191c:	bf00      	nop
    }
  }
  return sysclockfreq;
 800191e:	68bb      	ldr	r3, [r7, #8]
}
 8001920:	4618      	mov	r0, r3
 8001922:	3710      	adds	r7, #16
 8001924:	46bd      	mov	sp, r7
 8001926:	e8bd 83b0 	ldmia.w	sp!, {r4, r5, r7, r8, r9, pc}
 800192a:	bf00      	nop
 800192c:	40023800 	.word	0x40023800
 8001930:	00f42400 	.word	0x00f42400
 8001934:	007a1200 	.word	0x007a1200

08001938 <HAL_RCC_GetHCLKFreq>:
  * @note   The SystemCoreClock CMSIS variable is used to store System Clock Frequency
  *         and updated within this function
  * @retval HCLK frequency
  */
uint32_t HAL_RCC_GetHCLKFreq(void)
{
 8001938:	b480      	push	{r7}
 800193a:	af00      	add	r7, sp, #0
  return SystemCoreClock;
 800193c:	4b03      	ldr	r3, [pc, #12]	; (800194c <HAL_RCC_GetHCLKFreq+0x14>)
 800193e:	681b      	ldr	r3, [r3, #0]
}
 8001940:	4618      	mov	r0, r3
 8001942:	46bd      	mov	sp, r7
 8001944:	f85d 7b04 	ldr.w	r7, [sp], #4
 8001948:	4770      	bx	lr
 800194a:	bf00      	nop
 800194c:	20000000 	.word	0x20000000

08001950 <HAL_RCC_GetPCLK1Freq>:
  * @note   Each time PCLK1 changes, this function must be called to update the
  *         right PCLK1 value. Otherwise, any configuration based on this function will be incorrect.
  * @retval PCLK1 frequency
  */
uint32_t HAL_RCC_GetPCLK1Freq(void)
{
 8001950:	b580      	push	{r7, lr}
 8001952:	af00      	add	r7, sp, #0
  /* Get HCLK source and Compute PCLK1 frequency ---------------------------*/
  return (HAL_RCC_GetHCLKFreq() >> APBPrescTable[(RCC->CFGR & RCC_CFGR_PPRE1)>> RCC_CFGR_PPRE1_Pos]);
 8001954:	f7ff fff0 	bl	8001938 <HAL_RCC_GetHCLKFreq>
 8001958:	4602      	mov	r2, r0
 800195a:	4b05      	ldr	r3, [pc, #20]	; (8001970 <HAL_RCC_GetPCLK1Freq+0x20>)
 800195c:	689b      	ldr	r3, [r3, #8]
 800195e:	0a9b      	lsrs	r3, r3, #10
 8001960:	f003 0307 	and.w	r3, r3, #7
 8001964:	4903      	ldr	r1, [pc, #12]	; (8001974 <HAL_RCC_GetPCLK1Freq+0x24>)
 8001966:	5ccb      	ldrb	r3, [r1, r3]
 8001968:	fa22 f303 	lsr.w	r3, r2, r3
}
 800196c:	4618      	mov	r0, r3
 800196e:	bd80      	pop	{r7, pc}
 8001970:	40023800 	.word	0x40023800
 8001974:	08003c84 	.word	0x08003c84

08001978 <HAL_RCC_GetPCLK2Freq>:
  * @note   Each time PCLK2 changes, this function must be called to update the
  *         right PCLK2 value. Otherwise, any configuration based on this function will be incorrect.
  * @retval PCLK2 frequency
  */
uint32_t HAL_RCC_GetPCLK2Freq(void)
{
 8001978:	b580      	push	{r7, lr}
 800197a:	af00      	add	r7, sp, #0
  /* Get HCLK source and Compute PCLK2 frequency ---------------------------*/
  return (HAL_RCC_GetHCLKFreq()>> APBPrescTable[(RCC->CFGR & RCC_CFGR_PPRE2)>> RCC_CFGR_PPRE2_Pos]);
 800197c:	f7ff ffdc 	bl	8001938 <HAL_RCC_GetHCLKFreq>
 8001980:	4602      	mov	r2, r0
 8001982:	4b05      	ldr	r3, [pc, #20]	; (8001998 <HAL_RCC_GetPCLK2Freq+0x20>)
 8001984:	689b      	ldr	r3, [r3, #8]
 8001986:	0b5b      	lsrs	r3, r3, #13
 8001988:	f003 0307 	and.w	r3, r3, #7
 800198c:	4903      	ldr	r1, [pc, #12]	; (800199c <HAL_RCC_GetPCLK2Freq+0x24>)
 800198e:	5ccb      	ldrb	r3, [r1, r3]
 8001990:	fa22 f303 	lsr.w	r3, r2, r3
}
 8001994:	4618      	mov	r0, r3
 8001996:	bd80      	pop	{r7, pc}
 8001998:	40023800 	.word	0x40023800
 800199c:	08003c84 	.word	0x08003c84

080019a0 <HAL_RCC_GetClockConfig>:
  * will be configured.
  * @param  pFLatency Pointer on the Flash Latency.
  * @retval None
  */
void HAL_RCC_GetClockConfig(RCC_ClkInitTypeDef  *RCC_ClkInitStruct, uint32_t *pFLatency)
{
 80019a0:	b480      	push	{r7}
 80019a2:	b083      	sub	sp, #12
 80019a4:	af00      	add	r7, sp, #0
 80019a6:	6078      	str	r0, [r7, #4]
 80019a8:	6039      	str	r1, [r7, #0]
  /* Set all possible values for the Clock type parameter --------------------*/
  RCC_ClkInitStruct->ClockType = RCC_CLOCKTYPE_SYSCLK | RCC_CLOCKTYPE_HCLK | RCC_CLOCKTYPE_PCLK1 | RCC_CLOCKTYPE_PCLK2;
 80019aa:	687b      	ldr	r3, [r7, #4]
 80019ac:	220f      	movs	r2, #15
 80019ae:	601a      	str	r2, [r3, #0]

  /* Get the SYSCLK configuration --------------------------------------------*/
  RCC_ClkInitStruct->SYSCLKSource = (uint32_t)(RCC->CFGR & RCC_CFGR_SW);
 80019b0:	4b12      	ldr	r3, [pc, #72]	; (80019fc <HAL_RCC_GetClockConfig+0x5c>)
 80019b2:	689b      	ldr	r3, [r3, #8]
 80019b4:	f003 0203 	and.w	r2, r3, #3
 80019b8:	687b      	ldr	r3, [r7, #4]
 80019ba:	605a      	str	r2, [r3, #4]

  /* Get the HCLK configuration ----------------------------------------------*/
  RCC_ClkInitStruct->AHBCLKDivider = (uint32_t)(RCC->CFGR & RCC_CFGR_HPRE);
 80019bc:	4b0f      	ldr	r3, [pc, #60]	; (80019fc <HAL_RCC_GetClockConfig+0x5c>)
 80019be:	689b      	ldr	r3, [r3, #8]
 80019c0:	f003 02f0 	and.w	r2, r3, #240	; 0xf0
 80019c4:	687b      	ldr	r3, [r7, #4]
 80019c6:	609a      	str	r2, [r3, #8]

  /* Get the APB1 configuration ----------------------------------------------*/
  RCC_ClkInitStruct->APB1CLKDivider = (uint32_t)(RCC->CFGR & RCC_CFGR_PPRE1);
 80019c8:	4b0c      	ldr	r3, [pc, #48]	; (80019fc <HAL_RCC_GetClockConfig+0x5c>)
 80019ca:	689b      	ldr	r3, [r3, #8]
 80019cc:	f403 52e0 	and.w	r2, r3, #7168	; 0x1c00
 80019d0:	687b      	ldr	r3, [r7, #4]
 80019d2:	60da      	str	r2, [r3, #12]

  /* Get the APB2 configuration ----------------------------------------------*/
  RCC_ClkInitStruct->APB2CLKDivider = (uint32_t)((RCC->CFGR & RCC_CFGR_PPRE2) >> 3U);
 80019d4:	4b09      	ldr	r3, [pc, #36]	; (80019fc <HAL_RCC_GetClockConfig+0x5c>)
 80019d6:	689b      	ldr	r3, [r3, #8]
 80019d8:	08db      	lsrs	r3, r3, #3
 80019da:	f403 52e0 	and.w	r2, r3, #7168	; 0x1c00
 80019de:	687b      	ldr	r3, [r7, #4]
 80019e0:	611a      	str	r2, [r3, #16]

  /* Get the Flash Wait State (Latency) configuration ------------------------*/
  *pFLatency = (uint32_t)(FLASH->ACR & FLASH_ACR_LATENCY);
 80019e2:	4b07      	ldr	r3, [pc, #28]	; (8001a00 <HAL_RCC_GetClockConfig+0x60>)
 80019e4:	681b      	ldr	r3, [r3, #0]
 80019e6:	f003 0207 	and.w	r2, r3, #7
 80019ea:	683b      	ldr	r3, [r7, #0]
 80019ec:	601a      	str	r2, [r3, #0]
}
 80019ee:	bf00      	nop
 80019f0:	370c      	adds	r7, #12
 80019f2:	46bd      	mov	sp, r7
 80019f4:	f85d 7b04 	ldr.w	r7, [sp], #4
 80019f8:	4770      	bx	lr
 80019fa:	bf00      	nop
 80019fc:	40023800 	.word	0x40023800
 8001a00:	40023c00 	.word	0x40023c00

08001a04 <HAL_TIM_Base_Init>:
  *         Ex: call @ref HAL_TIM_Base_DeInit() before HAL_TIM_Base_Init()
  * @param  htim TIM Base handle
  * @retval HAL status
  */
HAL_StatusTypeDef HAL_TIM_Base_Init(TIM_HandleTypeDef *htim)
{
 8001a04:	b580      	push	{r7, lr}
 8001a06:	b082      	sub	sp, #8
 8001a08:	af00      	add	r7, sp, #0
 8001a0a:	6078      	str	r0, [r7, #4]
  /* Check the TIM handle allocation */
  if (htim == NULL)
 8001a0c:	687b      	ldr	r3, [r7, #4]
 8001a0e:	2b00      	cmp	r3, #0
 8001a10:	d101      	bne.n	8001a16 <HAL_TIM_Base_Init+0x12>
  {
    return HAL_ERROR;
 8001a12:	2301      	movs	r3, #1
 8001a14:	e041      	b.n	8001a9a <HAL_TIM_Base_Init+0x96>
  assert_param(IS_TIM_INSTANCE(htim->Instance));
  assert_param(IS_TIM_COUNTER_MODE(htim->Init.CounterMode));
  assert_param(IS_TIM_CLOCKDIVISION_DIV(htim->Init.ClockDivision));
  assert_param(IS_TIM_AUTORELOAD_PRELOAD(htim->Init.AutoReloadPreload));

  if (htim->State == HAL_TIM_STATE_RESET)
 8001a16:	687b      	ldr	r3, [r7, #4]
 8001a18:	f893 303d 	ldrb.w	r3, [r3, #61]	; 0x3d
 8001a1c:	b2db      	uxtb	r3, r3
 8001a1e:	2b00      	cmp	r3, #0
 8001a20:	d106      	bne.n	8001a30 <HAL_TIM_Base_Init+0x2c>
  {
    /* Allocate lock resource and initialize it */
    htim->Lock = HAL_UNLOCKED;
 8001a22:	687b      	ldr	r3, [r7, #4]
 8001a24:	2200      	movs	r2, #0
 8001a26:	f883 203c 	strb.w	r2, [r3, #60]	; 0x3c
    }
    /* Init the low level hardware : GPIO, CLOCK, NVIC */
    htim->Base_MspInitCallback(htim);
#else
    /* Init the low level hardware : GPIO, CLOCK, NVIC */
    HAL_TIM_Base_MspInit(htim);
 8001a2a:	6878      	ldr	r0, [r7, #4]
 8001a2c:	f000 f839 	bl	8001aa2 <HAL_TIM_Base_MspInit>
#endif /* USE_HAL_TIM_REGISTER_CALLBACKS */
  }

  /* Set the TIM state */
  htim->State = HAL_TIM_STATE_BUSY;
 8001a30:	687b      	ldr	r3, [r7, #4]
 8001a32:	2202      	movs	r2, #2
 8001a34:	f883 203d 	strb.w	r2, [r3, #61]	; 0x3d

  /* Set the Time Base configuration */
  TIM_Base_SetConfig(htim->Instance, &htim->Init);
 8001a38:	687b      	ldr	r3, [r7, #4]
 8001a3a:	681a      	ldr	r2, [r3, #0]
 8001a3c:	687b      	ldr	r3, [r7, #4]
 8001a3e:	3304      	adds	r3, #4
 8001a40:	4619      	mov	r1, r3
 8001a42:	4610      	mov	r0, r2
 8001a44:	f000 f9d8 	bl	8001df8 <TIM_Base_SetConfig>

  /* Initialize the DMA burst operation state */
  htim->DMABurstState = HAL_DMA_BURST_STATE_READY;
 8001a48:	687b      	ldr	r3, [r7, #4]
 8001a4a:	2201      	movs	r2, #1
 8001a4c:	f883 2046 	strb.w	r2, [r3, #70]	; 0x46

  /* Initialize the TIM channels state */
  TIM_CHANNEL_STATE_SET_ALL(htim, HAL_TIM_CHANNEL_STATE_READY);
 8001a50:	687b      	ldr	r3, [r7, #4]
 8001a52:	2201      	movs	r2, #1
 8001a54:	f883 203e 	strb.w	r2, [r3, #62]	; 0x3e
 8001a58:	687b      	ldr	r3, [r7, #4]
 8001a5a:	2201      	movs	r2, #1
 8001a5c:	f883 203f 	strb.w	r2, [r3, #63]	; 0x3f
 8001a60:	687b      	ldr	r3, [r7, #4]
 8001a62:	2201      	movs	r2, #1
 8001a64:	f883 2040 	strb.w	r2, [r3, #64]	; 0x40
 8001a68:	687b      	ldr	r3, [r7, #4]
 8001a6a:	2201      	movs	r2, #1
 8001a6c:	f883 2041 	strb.w	r2, [r3, #65]	; 0x41
  TIM_CHANNEL_N_STATE_SET_ALL(htim, HAL_TIM_CHANNEL_STATE_READY);
 8001a70:	687b      	ldr	r3, [r7, #4]
 8001a72:	2201      	movs	r2, #1
 8001a74:	f883 2042 	strb.w	r2, [r3, #66]	; 0x42
 8001a78:	687b      	ldr	r3, [r7, #4]
 8001a7a:	2201      	movs	r2, #1
 8001a7c:	f883 2043 	strb.w	r2, [r3, #67]	; 0x43
 8001a80:	687b      	ldr	r3, [r7, #4]
 8001a82:	2201      	movs	r2, #1
 8001a84:	f883 2044 	strb.w	r2, [r3, #68]	; 0x44
 8001a88:	687b      	ldr	r3, [r7, #4]
 8001a8a:	2201      	movs	r2, #1
 8001a8c:	f883 2045 	strb.w	r2, [r3, #69]	; 0x45

  /* Initialize the TIM state*/
  htim->State = HAL_TIM_STATE_READY;
 8001a90:	687b      	ldr	r3, [r7, #4]
 8001a92:	2201      	movs	r2, #1
 8001a94:	f883 203d 	strb.w	r2, [r3, #61]	; 0x3d

  return HAL_OK;
 8001a98:	2300      	movs	r3, #0
}
 8001a9a:	4618      	mov	r0, r3
 8001a9c:	3708      	adds	r7, #8
 8001a9e:	46bd      	mov	sp, r7
 8001aa0:	bd80      	pop	{r7, pc}

08001aa2 <HAL_TIM_Base_MspInit>:
  * @brief  Initializes the TIM Base MSP.
  * @param  htim TIM Base handle
  * @retval None
  */
__weak void HAL_TIM_Base_MspInit(TIM_HandleTypeDef *htim)
{
 8001aa2:	b480      	push	{r7}
 8001aa4:	b083      	sub	sp, #12
 8001aa6:	af00      	add	r7, sp, #0
 8001aa8:	6078      	str	r0, [r7, #4]
  UNUSED(htim);

  /* NOTE : This function should not be modified, when the callback is needed,
            the HAL_TIM_Base_MspInit could be implemented in the user file
   */
}
 8001aaa:	bf00      	nop
 8001aac:	370c      	adds	r7, #12
 8001aae:	46bd      	mov	sp, r7
 8001ab0:	f85d 7b04 	ldr.w	r7, [sp], #4
 8001ab4:	4770      	bx	lr
	...

08001ab8 <HAL_TIM_Base_Start_IT>:
  * @brief  Starts the TIM Base generation in interrupt mode.
  * @param  htim TIM Base handle
  * @retval HAL status
  */
HAL_StatusTypeDef HAL_TIM_Base_Start_IT(TIM_HandleTypeDef *htim)
{
 8001ab8:	b480      	push	{r7}
 8001aba:	b085      	sub	sp, #20
 8001abc:	af00      	add	r7, sp, #0
 8001abe:	6078      	str	r0, [r7, #4]

  /* Check the parameters */
  assert_param(IS_TIM_INSTANCE(htim->Instance));

  /* Check the TIM state */
  if (htim->State != HAL_TIM_STATE_READY)
 8001ac0:	687b      	ldr	r3, [r7, #4]
 8001ac2:	f893 303d 	ldrb.w	r3, [r3, #61]	; 0x3d
 8001ac6:	b2db      	uxtb	r3, r3
 8001ac8:	2b01      	cmp	r3, #1
 8001aca:	d001      	beq.n	8001ad0 <HAL_TIM_Base_Start_IT+0x18>
  {
    return HAL_ERROR;
 8001acc:	2301      	movs	r3, #1
 8001ace:	e04e      	b.n	8001b6e <HAL_TIM_Base_Start_IT+0xb6>
  }

  /* Set the TIM state */
  htim->State = HAL_TIM_STATE_BUSY;
 8001ad0:	687b      	ldr	r3, [r7, #4]
 8001ad2:	2202      	movs	r2, #2
 8001ad4:	f883 203d 	strb.w	r2, [r3, #61]	; 0x3d

  /* Enable the TIM Update interrupt */
  __HAL_TIM_ENABLE_IT(htim, TIM_IT_UPDATE);
 8001ad8:	687b      	ldr	r3, [r7, #4]
 8001ada:	681b      	ldr	r3, [r3, #0]
 8001adc:	68da      	ldr	r2, [r3, #12]
 8001ade:	687b      	ldr	r3, [r7, #4]
 8001ae0:	681b      	ldr	r3, [r3, #0]
 8001ae2:	f042 0201 	orr.w	r2, r2, #1
 8001ae6:	60da      	str	r2, [r3, #12]

  /* Enable the Peripheral, except in trigger mode where enable is automatically done with trigger */
  if (IS_TIM_SLAVE_INSTANCE(htim->Instance))
 8001ae8:	687b      	ldr	r3, [r7, #4]
 8001aea:	681b      	ldr	r3, [r3, #0]
 8001aec:	4a23      	ldr	r2, [pc, #140]	; (8001b7c <HAL_TIM_Base_Start_IT+0xc4>)
 8001aee:	4293      	cmp	r3, r2
 8001af0:	d022      	beq.n	8001b38 <HAL_TIM_Base_Start_IT+0x80>
 8001af2:	687b      	ldr	r3, [r7, #4]
 8001af4:	681b      	ldr	r3, [r3, #0]
 8001af6:	f1b3 4f80 	cmp.w	r3, #1073741824	; 0x40000000
 8001afa:	d01d      	beq.n	8001b38 <HAL_TIM_Base_Start_IT+0x80>
 8001afc:	687b      	ldr	r3, [r7, #4]
 8001afe:	681b      	ldr	r3, [r3, #0]
 8001b00:	4a1f      	ldr	r2, [pc, #124]	; (8001b80 <HAL_TIM_Base_Start_IT+0xc8>)
 8001b02:	4293      	cmp	r3, r2
 8001b04:	d018      	beq.n	8001b38 <HAL_TIM_Base_Start_IT+0x80>
 8001b06:	687b      	ldr	r3, [r7, #4]
 8001b08:	681b      	ldr	r3, [r3, #0]
 8001b0a:	4a1e      	ldr	r2, [pc, #120]	; (8001b84 <HAL_TIM_Base_Start_IT+0xcc>)
 8001b0c:	4293      	cmp	r3, r2
 8001b0e:	d013      	beq.n	8001b38 <HAL_TIM_Base_Start_IT+0x80>
 8001b10:	687b      	ldr	r3, [r7, #4]
 8001b12:	681b      	ldr	r3, [r3, #0]
 8001b14:	4a1c      	ldr	r2, [pc, #112]	; (8001b88 <HAL_TIM_Base_Start_IT+0xd0>)
 8001b16:	4293      	cmp	r3, r2
 8001b18:	d00e      	beq.n	8001b38 <HAL_TIM_Base_Start_IT+0x80>
 8001b1a:	687b      	ldr	r3, [r7, #4]
 8001b1c:	681b      	ldr	r3, [r3, #0]
 8001b1e:	4a1b      	ldr	r2, [pc, #108]	; (8001b8c <HAL_TIM_Base_Start_IT+0xd4>)
 8001b20:	4293      	cmp	r3, r2
 8001b22:	d009      	beq.n	8001b38 <HAL_TIM_Base_Start_IT+0x80>
 8001b24:	687b      	ldr	r3, [r7, #4]
 8001b26:	681b      	ldr	r3, [r3, #0]
 8001b28:	4a19      	ldr	r2, [pc, #100]	; (8001b90 <HAL_TIM_Base_Start_IT+0xd8>)
 8001b2a:	4293      	cmp	r3, r2
 8001b2c:	d004      	beq.n	8001b38 <HAL_TIM_Base_Start_IT+0x80>
 8001b2e:	687b      	ldr	r3, [r7, #4]
 8001b30:	681b      	ldr	r3, [r3, #0]
 8001b32:	4a18      	ldr	r2, [pc, #96]	; (8001b94 <HAL_TIM_Base_Start_IT+0xdc>)
 8001b34:	4293      	cmp	r3, r2
 8001b36:	d111      	bne.n	8001b5c <HAL_TIM_Base_Start_IT+0xa4>
  {
    tmpsmcr = htim->Instance->SMCR & TIM_SMCR_SMS;
 8001b38:	687b      	ldr	r3, [r7, #4]
 8001b3a:	681b      	ldr	r3, [r3, #0]
 8001b3c:	689b      	ldr	r3, [r3, #8]
 8001b3e:	f003 0307 	and.w	r3, r3, #7
 8001b42:	60fb      	str	r3, [r7, #12]
    if (!IS_TIM_SLAVEMODE_TRIGGER_ENABLED(tmpsmcr))
 8001b44:	68fb      	ldr	r3, [r7, #12]
 8001b46:	2b06      	cmp	r3, #6
 8001b48:	d010      	beq.n	8001b6c <HAL_TIM_Base_Start_IT+0xb4>
    {
      __HAL_TIM_ENABLE(htim);
 8001b4a:	687b      	ldr	r3, [r7, #4]
 8001b4c:	681b      	ldr	r3, [r3, #0]
 8001b4e:	681a      	ldr	r2, [r3, #0]
 8001b50:	687b      	ldr	r3, [r7, #4]
 8001b52:	681b      	ldr	r3, [r3, #0]
 8001b54:	f042 0201 	orr.w	r2, r2, #1
 8001b58:	601a      	str	r2, [r3, #0]
    if (!IS_TIM_SLAVEMODE_TRIGGER_ENABLED(tmpsmcr))
 8001b5a:	e007      	b.n	8001b6c <HAL_TIM_Base_Start_IT+0xb4>
    }
  }
  else
  {
    __HAL_TIM_ENABLE(htim);
 8001b5c:	687b      	ldr	r3, [r7, #4]
 8001b5e:	681b      	ldr	r3, [r3, #0]
 8001b60:	681a      	ldr	r2, [r3, #0]
 8001b62:	687b      	ldr	r3, [r7, #4]
 8001b64:	681b      	ldr	r3, [r3, #0]
 8001b66:	f042 0201 	orr.w	r2, r2, #1
 8001b6a:	601a      	str	r2, [r3, #0]
  }

  /* Return function status */
  return HAL_OK;
 8001b6c:	2300      	movs	r3, #0
}
 8001b6e:	4618      	mov	r0, r3
 8001b70:	3714      	adds	r7, #20
 8001b72:	46bd      	mov	sp, r7
 8001b74:	f85d 7b04 	ldr.w	r7, [sp], #4
 8001b78:	4770      	bx	lr
 8001b7a:	bf00      	nop
 8001b7c:	40010000 	.word	0x40010000
 8001b80:	40000400 	.word	0x40000400
 8001b84:	40000800 	.word	0x40000800
 8001b88:	40000c00 	.word	0x40000c00
 8001b8c:	40010400 	.word	0x40010400
 8001b90:	40014000 	.word	0x40014000
 8001b94:	40001800 	.word	0x40001800

08001b98 <HAL_TIM_IRQHandler>:
  * @brief  This function handles TIM interrupts requests.
  * @param  htim TIM  handle
  * @retval None
  */
void HAL_TIM_IRQHandler(TIM_HandleTypeDef *htim)
{
 8001b98:	b580      	push	{r7, lr}
 8001b9a:	b082      	sub	sp, #8
 8001b9c:	af00      	add	r7, sp, #0
 8001b9e:	6078      	str	r0, [r7, #4]
  /* Capture compare 1 event */
  if (__HAL_TIM_GET_FLAG(htim, TIM_FLAG_CC1) != RESET)
 8001ba0:	687b      	ldr	r3, [r7, #4]
 8001ba2:	681b      	ldr	r3, [r3, #0]
 8001ba4:	691b      	ldr	r3, [r3, #16]
 8001ba6:	f003 0302 	and.w	r3, r3, #2
 8001baa:	2b02      	cmp	r3, #2
 8001bac:	d122      	bne.n	8001bf4 <HAL_TIM_IRQHandler+0x5c>
  {
    if (__HAL_TIM_GET_IT_SOURCE(htim, TIM_IT_CC1) != RESET)
 8001bae:	687b      	ldr	r3, [r7, #4]
 8001bb0:	681b      	ldr	r3, [r3, #0]
 8001bb2:	68db      	ldr	r3, [r3, #12]
 8001bb4:	f003 0302 	and.w	r3, r3, #2
 8001bb8:	2b02      	cmp	r3, #2
 8001bba:	d11b      	bne.n	8001bf4 <HAL_TIM_IRQHandler+0x5c>
    {
      {
        __HAL_TIM_CLEAR_IT(htim, TIM_IT_CC1);
 8001bbc:	687b      	ldr	r3, [r7, #4]
 8001bbe:	681b      	ldr	r3, [r3, #0]
 8001bc0:	f06f 0202 	mvn.w	r2, #2
 8001bc4:	611a      	str	r2, [r3, #16]
        htim->Channel = HAL_TIM_ACTIVE_CHANNEL_1;
 8001bc6:	687b      	ldr	r3, [r7, #4]
 8001bc8:	2201      	movs	r2, #1
 8001bca:	771a      	strb	r2, [r3, #28]

        /* Input capture event */
        if ((htim->Instance->CCMR1 & TIM_CCMR1_CC1S) != 0x00U)
 8001bcc:	687b      	ldr	r3, [r7, #4]
 8001bce:	681b      	ldr	r3, [r3, #0]
 8001bd0:	699b      	ldr	r3, [r3, #24]
 8001bd2:	f003 0303 	and.w	r3, r3, #3
 8001bd6:	2b00      	cmp	r3, #0
 8001bd8:	d003      	beq.n	8001be2 <HAL_TIM_IRQHandler+0x4a>
        {
#if (USE_HAL_TIM_REGISTER_CALLBACKS == 1)
          htim->IC_CaptureCallback(htim);
#else
          HAL_TIM_IC_CaptureCallback(htim);
 8001bda:	6878      	ldr	r0, [r7, #4]
 8001bdc:	f000 f8ee 	bl	8001dbc <HAL_TIM_IC_CaptureCallback>
 8001be0:	e005      	b.n	8001bee <HAL_TIM_IRQHandler+0x56>
        {
#if (USE_HAL_TIM_REGISTER_CALLBACKS == 1)
          htim->OC_DelayElapsedCallback(htim);
          htim->PWM_PulseFinishedCallback(htim);
#else
          HAL_TIM_OC_DelayElapsedCallback(htim);
 8001be2:	6878      	ldr	r0, [r7, #4]
 8001be4:	f000 f8e0 	bl	8001da8 <HAL_TIM_OC_DelayElapsedCallback>
          HAL_TIM_PWM_PulseFinishedCallback(htim);
 8001be8:	6878      	ldr	r0, [r7, #4]
 8001bea:	f000 f8f1 	bl	8001dd0 <HAL_TIM_PWM_PulseFinishedCallback>
#endif /* USE_HAL_TIM_REGISTER_CALLBACKS */
        }
        htim->Channel = HAL_TIM_ACTIVE_CHANNEL_CLEARED;
 8001bee:	687b      	ldr	r3, [r7, #4]
 8001bf0:	2200      	movs	r2, #0
 8001bf2:	771a      	strb	r2, [r3, #28]
      }
    }
  }
  /* Capture compare 2 event */
  if (__HAL_TIM_GET_FLAG(htim, TIM_FLAG_CC2) != RESET)
 8001bf4:	687b      	ldr	r3, [r7, #4]
 8001bf6:	681b      	ldr	r3, [r3, #0]
 8001bf8:	691b      	ldr	r3, [r3, #16]
 8001bfa:	f003 0304 	and.w	r3, r3, #4
 8001bfe:	2b04      	cmp	r3, #4
 8001c00:	d122      	bne.n	8001c48 <HAL_TIM_IRQHandler+0xb0>
  {
    if (__HAL_TIM_GET_IT_SOURCE(htim, TIM_IT_CC2) != RESET)
 8001c02:	687b      	ldr	r3, [r7, #4]
 8001c04:	681b      	ldr	r3, [r3, #0]
 8001c06:	68db      	ldr	r3, [r3, #12]
 8001c08:	f003 0304 	and.w	r3, r3, #4
 8001c0c:	2b04      	cmp	r3, #4
 8001c0e:	d11b      	bne.n	8001c48 <HAL_TIM_IRQHandler+0xb0>
    {
      __HAL_TIM_CLEAR_IT(htim, TIM_IT_CC2);
 8001c10:	687b      	ldr	r3, [r7, #4]
 8001c12:	681b      	ldr	r3, [r3, #0]
 8001c14:	f06f 0204 	mvn.w	r2, #4
 8001c18:	611a      	str	r2, [r3, #16]
      htim->Channel = HAL_TIM_ACTIVE_CHANNEL_2;
 8001c1a:	687b      	ldr	r3, [r7, #4]
 8001c1c:	2202      	movs	r2, #2
 8001c1e:	771a      	strb	r2, [r3, #28]
      /* Input capture event */
      if ((htim->Instance->CCMR1 & TIM_CCMR1_CC2S) != 0x00U)
 8001c20:	687b      	ldr	r3, [r7, #4]
 8001c22:	681b      	ldr	r3, [r3, #0]
 8001c24:	699b      	ldr	r3, [r3, #24]
 8001c26:	f403 7340 	and.w	r3, r3, #768	; 0x300
 8001c2a:	2b00      	cmp	r3, #0
 8001c2c:	d003      	beq.n	8001c36 <HAL_TIM_IRQHandler+0x9e>
      {
#if (USE_HAL_TIM_REGISTER_CALLBACKS == 1)
        htim->IC_CaptureCallback(htim);
#else
        HAL_TIM_IC_CaptureCallback(htim);
 8001c2e:	6878      	ldr	r0, [r7, #4]
 8001c30:	f000 f8c4 	bl	8001dbc <HAL_TIM_IC_CaptureCallback>
 8001c34:	e005      	b.n	8001c42 <HAL_TIM_IRQHandler+0xaa>
      {
#if (USE_HAL_TIM_REGISTER_CALLBACKS == 1)
        htim->OC_DelayElapsedCallback(htim);
        htim->PWM_PulseFinishedCallback(htim);
#else
        HAL_TIM_OC_DelayElapsedCallback(htim);
 8001c36:	6878      	ldr	r0, [r7, #4]
 8001c38:	f000 f8b6 	bl	8001da8 <HAL_TIM_OC_DelayElapsedCallback>
        HAL_TIM_PWM_PulseFinishedCallback(htim);
 8001c3c:	6878      	ldr	r0, [r7, #4]
 8001c3e:	f000 f8c7 	bl	8001dd0 <HAL_TIM_PWM_PulseFinishedCallback>
#endif /* USE_HAL_TIM_REGISTER_CALLBACKS */
      }
      htim->Channel = HAL_TIM_ACTIVE_CHANNEL_CLEARED;
 8001c42:	687b      	ldr	r3, [r7, #4]
 8001c44:	2200      	movs	r2, #0
 8001c46:	771a      	strb	r2, [r3, #28]
    }
  }
  /* Capture compare 3 event */
  if (__HAL_TIM_GET_FLAG(htim, TIM_FLAG_CC3) != RESET)
 8001c48:	687b      	ldr	r3, [r7, #4]
 8001c4a:	681b      	ldr	r3, [r3, #0]
 8001c4c:	691b      	ldr	r3, [r3, #16]
 8001c4e:	f003 0308 	and.w	r3, r3, #8
 8001c52:	2b08      	cmp	r3, #8
 8001c54:	d122      	bne.n	8001c9c <HAL_TIM_IRQHandler+0x104>
  {
    if (__HAL_TIM_GET_IT_SOURCE(htim, TIM_IT_CC3) != RESET)
 8001c56:	687b      	ldr	r3, [r7, #4]
 8001c58:	681b      	ldr	r3, [r3, #0]
 8001c5a:	68db      	ldr	r3, [r3, #12]
 8001c5c:	f003 0308 	and.w	r3, r3, #8
 8001c60:	2b08      	cmp	r3, #8
 8001c62:	d11b      	bne.n	8001c9c <HAL_TIM_IRQHandler+0x104>
    {
      __HAL_TIM_CLEAR_IT(htim, TIM_IT_CC3);
 8001c64:	687b      	ldr	r3, [r7, #4]
 8001c66:	681b      	ldr	r3, [r3, #0]
 8001c68:	f06f 0208 	mvn.w	r2, #8
 8001c6c:	611a      	str	r2, [r3, #16]
      htim->Channel = HAL_TIM_ACTIVE_CHANNEL_3;
 8001c6e:	687b      	ldr	r3, [r7, #4]
 8001c70:	2204      	movs	r2, #4
 8001c72:	771a      	strb	r2, [r3, #28]
      /* Input capture event */
      if ((htim->Instance->CCMR2 & TIM_CCMR2_CC3S) != 0x00U)
 8001c74:	687b      	ldr	r3, [r7, #4]
 8001c76:	681b      	ldr	r3, [r3, #0]
 8001c78:	69db      	ldr	r3, [r3, #28]
 8001c7a:	f003 0303 	and.w	r3, r3, #3
 8001c7e:	2b00      	cmp	r3, #0
 8001c80:	d003      	beq.n	8001c8a <HAL_TIM_IRQHandler+0xf2>
      {
#if (USE_HAL_TIM_REGISTER_CALLBACKS == 1)
        htim->IC_CaptureCallback(htim);
#else
        HAL_TIM_IC_CaptureCallback(htim);
 8001c82:	6878      	ldr	r0, [r7, #4]
 8001c84:	f000 f89a 	bl	8001dbc <HAL_TIM_IC_CaptureCallback>
 8001c88:	e005      	b.n	8001c96 <HAL_TIM_IRQHandler+0xfe>
      {
#if (USE_HAL_TIM_REGISTER_CALLBACKS == 1)
        htim->OC_DelayElapsedCallback(htim);
        htim->PWM_PulseFinishedCallback(htim);
#else
        HAL_TIM_OC_DelayElapsedCallback(htim);
 8001c8a:	6878      	ldr	r0, [r7, #4]
 8001c8c:	f000 f88c 	bl	8001da8 <HAL_TIM_OC_DelayElapsedCallback>
        HAL_TIM_PWM_PulseFinishedCallback(htim);
 8001c90:	6878      	ldr	r0, [r7, #4]
 8001c92:	f000 f89d 	bl	8001dd0 <HAL_TIM_PWM_PulseFinishedCallback>
#endif /* USE_HAL_TIM_REGISTER_CALLBACKS */
      }
      htim->Channel = HAL_TIM_ACTIVE_CHANNEL_CLEARED;
 8001c96:	687b      	ldr	r3, [r7, #4]
 8001c98:	2200      	movs	r2, #0
 8001c9a:	771a      	strb	r2, [r3, #28]
    }
  }
  /* Capture compare 4 event */
  if (__HAL_TIM_GET_FLAG(htim, TIM_FLAG_CC4) != RESET)
 8001c9c:	687b      	ldr	r3, [r7, #4]
 8001c9e:	681b      	ldr	r3, [r3, #0]
 8001ca0:	691b      	ldr	r3, [r3, #16]
 8001ca2:	f003 0310 	and.w	r3, r3, #16
 8001ca6:	2b10      	cmp	r3, #16
 8001ca8:	d122      	bne.n	8001cf0 <HAL_TIM_IRQHandler+0x158>
  {
    if (__HAL_TIM_GET_IT_SOURCE(htim, TIM_IT_CC4) != RESET)
 8001caa:	687b      	ldr	r3, [r7, #4]
 8001cac:	681b      	ldr	r3, [r3, #0]
 8001cae:	68db      	ldr	r3, [r3, #12]
 8001cb0:	f003 0310 	and.w	r3, r3, #16
 8001cb4:	2b10      	cmp	r3, #16
 8001cb6:	d11b      	bne.n	8001cf0 <HAL_TIM_IRQHandler+0x158>
    {
      __HAL_TIM_CLEAR_IT(htim, TIM_IT_CC4);
 8001cb8:	687b      	ldr	r3, [r7, #4]
 8001cba:	681b      	ldr	r3, [r3, #0]
 8001cbc:	f06f 0210 	mvn.w	r2, #16
 8001cc0:	611a      	str	r2, [r3, #16]
      htim->Channel = HAL_TIM_ACTIVE_CHANNEL_4;
 8001cc2:	687b      	ldr	r3, [r7, #4]
 8001cc4:	2208      	movs	r2, #8
 8001cc6:	771a      	strb	r2, [r3, #28]
      /* Input capture event */
      if ((htim->Instance->CCMR2 & TIM_CCMR2_CC4S) != 0x00U)
 8001cc8:	687b      	ldr	r3, [r7, #4]
 8001cca:	681b      	ldr	r3, [r3, #0]
 8001ccc:	69db      	ldr	r3, [r3, #28]
 8001cce:	f403 7340 	and.w	r3, r3, #768	; 0x300
 8001cd2:	2b00      	cmp	r3, #0
 8001cd4:	d003      	beq.n	8001cde <HAL_TIM_IRQHandler+0x146>
      {
#if (USE_HAL_TIM_REGISTER_CALLBACKS == 1)
        htim->IC_CaptureCallback(htim);
#else
        HAL_TIM_IC_CaptureCallback(htim);
 8001cd6:	6878      	ldr	r0, [r7, #4]
 8001cd8:	f000 f870 	bl	8001dbc <HAL_TIM_IC_CaptureCallback>
 8001cdc:	e005      	b.n	8001cea <HAL_TIM_IRQHandler+0x152>
      {
#if (USE_HAL_TIM_REGISTER_CALLBACKS == 1)
        htim->OC_DelayElapsedCallback(htim);
        htim->PWM_PulseFinishedCallback(htim);
#else
        HAL_TIM_OC_DelayElapsedCallback(htim);
 8001cde:	6878      	ldr	r0, [r7, #4]
 8001ce0:	f000 f862 	bl	8001da8 <HAL_TIM_OC_DelayElapsedCallback>
        HAL_TIM_PWM_PulseFinishedCallback(htim);
 8001ce4:	6878      	ldr	r0, [r7, #4]
 8001ce6:	f000 f873 	bl	8001dd0 <HAL_TIM_PWM_PulseFinishedCallback>
#endif /* USE_HAL_TIM_REGISTER_CALLBACKS */
      }
      htim->Channel = HAL_TIM_ACTIVE_CHANNEL_CLEARED;
 8001cea:	687b      	ldr	r3, [r7, #4]
 8001cec:	2200      	movs	r2, #0
 8001cee:	771a      	strb	r2, [r3, #28]
    }
  }
  /* TIM Update event */
  if (__HAL_TIM_GET_FLAG(htim, TIM_FLAG_UPDATE) != RESET)
 8001cf0:	687b      	ldr	r3, [r7, #4]
 8001cf2:	681b      	ldr	r3, [r3, #0]
 8001cf4:	691b      	ldr	r3, [r3, #16]
 8001cf6:	f003 0301 	and.w	r3, r3, #1
 8001cfa:	2b01      	cmp	r3, #1
 8001cfc:	d10e      	bne.n	8001d1c <HAL_TIM_IRQHandler+0x184>
  {
    if (__HAL_TIM_GET_IT_SOURCE(htim, TIM_IT_UPDATE) != RESET)
 8001cfe:	687b      	ldr	r3, [r7, #4]
 8001d00:	681b      	ldr	r3, [r3, #0]
 8001d02:	68db      	ldr	r3, [r3, #12]
 8001d04:	f003 0301 	and.w	r3, r3, #1
 8001d08:	2b01      	cmp	r3, #1
 8001d0a:	d107      	bne.n	8001d1c <HAL_TIM_IRQHandler+0x184>
    {
      __HAL_TIM_CLEAR_IT(htim, TIM_IT_UPDATE);
 8001d0c:	687b      	ldr	r3, [r7, #4]
 8001d0e:	681b      	ldr	r3, [r3, #0]
 8001d10:	f06f 0201 	mvn.w	r2, #1
 8001d14:	611a      	str	r2, [r3, #16]
#if (USE_HAL_TIM_REGISTER_CALLBACKS == 1)
      htim->PeriodElapsedCallback(htim);
#else
      HAL_TIM_PeriodElapsedCallback(htim);
 8001d16:	6878      	ldr	r0, [r7, #4]
 8001d18:	f7fe fd9a 	bl	8000850 <HAL_TIM_PeriodElapsedCallback>
#endif /* USE_HAL_TIM_REGISTER_CALLBACKS */
    }
  }
  /* TIM Break input event */
  if (__HAL_TIM_GET_FLAG(htim, TIM_FLAG_BREAK) != RESET)
 8001d1c:	687b      	ldr	r3, [r7, #4]
 8001d1e:	681b      	ldr	r3, [r3, #0]
 8001d20:	691b      	ldr	r3, [r3, #16]
 8001d22:	f003 0380 	and.w	r3, r3, #128	; 0x80
 8001d26:	2b80      	cmp	r3, #128	; 0x80
 8001d28:	d10e      	bne.n	8001d48 <HAL_TIM_IRQHandler+0x1b0>
  {
    if (__HAL_TIM_GET_IT_SOURCE(htim, TIM_IT_BREAK) != RESET)
 8001d2a:	687b      	ldr	r3, [r7, #4]
 8001d2c:	681b      	ldr	r3, [r3, #0]
 8001d2e:	68db      	ldr	r3, [r3, #12]
 8001d30:	f003 0380 	and.w	r3, r3, #128	; 0x80
 8001d34:	2b80      	cmp	r3, #128	; 0x80
 8001d36:	d107      	bne.n	8001d48 <HAL_TIM_IRQHandler+0x1b0>
    {
      __HAL_TIM_CLEAR_IT(htim, TIM_IT_BREAK);
 8001d38:	687b      	ldr	r3, [r7, #4]
 8001d3a:	681b      	ldr	r3, [r3, #0]
 8001d3c:	f06f 0280 	mvn.w	r2, #128	; 0x80
 8001d40:	611a      	str	r2, [r3, #16]
#if (USE_HAL_TIM_REGISTER_CALLBACKS == 1)
      htim->BreakCallback(htim);
#else
      HAL_TIMEx_BreakCallback(htim);
 8001d42:	6878      	ldr	r0, [r7, #4]
 8001d44:	f000 f902 	bl	8001f4c <HAL_TIMEx_BreakCallback>
#endif /* USE_HAL_TIM_REGISTER_CALLBACKS */
    }
  }
  /* TIM Trigger detection event */
  if (__HAL_TIM_GET_FLAG(htim, TIM_FLAG_TRIGGER) != RESET)
 8001d48:	687b      	ldr	r3, [r7, #4]
 8001d4a:	681b      	ldr	r3, [r3, #0]
 8001d4c:	691b      	ldr	r3, [r3, #16]
 8001d4e:	f003 0340 	and.w	r3, r3, #64	; 0x40
 8001d52:	2b40      	cmp	r3, #64	; 0x40
 8001d54:	d10e      	bne.n	8001d74 <HAL_TIM_IRQHandler+0x1dc>
  {
    if (__HAL_TIM_GET_IT_SOURCE(htim, TIM_IT_TRIGGER) != RESET)
 8001d56:	687b      	ldr	r3, [r7, #4]
 8001d58:	681b      	ldr	r3, [r3, #0]
 8001d5a:	68db      	ldr	r3, [r3, #12]
 8001d5c:	f003 0340 	and.w	r3, r3, #64	; 0x40
 8001d60:	2b40      	cmp	r3, #64	; 0x40
 8001d62:	d107      	bne.n	8001d74 <HAL_TIM_IRQHandler+0x1dc>
    {
      __HAL_TIM_CLEAR_IT(htim, TIM_IT_TRIGGER);
 8001d64:	687b      	ldr	r3, [r7, #4]
 8001d66:	681b      	ldr	r3, [r3, #0]
 8001d68:	f06f 0240 	mvn.w	r2, #64	; 0x40
 8001d6c:	611a      	str	r2, [r3, #16]
#if (USE_HAL_TIM_REGISTER_CALLBACKS == 1)
      htim->TriggerCallback(htim);
#else
      HAL_TIM_TriggerCallback(htim);
 8001d6e:	6878      	ldr	r0, [r7, #4]
 8001d70:	f000 f838 	bl	8001de4 <HAL_TIM_TriggerCallback>
#endif /* USE_HAL_TIM_REGISTER_CALLBACKS */
    }
  }
  /* TIM commutation event */
  if (__HAL_TIM_GET_FLAG(htim, TIM_FLAG_COM) != RESET)
 8001d74:	687b      	ldr	r3, [r7, #4]
 8001d76:	681b      	ldr	r3, [r3, #0]
 8001d78:	691b      	ldr	r3, [r3, #16]
 8001d7a:	f003 0320 	and.w	r3, r3, #32
 8001d7e:	2b20      	cmp	r3, #32
 8001d80:	d10e      	bne.n	8001da0 <HAL_TIM_IRQHandler+0x208>
  {
    if (__HAL_TIM_GET_IT_SOURCE(htim, TIM_IT_COM) != RESET)
 8001d82:	687b      	ldr	r3, [r7, #4]
 8001d84:	681b      	ldr	r3, [r3, #0]
 8001d86:	68db      	ldr	r3, [r3, #12]
 8001d88:	f003 0320 	and.w	r3, r3, #32
 8001d8c:	2b20      	cmp	r3, #32
 8001d8e:	d107      	bne.n	8001da0 <HAL_TIM_IRQHandler+0x208>
    {
      __HAL_TIM_CLEAR_IT(htim, TIM_FLAG_COM);
 8001d90:	687b      	ldr	r3, [r7, #4]
 8001d92:	681b      	ldr	r3, [r3, #0]
 8001d94:	f06f 0220 	mvn.w	r2, #32
 8001d98:	611a      	str	r2, [r3, #16]
#if (USE_HAL_TIM_REGISTER_CALLBACKS == 1)
      htim->CommutationCallback(htim);
#else
      HAL_TIMEx_CommutCallback(htim);
 8001d9a:	6878      	ldr	r0, [r7, #4]
 8001d9c:	f000 f8cc 	bl	8001f38 <HAL_TIMEx_CommutCallback>
#endif /* USE_HAL_TIM_REGISTER_CALLBACKS */
    }
  }
}
 8001da0:	bf00      	nop
 8001da2:	3708      	adds	r7, #8
 8001da4:	46bd      	mov	sp, r7
 8001da6:	bd80      	pop	{r7, pc}

08001da8 <HAL_TIM_OC_DelayElapsedCallback>:
  * @brief  Output Compare callback in non-blocking mode
  * @param  htim TIM OC handle
  * @retval None
  */
__weak void HAL_TIM_OC_DelayElapsedCallback(TIM_HandleTypeDef *htim)
{
 8001da8:	b480      	push	{r7}
 8001daa:	b083      	sub	sp, #12
 8001dac:	af00      	add	r7, sp, #0
 8001dae:	6078      	str	r0, [r7, #4]
  UNUSED(htim);

  /* NOTE : This function should not be modified, when the callback is needed,
            the HAL_TIM_OC_DelayElapsedCallback could be implemented in the user file
   */
}
 8001db0:	bf00      	nop
 8001db2:	370c      	adds	r7, #12
 8001db4:	46bd      	mov	sp, r7
 8001db6:	f85d 7b04 	ldr.w	r7, [sp], #4
 8001dba:	4770      	bx	lr

08001dbc <HAL_TIM_IC_CaptureCallback>:
  * @brief  Input Capture callback in non-blocking mode
  * @param  htim TIM IC handle
  * @retval None
  */
__weak void HAL_TIM_IC_CaptureCallback(TIM_HandleTypeDef *htim)
{
 8001dbc:	b480      	push	{r7}
 8001dbe:	b083      	sub	sp, #12
 8001dc0:	af00      	add	r7, sp, #0
 8001dc2:	6078      	str	r0, [r7, #4]
  UNUSED(htim);

  /* NOTE : This function should not be modified, when the callback is needed,
            the HAL_TIM_IC_CaptureCallback could be implemented in the user file
   */
}
 8001dc4:	bf00      	nop
 8001dc6:	370c      	adds	r7, #12
 8001dc8:	46bd      	mov	sp, r7
 8001dca:	f85d 7b04 	ldr.w	r7, [sp], #4
 8001dce:	4770      	bx	lr

08001dd0 <HAL_TIM_PWM_PulseFinishedCallback>:
  * @brief  PWM Pulse finished callback in non-blocking mode
  * @param  htim TIM handle
  * @retval None
  */
__weak void HAL_TIM_PWM_PulseFinishedCallback(TIM_HandleTypeDef *htim)
{
 8001dd0:	b480      	push	{r7}
 8001dd2:	b083      	sub	sp, #12
 8001dd4:	af00      	add	r7, sp, #0
 8001dd6:	6078      	str	r0, [r7, #4]
  UNUSED(htim);

  /* NOTE : This function should not be modified, when the callback is needed,
            the HAL_TIM_PWM_PulseFinishedCallback could be implemented in the user file
   */
}
 8001dd8:	bf00      	nop
 8001dda:	370c      	adds	r7, #12
 8001ddc:	46bd      	mov	sp, r7
 8001dde:	f85d 7b04 	ldr.w	r7, [sp], #4
 8001de2:	4770      	bx	lr

08001de4 <HAL_TIM_TriggerCallback>:
  * @brief  Hall Trigger detection callback in non-blocking mode
  * @param  htim TIM handle
  * @retval None
  */
__weak void HAL_TIM_TriggerCallback(TIM_HandleTypeDef *htim)
{
 8001de4:	b480      	push	{r7}
 8001de6:	b083      	sub	sp, #12
 8001de8:	af00      	add	r7, sp, #0
 8001dea:	6078      	str	r0, [r7, #4]
  UNUSED(htim);

  /* NOTE : This function should not be modified, when the callback is needed,
            the HAL_TIM_TriggerCallback could be implemented in the user file
   */
}
 8001dec:	bf00      	nop
 8001dee:	370c      	adds	r7, #12
 8001df0:	46bd      	mov	sp, r7
 8001df2:	f85d 7b04 	ldr.w	r7, [sp], #4
 8001df6:	4770      	bx	lr

08001df8 <TIM_Base_SetConfig>:
  * @param  TIMx TIM peripheral
  * @param  Structure TIM Base configuration structure
  * @retval None
  */
void TIM_Base_SetConfig(TIM_TypeDef *TIMx, TIM_Base_InitTypeDef *Structure)
{
 8001df8:	b480      	push	{r7}
 8001dfa:	b085      	sub	sp, #20
 8001dfc:	af00      	add	r7, sp, #0
 8001dfe:	6078      	str	r0, [r7, #4]
 8001e00:	6039      	str	r1, [r7, #0]
  uint32_t tmpcr1;
  tmpcr1 = TIMx->CR1;
 8001e02:	687b      	ldr	r3, [r7, #4]
 8001e04:	681b      	ldr	r3, [r3, #0]
 8001e06:	60fb      	str	r3, [r7, #12]

  /* Set TIM Time Base Unit parameters ---------------------------------------*/
  if (IS_TIM_COUNTER_MODE_SELECT_INSTANCE(TIMx))
 8001e08:	687b      	ldr	r3, [r7, #4]
 8001e0a:	4a40      	ldr	r2, [pc, #256]	; (8001f0c <TIM_Base_SetConfig+0x114>)
 8001e0c:	4293      	cmp	r3, r2
 8001e0e:	d013      	beq.n	8001e38 <TIM_Base_SetConfig+0x40>
 8001e10:	687b      	ldr	r3, [r7, #4]
 8001e12:	f1b3 4f80 	cmp.w	r3, #1073741824	; 0x40000000
 8001e16:	d00f      	beq.n	8001e38 <TIM_Base_SetConfig+0x40>
 8001e18:	687b      	ldr	r3, [r7, #4]
 8001e1a:	4a3d      	ldr	r2, [pc, #244]	; (8001f10 <TIM_Base_SetConfig+0x118>)
 8001e1c:	4293      	cmp	r3, r2
 8001e1e:	d00b      	beq.n	8001e38 <TIM_Base_SetConfig+0x40>
 8001e20:	687b      	ldr	r3, [r7, #4]
 8001e22:	4a3c      	ldr	r2, [pc, #240]	; (8001f14 <TIM_Base_SetConfig+0x11c>)
 8001e24:	4293      	cmp	r3, r2
 8001e26:	d007      	beq.n	8001e38 <TIM_Base_SetConfig+0x40>
 8001e28:	687b      	ldr	r3, [r7, #4]
 8001e2a:	4a3b      	ldr	r2, [pc, #236]	; (8001f18 <TIM_Base_SetConfig+0x120>)
 8001e2c:	4293      	cmp	r3, r2
 8001e2e:	d003      	beq.n	8001e38 <TIM_Base_SetConfig+0x40>
 8001e30:	687b      	ldr	r3, [r7, #4]
 8001e32:	4a3a      	ldr	r2, [pc, #232]	; (8001f1c <TIM_Base_SetConfig+0x124>)
 8001e34:	4293      	cmp	r3, r2
 8001e36:	d108      	bne.n	8001e4a <TIM_Base_SetConfig+0x52>
  {
    /* Select the Counter Mode */
    tmpcr1 &= ~(TIM_CR1_DIR | TIM_CR1_CMS);
 8001e38:	68fb      	ldr	r3, [r7, #12]
 8001e3a:	f023 0370 	bic.w	r3, r3, #112	; 0x70
 8001e3e:	60fb      	str	r3, [r7, #12]
    tmpcr1 |= Structure->CounterMode;
 8001e40:	683b      	ldr	r3, [r7, #0]
 8001e42:	685b      	ldr	r3, [r3, #4]
 8001e44:	68fa      	ldr	r2, [r7, #12]
 8001e46:	4313      	orrs	r3, r2
 8001e48:	60fb      	str	r3, [r7, #12]
  }

  if (IS_TIM_CLOCK_DIVISION_INSTANCE(TIMx))
 8001e4a:	687b      	ldr	r3, [r7, #4]
 8001e4c:	4a2f      	ldr	r2, [pc, #188]	; (8001f0c <TIM_Base_SetConfig+0x114>)
 8001e4e:	4293      	cmp	r3, r2
 8001e50:	d02b      	beq.n	8001eaa <TIM_Base_SetConfig+0xb2>
 8001e52:	687b      	ldr	r3, [r7, #4]
 8001e54:	f1b3 4f80 	cmp.w	r3, #1073741824	; 0x40000000
 8001e58:	d027      	beq.n	8001eaa <TIM_Base_SetConfig+0xb2>
 8001e5a:	687b      	ldr	r3, [r7, #4]
 8001e5c:	4a2c      	ldr	r2, [pc, #176]	; (8001f10 <TIM_Base_SetConfig+0x118>)
 8001e5e:	4293      	cmp	r3, r2
 8001e60:	d023      	beq.n	8001eaa <TIM_Base_SetConfig+0xb2>
 8001e62:	687b      	ldr	r3, [r7, #4]
 8001e64:	4a2b      	ldr	r2, [pc, #172]	; (8001f14 <TIM_Base_SetConfig+0x11c>)
 8001e66:	4293      	cmp	r3, r2
 8001e68:	d01f      	beq.n	8001eaa <TIM_Base_SetConfig+0xb2>
 8001e6a:	687b      	ldr	r3, [r7, #4]
 8001e6c:	4a2a      	ldr	r2, [pc, #168]	; (8001f18 <TIM_Base_SetConfig+0x120>)
 8001e6e:	4293      	cmp	r3, r2
 8001e70:	d01b      	beq.n	8001eaa <TIM_Base_SetConfig+0xb2>
 8001e72:	687b      	ldr	r3, [r7, #4]
 8001e74:	4a29      	ldr	r2, [pc, #164]	; (8001f1c <TIM_Base_SetConfig+0x124>)
 8001e76:	4293      	cmp	r3, r2
 8001e78:	d017      	beq.n	8001eaa <TIM_Base_SetConfig+0xb2>
 8001e7a:	687b      	ldr	r3, [r7, #4]
 8001e7c:	4a28      	ldr	r2, [pc, #160]	; (8001f20 <TIM_Base_SetConfig+0x128>)
 8001e7e:	4293      	cmp	r3, r2
 8001e80:	d013      	beq.n	8001eaa <TIM_Base_SetConfig+0xb2>
 8001e82:	687b      	ldr	r3, [r7, #4]
 8001e84:	4a27      	ldr	r2, [pc, #156]	; (8001f24 <TIM_Base_SetConfig+0x12c>)
 8001e86:	4293      	cmp	r3, r2
 8001e88:	d00f      	beq.n	8001eaa <TIM_Base_SetConfig+0xb2>
 8001e8a:	687b      	ldr	r3, [r7, #4]
 8001e8c:	4a26      	ldr	r2, [pc, #152]	; (8001f28 <TIM_Base_SetConfig+0x130>)
 8001e8e:	4293      	cmp	r3, r2
 8001e90:	d00b      	beq.n	8001eaa <TIM_Base_SetConfig+0xb2>
 8001e92:	687b      	ldr	r3, [r7, #4]
 8001e94:	4a25      	ldr	r2, [pc, #148]	; (8001f2c <TIM_Base_SetConfig+0x134>)
 8001e96:	4293      	cmp	r3, r2
 8001e98:	d007      	beq.n	8001eaa <TIM_Base_SetConfig+0xb2>
 8001e9a:	687b      	ldr	r3, [r7, #4]
 8001e9c:	4a24      	ldr	r2, [pc, #144]	; (8001f30 <TIM_Base_SetConfig+0x138>)
 8001e9e:	4293      	cmp	r3, r2
 8001ea0:	d003      	beq.n	8001eaa <TIM_Base_SetConfig+0xb2>
 8001ea2:	687b      	ldr	r3, [r7, #4]
 8001ea4:	4a23      	ldr	r2, [pc, #140]	; (8001f34 <TIM_Base_SetConfig+0x13c>)
 8001ea6:	4293      	cmp	r3, r2
 8001ea8:	d108      	bne.n	8001ebc <TIM_Base_SetConfig+0xc4>
  {
    /* Set the clock division */
    tmpcr1 &= ~TIM_CR1_CKD;
 8001eaa:	68fb      	ldr	r3, [r7, #12]
 8001eac:	f423 7340 	bic.w	r3, r3, #768	; 0x300
 8001eb0:	60fb      	str	r3, [r7, #12]
    tmpcr1 |= (uint32_t)Structure->ClockDivision;
 8001eb2:	683b      	ldr	r3, [r7, #0]
 8001eb4:	68db      	ldr	r3, [r3, #12]
 8001eb6:	68fa      	ldr	r2, [r7, #12]
 8001eb8:	4313      	orrs	r3, r2
 8001eba:	60fb      	str	r3, [r7, #12]
  }

  /* Set the auto-reload preload */
  MODIFY_REG(tmpcr1, TIM_CR1_ARPE, Structure->AutoReloadPreload);
 8001ebc:	68fb      	ldr	r3, [r7, #12]
 8001ebe:	f023 0280 	bic.w	r2, r3, #128	; 0x80
 8001ec2:	683b      	ldr	r3, [r7, #0]
 8001ec4:	695b      	ldr	r3, [r3, #20]
 8001ec6:	4313      	orrs	r3, r2
 8001ec8:	60fb      	str	r3, [r7, #12]

  TIMx->CR1 = tmpcr1;
 8001eca:	687b      	ldr	r3, [r7, #4]
 8001ecc:	68fa      	ldr	r2, [r7, #12]
 8001ece:	601a      	str	r2, [r3, #0]

  /* Set the Autoreload value */
  TIMx->ARR = (uint32_t)Structure->Period ;
 8001ed0:	683b      	ldr	r3, [r7, #0]
 8001ed2:	689a      	ldr	r2, [r3, #8]
 8001ed4:	687b      	ldr	r3, [r7, #4]
 8001ed6:	62da      	str	r2, [r3, #44]	; 0x2c

  /* Set the Prescaler value */
  TIMx->PSC = Structure->Prescaler;
 8001ed8:	683b      	ldr	r3, [r7, #0]
 8001eda:	681a      	ldr	r2, [r3, #0]
 8001edc:	687b      	ldr	r3, [r7, #4]
 8001ede:	629a      	str	r2, [r3, #40]	; 0x28

  if (IS_TIM_REPETITION_COUNTER_INSTANCE(TIMx))
 8001ee0:	687b      	ldr	r3, [r7, #4]
 8001ee2:	4a0a      	ldr	r2, [pc, #40]	; (8001f0c <TIM_Base_SetConfig+0x114>)
 8001ee4:	4293      	cmp	r3, r2
 8001ee6:	d003      	beq.n	8001ef0 <TIM_Base_SetConfig+0xf8>
 8001ee8:	687b      	ldr	r3, [r7, #4]
 8001eea:	4a0c      	ldr	r2, [pc, #48]	; (8001f1c <TIM_Base_SetConfig+0x124>)
 8001eec:	4293      	cmp	r3, r2
 8001eee:	d103      	bne.n	8001ef8 <TIM_Base_SetConfig+0x100>
  {
    /* Set the Repetition Counter value */
    TIMx->RCR = Structure->RepetitionCounter;
 8001ef0:	683b      	ldr	r3, [r7, #0]
 8001ef2:	691a      	ldr	r2, [r3, #16]
 8001ef4:	687b      	ldr	r3, [r7, #4]
 8001ef6:	631a      	str	r2, [r3, #48]	; 0x30
  }

  /* Generate an update event to reload the Prescaler
     and the repetition counter (only for advanced timer) value immediately */
  TIMx->EGR = TIM_EGR_UG;
 8001ef8:	687b      	ldr	r3, [r7, #4]
 8001efa:	2201      	movs	r2, #1
 8001efc:	615a      	str	r2, [r3, #20]
}
 8001efe:	bf00      	nop
 8001f00:	3714      	adds	r7, #20
 8001f02:	46bd      	mov	sp, r7
 8001f04:	f85d 7b04 	ldr.w	r7, [sp], #4
 8001f08:	4770      	bx	lr
 8001f0a:	bf00      	nop
 8001f0c:	40010000 	.word	0x40010000
 8001f10:	40000400 	.word	0x40000400
 8001f14:	40000800 	.word	0x40000800
 8001f18:	40000c00 	.word	0x40000c00
 8001f1c:	40010400 	.word	0x40010400
 8001f20:	40014000 	.word	0x40014000
 8001f24:	40014400 	.word	0x40014400
 8001f28:	40014800 	.word	0x40014800
 8001f2c:	40001800 	.word	0x40001800
 8001f30:	40001c00 	.word	0x40001c00
 8001f34:	40002000 	.word	0x40002000

08001f38 <HAL_TIMEx_CommutCallback>:
  * @brief  Hall commutation changed callback in non-blocking mode
  * @param  htim TIM handle
  * @retval None
  */
__weak void HAL_TIMEx_CommutCallback(TIM_HandleTypeDef *htim)
{
 8001f38:	b480      	push	{r7}
 8001f3a:	b083      	sub	sp, #12
 8001f3c:	af00      	add	r7, sp, #0
 8001f3e:	6078      	str	r0, [r7, #4]
  UNUSED(htim);

  /* NOTE : This function should not be modified, when the callback is needed,
            the HAL_TIMEx_CommutCallback could be implemented in the user file
   */
}
 8001f40:	bf00      	nop
 8001f42:	370c      	adds	r7, #12
 8001f44:	46bd      	mov	sp, r7
 8001f46:	f85d 7b04 	ldr.w	r7, [sp], #4
 8001f4a:	4770      	bx	lr

08001f4c <HAL_TIMEx_BreakCallback>:
  * @brief  Hall Break detection callback in non-blocking mode
  * @param  htim TIM handle
  * @retval None
  */
__weak void HAL_TIMEx_BreakCallback(TIM_HandleTypeDef *htim)
{
 8001f4c:	b480      	push	{r7}
 8001f4e:	b083      	sub	sp, #12
 8001f50:	af00      	add	r7, sp, #0
 8001f52:	6078      	str	r0, [r7, #4]
  UNUSED(htim);

  /* NOTE : This function should not be modified, when the callback is needed,
            the HAL_TIMEx_BreakCallback could be implemented in the user file
   */
}
 8001f54:	bf00      	nop
 8001f56:	370c      	adds	r7, #12
 8001f58:	46bd      	mov	sp, r7
 8001f5a:	f85d 7b04 	ldr.w	r7, [sp], #4
 8001f5e:	4770      	bx	lr

08001f60 <HAL_MultiProcessor_Init>:
  *            @arg UART_WAKEUPMETHOD_IDLELINE: Wake-up by an idle line detection
  *            @arg UART_WAKEUPMETHOD_ADDRESSMARK: Wake-up by an address mark
  * @retval HAL status
  */
HAL_StatusTypeDef HAL_MultiProcessor_Init(UART_HandleTypeDef *huart, uint8_t Address, uint32_t WakeUpMethod)
{
 8001f60:	b580      	push	{r7, lr}
 8001f62:	b084      	sub	sp, #16
 8001f64:	af00      	add	r7, sp, #0
 8001f66:	60f8      	str	r0, [r7, #12]
 8001f68:	460b      	mov	r3, r1
 8001f6a:	607a      	str	r2, [r7, #4]
 8001f6c:	72fb      	strb	r3, [r7, #11]
  /* Check the UART handle allocation */
  if (huart == NULL)
 8001f6e:	68fb      	ldr	r3, [r7, #12]
 8001f70:	2b00      	cmp	r3, #0
 8001f72:	d101      	bne.n	8001f78 <HAL_MultiProcessor_Init+0x18>
  {
    return HAL_ERROR;
 8001f74:	2301      	movs	r3, #1
 8001f76:	e05f      	b.n	8002038 <HAL_MultiProcessor_Init+0xd8>
  assert_param(IS_UART_WAKEUPMETHOD(WakeUpMethod));
  assert_param(IS_UART_ADDRESS(Address));
  assert_param(IS_UART_WORD_LENGTH(huart->Init.WordLength));
  assert_param(IS_UART_OVERSAMPLING(huart->Init.OverSampling));

  if (huart->gState == HAL_UART_STATE_RESET)
 8001f78:	68fb      	ldr	r3, [r7, #12]
 8001f7a:	f893 303d 	ldrb.w	r3, [r3, #61]	; 0x3d
 8001f7e:	b2db      	uxtb	r3, r3
 8001f80:	2b00      	cmp	r3, #0
 8001f82:	d106      	bne.n	8001f92 <HAL_MultiProcessor_Init+0x32>
  {
    /* Allocate lock resource and initialize it */
    huart->Lock = HAL_UNLOCKED;
 8001f84:	68fb      	ldr	r3, [r7, #12]
 8001f86:	2200      	movs	r2, #0
 8001f88:	f883 203c 	strb.w	r2, [r3, #60]	; 0x3c

    /* Init the low level hardware */
    huart->MspInitCallback(huart);
#else
    /* Init the low level hardware : GPIO, CLOCK */
    HAL_UART_MspInit(huart);
 8001f8c:	68f8      	ldr	r0, [r7, #12]
 8001f8e:	f7fe fca3 	bl	80008d8 <HAL_UART_MspInit>
#endif /* (USE_HAL_UART_REGISTER_CALLBACKS) */
  }

  huart->gState = HAL_UART_STATE_BUSY;
 8001f92:	68fb      	ldr	r3, [r7, #12]
 8001f94:	2224      	movs	r2, #36	; 0x24
 8001f96:	f883 203d 	strb.w	r2, [r3, #61]	; 0x3d

  /* Disable the peripheral */
  __HAL_UART_DISABLE(huart);
 8001f9a:	68fb      	ldr	r3, [r7, #12]
